:020000040800F2
:1000000000500020651601080000000000000000FC
:1000100099160108991601089916010800000000B8
:100020000000000000000000000000009916010818
:100030009916010800000000991601082D07010813
:1000400099160108991601089916010899160108D0
:1000500099160108991601089916010899160108C0
:1000600099160108991601089916010899160108B0
:1000700099160108991601089916010899160108A0
:100080009916010899160108991601089916010890
:100090009916010899160108991601089916010880
:1000A0009916010899160108991601089916010870
:1000B000CD0F0108CD0D0108991601089916010808
:1000C0009916010899160108991601089916010850
:1000D00099160108390C01089916010899160108AA
:1000E00099160108991601089916010800000000E8
:1000F0000000000000000000000000000000000000
:1001000000000000000000005FF808F181F00041ED
:1001100002E000BF83F0004330B54FEA41044FEAEC
:10012000430594EA050F08BF90EA020F1FBF54EA87
:10013000000C55EA020C7FEA645C7FEA655C00F023
:10014000E2804FEA5454D4EB5555B8BF6D420CDDF4
:100150002C4480EA020281EA030382EA000083EA77
:10016000010180EA020281EA0303362D88BF30BD17
:1001700011F0004F4FEA01314FF4801C4CEA11316D
:1001800002D0404261EB410113F0004F4FEA0333CC
:100190004CEA133302D0524263EB430394EA050F57
:1001A00000F0A780A4F10104D5F1200E0DDB02FAC6
:1001B0000EFC22FA05F2801841F1000103FA0EF25A
:1001C000801843FA05F359410EE0A5F120050EF120
:1001D000200E012A03FA0EFC28BF4CF0020C43FA51
:1001E00005F3C01851EBE37101F0004507D54FF05E
:1001F000000EDCF1000C7EEB00006EEB0101B1F5AE
:10020000801F1BD3B1F5001F0CD349085FEA3000F3
:100210004FEA3C0C04F101044FEA445212F5800FFE
:1002200080F09A80BCF1004F08BF5FEA500C50F19B
:10023000000041EB045141EA050130BD5FEA4C0C7E
:10024000404141EB010111F4801FA4F10104E9D107
:1002500091F0000F04BF01460020B1FA81F308BFFE
:100260002033A3F10B03B3F120020CDA0C3208DDCA
:1002700002F1140CC2F10C0201FA0CF021FA02F1A5
:100280000CE002F11402D8BFC2F1200C01FA02F115
:1002900020FA0CFCDCBF41EA0C019040E41AA2BF3A
:1002A00001EB0451294330BD6FEA04041F3C1CDA02
:1002B0000C340EDC04F11404C4F1200220FA04F022
:1002C00001FA02F340EA030021FA04F345EA0301CC
:1002D00030BDC4F10C04C4F1200220FA02F001FA8E
:1002E00004F340EA0300294630BD21FA04F0294610
:1002F00030BD94F0000F83F4801306BF81F48011A9
:100300000134013D4EE77FEA645C18BF7FEA655C1B
:1003100029D094EA050F08BF90EA020F05D054EAED
:10032000000C04BF1946104630BD91EA030F1EBFF2
:100330000021002030BD5FEA545C05D140004941F6
:1003400028BF41F0004130BD14F580043CBF01F5E9
:10035000801130BD01F0004545F0FE4141F47001CF
:100360004FF0000030BD7FEA645C1ABF19461046AA
:100370007FEA655C1CBF0B46024650EA013406BFAB
:1003800052EA033591EA030F41F4002130BD00BF6A
:1003900090F0000F04BF0021704730B54FF4806427
:1003A00004F132044FF000054FF0000150E700BFA8
:1003B00090F0000F04BF0021704730B54FF4806407
:1003C00004F1320410F0004548BF40424FF00001F4
:1003D0003EE700BF42004FEAE2014FEA31014FEA37
:1003E00002701FBF12F07F4393F07F4F81F0605186
:1003F000704792F0000F14BF93F07F4F704730B5F5
:100400004FF4607401F0004521F0004120E700BF87
:1004100050EA010208BF704730B54FF000050AE00E
:1004200050EA010208BF704730B511F0004502D50F
:10043000404261EB41014FF4806404F132045FEA11
:10044000915C3FF4DCAE4FF003025FEADC0C18BFB6
:1004500003325FEADC0C18BF033202EBDC02C2F1AC
:10046000200300FA03FC20FA02F001FA03FE40EA3E
:100470000E0021FA02F11444C1E600BF70B54FF03E
:10048000FF0C4CF4E06C1CEA11541DBF1CEA135520
:1004900094EA0C0F95EA0C0F00F0DEF82C4481EA88
:1004A000030621EA4C5123EA4C5350EA013518BFA8
:1004B00052EA033541F4801143F4801338D0A0FB95
:1004C00002CE4FF00005E1FB02E506F00042E0FB42
:1004D00003E54FF00006E1FB03569CF0000F18BF48
:1004E0004EF0010EA4F1FF04B6F5007F64F54074F0
:1004F00004D25FEA4E0E6D4146EB060642EAC62183
:1005000041EA55514FEAC52040EA5E504FEACE2EEF
:10051000B4F1FD0C88BFBCF5E06F1ED8BEF1004FF2
:1005200008BF5FEA500E50F1000041EB045170BD6E
:1005300006F0004646EA010140EA020081EA0301B2
:10054000B4EB5C04C2BFD4EB0C0541EA045170BDAE
:1005500041F480114FF0000E013C00F3AB8014F128
:10056000360FDEBF002001F0004170BDC4F1000471
:10057000203C35DA0C341BDC04F11404C4F12005F2
:1005800000FA05F320FA04F001FA05F240EA02004D
:1005900001F0004221F0004110EBD37021FA04F683
:1005A00042EB06015EEA430E08BF20EAD37070BD3D
:1005B000C4F10C04C4F1200500FA04F320FA05F09C
:1005C00001FA04F240EA020001F0004110EBD3709E
:1005D00041F100015EEA430E08BF20EAD37070BD0E
:1005E000C4F1200500FA05F24EEA020E20FA04F3E7
:1005F00001FA05F243EA020321FA04F001F0004196
:1006000021FA04F220EA020000EBD3705EEA430E06
:1006100008BF20EAD37070BD94F0000F0FD101F035
:100620000046400041EB010111F4801F08BF013C6E
:10063000F7D041EA060195F0000F18BF704703F0AC
:100640000046520043EB030313F4801F08BF013D33
:10065000F7D043EA0603704794EA0C0F0CEA1355EF
:1006600018BF95EA0C0F0CD050EA410618BF52EAA9
:100670004306D1D181EA030101F000414FF00000AF
:1006800070BD50EA410606BF1046194652EA4306BD
:1006900019D094EA0C0F02D150EA013613D195EA31
:1006A0000C0F05D152EA03361CBF104619460AD179
:1006B00081EA030101F0004141F0FE4141F4700183
:1006C0004FF0000070BD41F0FE4141F4780170BD73
:1006D00070B54FF0FF0C4CF4E06C1CEA11541DBFD8
:1006E0001CEA135594EA0C0F95EA0C0F00F0A7F8DA
:1006F000A4EB050481EA030E52EA03354FEA013107
:1007000000F088804FEA03334FF0805545EA131319
:1007100043EA12634FEA022245EA111545EA1065E1
:100720004FEA00260EF000419D4208BF964244F178
:10073000FD0404F5407402D25B084FEA3202B61A97
:1007400065EB03055B084FEA32024FF480104FF46B
:10075000002CB6EB020E75EB030E22BFB61A7546DF
:1007600040EA0C005B084FEA3202B6EB020E75EB72
:10077000030E22BFB61A754640EA5C005B084FEADA
:100780003202B6EB020E75EB030E22BFB61A7546A7
:1007900040EA9C005B084FEA3202B6EB020E75EBB2
:1007A000030E22BFB61A754640EADC0055EA060E73
:1007B00018D04FEA051545EA16754FEA06164FEAB6
:1007C000C30343EA52734FEAC2025FEA1C1CC0D162
:1007D00011F4801F0BD141EA00014FF000004FF0EF
:1007E000004CB6E711F4801F04BF01430020B4F1B0
:1007F000FD0C88BFBCF5E06F3FF6AFAEB5EB030C68
:1008000004BFB6EB020C5FEA500C50F1000041EB64
:10081000045170BD0EF0004E4EEA113114EB5C0431
:10082000C2BFD4EB0C0541EA045170BD41F4801104
:100830004FF0000E013C90E645EA060E8DE60CEA0C
:10084000135594EA0C0F08BF95EA0C0F3FF43BAF29
:1008500094EA0C0F0AD150EA01347FF434AF95EAE0
:100860000C0F7FF425AF104619462CE795EA0C0FC4
:1008700006D152EA03353FF4FDAE1046194622E791
:1008800050EA410618BF52EA43067FF4C5AE50EA6B
:1008900041047FF40DAF52EA43057FF4EBAE12E75B
:1008A0004FF0FF3C06E000BF4FF0010C02E000BF3C
:1008B0004FF0010C4DF804CD4FEA410C7FEA6C5C1F
:1008C0004FEA430C18BF7FEA6C5C1BD001B050EAC2
:1008D000410C0CBF52EA430C91EA030F02BF90EAAD
:1008E000020F0020704710F1000F91EA030F58BF6C
:1008F000994208BF90422CBFD8176FEAE37040F0CE
:10090000010070474FEA410C7FEA6C5C02D150EA6B
:10091000013C07D14FEA430C7FEA6C5CD6D152EA26
:10092000033CD3D05DF8040B704700BF84461046EB
:1009300062468C461946634600E000BF01B5FFF7EA
:10094000B7FF002848BF10F1000F01BD4DF808EDBA
:10095000FFF7F4FF0CBF012000205DF808FB00BF8B
:100960004DF808EDFFF7EAFF34BF012000205DF8E5
:1009700008FB00BF4DF808EDFFF7E0FF94BF012032
:1009800000205DF808FB00BF4DF808EDFFF7CEFF33
:1009900094BF012000205DF808FB00BF4DF808ED72
:1009A000FFF7C4FF34BF012000205DF808FB00BF43
:1009B0004FEA410212F5001215D211D56FF4787387
:1009C000B3EB625212D94FEAC12343F0004343EA2A
:1009D000505311F0004F23FA02F018BF4042704705
:1009E0004FF00000704750EA013005D111F000408F
:1009F00008BF6FF0004070474FF00000704700BF25
:100A00004A0011D212F5001211D20DD56FF478738D
:100A1000B3EB62520ED44FEAC12343F0004343EAE2
:100A2000505323FA02F070474FF00000704750EA2D
:100A3000013002D14FF0FF3070474FF00000704797
:100A40004FEA4102B2F1E04324BFB3F5001CDCF1F0
:100A5000FE5C0DD901F0004C4FEAC0024CEA507028
:100A6000B2F1004F40EB830008BF20F00100704757
:100A700011F0804F21D113F13872BCBF01F000405A
:100A8000704741F480114FEA5252C2F11802C2F18C
:100A9000200C10FA0CF320FA02F018BF40F001000D
:100AA0004FEAC1234FEAD32303FA0CFC40EA0C00BF
:100AB00023FA02F34FEA4303CCE77FEA625307D1FC
:100AC00050EA01331EBF4FF0FE4040F44000704733
:100AD00001F0004040F0FE4040F40000704700BFCD
:100AE00080F0004002E000BF81F0004142001FBFE3
:100AF0005FEA410392EA030F7FEA226C7FEA236CEC
:100B00006AD04FEA1262D2EB1363C1BFD2184140E0
:100B100048404140B8BF5B42192B88BF704710F076
:100B2000004F40F4000020F07F4018BF404211F019
:100B3000004F41F4000121F07F4118BF494292EA81
:100B4000030F3FD0A2F1010241FA03FC10EB0C00AD
:100B5000C3F1200301FA03F100F0004302D549423A
:100B600060EB4000B0F5000F13D3B0F1807F06D3E7
:100B700040084FEA310102F10102FE2A51D2B1F1DF
:100B8000004F40EBC25008BF20F0010040EA0300D4
:100B90007047490040EB000010F4000FA2F1010281
:100BA000EDD1B0FA80FCACF1080CB2EB0C0200FA0B
:100BB0000CF0AABF00EBC25052421843BCBFD04059
:100BC0001843704792F0000F81F4000106BF80F4D3
:100BD00000000132013BB5E74FEA41037FEA226C96
:100BE00018BF7FEA236C21D092EA030F04D092F061
:100BF000000F08BF0846704790EA010F1CBF002095
:100C0000704712F07F4F04D1400028BF40F00040F1
:100C1000704712F100723CBF00F50000704700F011
:100C2000004343F0FE4040F4000070477FEA226238
:100C300016BF08467FEA23630146420206BF5FEA09
:100C4000412390EA010F40F4800070474FF0000309
:100C500004E000BF10F0004348BF40425FEA000CD0
:100C600008BF704743F0964301464FF000001CE078
:100C700050EA010208BF70474FF000030AE000BFCE
:100C800050EA010208BF704711F0004302D540420C
:100C900061EB41015FEA010C02BF8446014600207E
:100CA00043F0B64308BFA3F18053A3F50003BCFA99
:100CB0008CF2083AA3EBC25310DB01FA02FC634446
:100CC00000FA02FCC2F12002BCF1004F20FA02F24D
:100CD00043EB020008BF20F00100704702F1200240
:100CE00001FA02FCC2F1200250EA4C0021FA02F2A1
:100CF00043EB020008BF20EADC7070474FF0FF0CA6
:100D00001CEAD0521EBF1CEAD15392EA0C0F93EAA0
:100D10000C0F6FD01A4480EA010C400218BF5FEA42
:100D200041211ED04FF0006343EA501043EA5111B5
:100D3000A0FB01310CF00040B1F5000F3EBF4900AF
:100D400041EAD3715B0040EA010062F17F02FD2AB3
:100D50001DD8B3F1004F40EBC25008BF20F0010096
:100D6000704790F0000F0CF0004C08BF49024CEAAD
:100D7000502040EA51207F3AC2BFD2F1FF0340EA3F
:100D8000C250704740F400004FF00003013A5DDCB0
:100D900012F1190FDCBF00F000407047C2F10002F1
:100DA000410021FA02F1C2F1200200FA02FC5FEADE
:100DB000310040F1000053EA4C0308BF20EADC7028
:100DC000704792F0000F00F0004C02BF400010F49A
:100DD000000F013AF9D040EA0C0093F0000F01F047
:100DE000004C02BF490011F4000F013BF9D041EA69
:100DF0000C018FE70CEAD15392EA0C0F18BF93EA6B
:100E00000C0F0AD030F0004C18BF31F0004CD8D194
:100E100080EA010000F00040704790F0000F17BF1B
:100E200090F0004F084691F0000F91F0004F14D061
:100E300092EA0C0F01D142020FD193EA0C0F03D1B9
:100E40004B0218BF084608D180EA010000F00040BC
:100E500040F0FE4040F40000704740F0FE4040F497
:100E6000400070474FF0FF0C1CEAD0521EBF1CEA36
:100E7000D15392EA0C0F93EA0C0F69D0A2EB030254
:100E800080EA010C49024FEA402037D04FF08053EE
:100E900043EA111143EA10130CF000408B4238BFB3
:100EA0005B0042F17D024FF4000C8B4224BF5B1AC1
:100EB00040EA0C00B3EB510F24BFA3EB510340EA0F
:100EC0005C00B3EB910F24BFA3EB910340EA9C00BD
:100ED000B3EBD10F24BFA3EBD10340EADC001B012D
:100EE00018BF5FEA1C1CE0D1FD2A3FF650AF8B42D1
:100EF00040EBC25008BF20F0010070470CF0004CDE
:100F00004CEA50207F32C2BFD2F1FF0340EAC25008
:100F1000704740F400004FF00003013A37E792F0C9
:100F2000000F00F0004C02BF400010F4000F013A27
:100F3000F9D040EA0C0093F0000F01F0004C02BF22
:100F4000490011F4000F013BF9D041EA0C0195E78B
:100F50000CEAD15392EA0C0F08D142027FF47DAF24
:100F600093EA0C0F7FF470AF084676E793EA0C0F14
:100F700004D14B023FF44CAF08466EE730F0004C12
:100F800018BF31F0004CCAD130F000427FF45CAFA2
:100F900031F000437FF43CAF5FE700BF4FF0FF3C10
:100FA00006E000BF4FF0010C02E000BF4FF0010C63
:100FB0004DF804CD4FEA40024FEA41037FEA226C2C
:100FC00018BF7FEA236C11D001B052EA530C18BF4E
:100FD00090EA010F58BFB2EB030088BFC81738BFB3
:100FE0006FEAE17018BF40F0010070477FEA226CA1
:100FF00002D15FEA402C05D17FEA236CE4D15FEA9D
:10100000412CE1D05DF8040B704700BF84460846D0
:101010006146FFE70FB5FFF7C9FF002848BF10F191
:10102000000F0FBD4DF808EDFFF7F4FF0CBF0120D6
:1010300000205DF808FB00BF4DF808EDFFF7EAFF60
:1010400034BF012000205DF808FB00BF4DF808ED1B
:10105000FFF7E0FF94BF012000205DF808FB00BF10
:101060004DF808EDFFF7D2FF94BF012000205DF896
:1010700008FB00BF4DF808EDFFF7C8FF34BF0120A3
:1010800000205DF808FB00BF4FEA4002B2F1FE4FBE
:101090000FD34FF09E03B3EB12620DD94FEA00233A
:1010A00043F0004310F0004F23FA02F018BF404213
:1010B00070474FF00000704712F1610F01D14202FA
:1010C00005D110F0004008BF6FF0004070474FF0AE
:1010D0000000704700210A2200F0C2B900220A2352
:1010E00000F00CB9032AC9B270B408D82AB103467B
:1010F000121803F8011B9342FBD170BC7047821891
:10110000044601E004F8011B14F0030FFAD14FF07C
:10111000013303FB01F31FE044F8403C44F83C3C3E
:1011200044F8383C44F8343C44F8303C44F82C3C17
:1011300044F8283C44F8243C44F8203C44F81C3C47
:1011400044F8183C44F8143C44F8103C44F80C3C77
:1011500044F8083C44F8043C161B254640343F2E16
:10116000DADC2C4607E044F8103C44F80C3C44F828
:10117000083C44F8043C161B254610340F2EF2DCC4
:1011800001E045F8043B541B032CFADC01E005F8B0
:10119000011B9542FBD3B0E710F0030F38B50446AE
:1011A00012D10368A3F1013222EA030313F0803F56
:1011B0000AD1031D184653F8042BA2F1013525EA84
:1011C000020212F0803FF5D003782BB1431C184681
:1011D00013F8012B002AFAD100F002F8204638BD9E
:1011E00080EA0102844612F0030F4FD111F0030F81
:1011F00032D14DF8044D11F0040F51F8043B0BD0DF
:10120000A3F101329A4312F0803F04BF4CF8043B33
:1012100051F8043B16D100BF51F8044BA3F1013241
:101220009A4312F0803FA4F101320BD14CF8043BF9
:10123000A24312F0803F04BF51F8043B4CF8044B2A
:10124000EAD023460CF8013B13F0FF0F4FEA33239B
:10125000F8D15DF8044B704711F0010F06D011F87A
:10126000012B0CF8012B002A08BF704711F0020F68
:10127000BFD031F8022B12F0FF0F16BF2CF8022B53
:101280008CF8002012F47F4FB3D1704711F8012B76
:101290000CF8012B002AF9D1704700BF20F00301A0
:1012A00010F00300C0F1000051F8043B00F1040C01
:1012B0004FEACC0C6FF000021CBF22FA0CF2134371
:1012C0004FF0010C4CEA0C2C4CEA0C4CA3EB0C023A
:1012D00022EA030212EACC1204BF51F8043B0430A4
:1012E000F4D013F0FF0F1FBF013013F47F4F013014
:1012F00013F47F0F18BF0130704700BF2DE9F04F86
:1013000040F20424C2F2000485B01F468C462668D1
:101310000B460390029213F8014B32191D4692F8C6
:1013200001B01BF0080BF6D12D2C73D02B2C08BF6D
:1013300015F8014BD7F1010338BF0023102F14BF5C
:101340001A4643F0010232B1302C73D01BB1302C5D
:1013500000F083800A27B946BBF1000F49460CBF55
:101360006FF0004A4FF0004ACDF804C0504600F03C
:10137000B1F950468846494600F07EF833190022FC
:10138000DDF804C05B78114613F0040F1ED0303C2A
:10139000A74225DD814294BF0023012353EAD27284
:1013A0002ED10A1A534243EB02034445D4BF002313
:1013B00003F00103002B23D109FB014115F8014B78
:1013C000012233195B7813F0040FE0D113F003030B
:1013D00006D0012B14BF57233723E41AA742D9DCC8
:1013E000B2F1FF3F1BD00846BBF1000F10D1029BAA
:1013F0001BB152B90299C1F800C005B0BDE8F08F29
:101400004FF0FF3215F8014BDBE705F1FF3CF1E748
:101410004842ECE715F8014B4FF0010B8AE70399BE
:10142000BBF1000F0CBF6FF000404FF000402223D3
:101430000B60DCE72A78A2F17800414241EB000121
:10144000582A14BF0A4641F00102002A3FF47EAF39
:1014500010276C78B94602357EE70827B9467BE746
:1014600030B440F20824C2F200040D46134601468F
:101470002A46206830BC41E74A1E08BF7047C0F0CA
:101480002481884240F21681114200F01781B0FA9F
:1014900080F3B1FA81F2A2EB0303C3F11F0304A2AC
:1014A00002EB03134FF000029F4600BFAFF3008032
:1014B000B0EBC17F00BF42EB020228BFA0EBC170BE
:1014C000B0EB817F00BF42EB020228BFA0EB81702E
:1014D000B0EB417F00BF42EB020228BFA0EB41709E
:1014E000B0EB017F00BF42EB020228BFA0EB01700E
:1014F000B0EBC16F00BF42EB020228BFA0EBC1609E
:10150000B0EB816F00BF42EB020228BFA0EB81600D
:10151000B0EB416F00BF42EB020228BFA0EB41607D
:10152000B0EB016F00BF42EB020228BFA0EB0160ED
:10153000B0EBC15F00BF42EB020228BFA0EBC1507D
:10154000B0EB815F00BF42EB020228BFA0EB8150ED
:10155000B0EB415F00BF42EB020228BFA0EB41505D
:10156000B0EB015F00BF42EB020228BFA0EB0150CD
:10157000B0EBC14F00BF42EB020228BFA0EBC1405D
:10158000B0EB814F00BF42EB020228BFA0EB8140CD
:10159000B0EB414F00BF42EB020228BFA0EB41403D
:1015A000B0EB014F00BF42EB020228BFA0EB0140AD
:1015B000B0EBC13F00BF42EB020228BFA0EBC1303D
:1015C000B0EB813F00BF42EB020228BFA0EB8130AD
:1015D000B0EB413F00BF42EB020228BFA0EB41301D
:1015E000B0EB013F00BF42EB020228BFA0EB01308D
:1015F000B0EBC12F00BF42EB020228BFA0EBC1201D
:10160000B0EB812F00BF42EB020228BFA0EB81208C
:10161000B0EB412F00BF42EB020228BFA0EB4120FC
:10162000B0EB012F00BF42EB020228BFA0EB01206C
:10163000B0EBC11F00BF42EB020228BFA0EBC110FC
:10164000B0EB811F00BF42EB020228BFA0EB81106C
:10165000B0EB411F00BF42EB020228BFA0EB4110DC
:10166000B0EB011F00BF42EB020228BFA0EB01104C
:10167000B0EBC10F00BF42EB020228BFA0EBC100DC
:10168000B0EB810F00BF42EB020228BFA0EB81004C
:10169000B0EB410F00BF42EB020228BFA0EB4100BC
:1016A000B0EB010F00BF42EB020228BFA0EB01002C
:1016B000104670470CBF012000207047B1FA81F23C
:1016C000C2F11F0220FA02F0704708B14FF0FF305C
:1016D00000F00EB80029F8D02DE90340FFF7CCFE4A
:1016E000BDE8064002FB00F3A1EB0301704700BF19
:1016F000704700BFFF230370FF3B83706433437068
:101700007047FF230370F53B83705A334370643B8B
:10171000C370704738B50025044645700E4B043041
:1017200098470E4B04F108009847FF23642223706A
:1017300023736273A373E27323746274A374E274F9
:10174000072395FBF3F3643BC835237563750434B5
:10175000B5F5C86FF4D138BD03170008F5160008B9
:1017600037B50D4B04460D4998470D4B2046984719
:101770000C4B201819780C4D4A1C1A7001230022BA
:1017800000931346A847002323826382A382A37594
:10179000E3750023A3613EBDE1110008D4210108D7
:1017A0009D120008FD020020F523000837B5114BFB
:1017B0000446114998472046104B9847104B201873
:1017C0001978104D4A1C1A70002201230093134609
:1017D000A84700222282A274E27422756275A27563
:1017E000E27522766276A276E27604F11C00064B60
:1017F00098473EBDE1110008E02101089D12000854
:1018000000030020F5230008F516000800230370EC
:1018100043708370C370704770B5FF230025044682
:1018200043700570074B8570C57004309847064EAD
:1018300004F10800B04704F10C00B047258265822E
:1018400070BD00BF03170008F5160008FF2310B590
:101850000370FF3B044643708370C3700430034B36
:10186000984704F10800024B984710BD0317000881
:10187000F5160008FF2310B50370FF3B04464370C4
:101880008370C3700430034B984704F10800024B87
:10189000984710BD03170008F516000838B5FF2358
:1018A0000370FF3B044643708370C3700430054BE4
:1018B0009847054D04F10800A84704F10C00A8471B
:1018C00038BD00BF03170008F516000838B5FF2320
:1018D0000370FF3B044643708370C3700430054BB4
:1018E0009847054D04F10800A84704F10C00A847EB
:1018F00038BD00BF03170008F516000837B50D4BBB
:1019000004460D49984720460C4B98470C4B20182D
:1019100019780C4D4A1C1A700123002200931346BB
:10192000A84700232382A374E37404F11400064B38
:1019300098473EBDE1110008E72101089D1200080B
:10194000FE020020F5230008F516000800230370AE
:1019500043708370C3708380C3800381438100F12F
:1019600020030022828102309842FAD1704700237E
:1019700043708370C370C21802330021202B918002
:10198000F9D170470023037043708370C3707047B0
:1019900038B50446124DA847201DA84704F1080099
:1019A000A84704F10C00A847002525746574A574A8
:1019B000E57425756575A575E57504F11800094B85
:1019C000984725776577A577E5772584658484F83A
:1019D000245084F8255084F8265084F8275038BDC8
:1019E00085190008F51600082DE9F74F0024064672
:1019F00046F8044B05463A4F3A493046B847DFF8B7
:101A0000EC803046C047384E281831784FF0010935
:101A10004B1CDFF8DCA02246337005F1140B234683
:101A20000430CDF80090D0472E495846B847584664
:101A3000C0473178281801EB09032246337005F1BD
:101A4000240B23461430CDF80090D0472549584642
:101A5000B8475846C0473178281801EB0903224699
:101A6000337005F1340B23462430CDF80090D04775
:101A70001C495846B8475846C0473178281801EBEA
:101A800009032246337005F1440B23463430CDF868
:101A90000090D04713495846B8475846C047317858
:101AA000281801EB09032246337005F5A27B234673
:101AB0004430CDF80090D0470A495846B8475846B8
:101AC000C0473178281801EB0903337022462346BA
:101AD00000F5A270CDF80090D047BDE8FE8F00BFA2
:101AE000E1110008EF210108FF0200209D1200080B
:101AF000F52300080023038043808380C380704760
:101B000038B50546002405EBC400034B0134984763
:101B1000042CF8D138BD00BFF51A0008002343702B
:101B2000C3704371C371704770B5002504460560EA
:101B3000057145718571C571A81C04EB80002E4BA1
:101B400001359847102DF7D1103D0C2000FB0540C2
:101B50002A4B483001359847102DF6D1103D0C2006
:101B600000FB0540264B00F5847001359847102D89
:101B7000F5D1103D142000FB0540224B00F5E47028
:101B800001359847102DF5D1103D342000FB05405C
:101B90001D4B00F5427001359847402DF5D1403D71
:101BA000280100F5805008302018184B013598475F
:101BB000102DF5D1103D280100F58850083020186F
:101BC000134B01359847102DF5D104F5905606F1C9
:101BD0000800104DA84706F13400A84704F59350BB
:101BE0000D4D04F59454A847201DA84704F1280082
:101BF0000A4B984770BD00BF0D1800084D1800082B
:101C00007518000819180008151700089D18000815
:101C1000CD1800084D1900086F1900081D1B000899
:101C20000023037043708370C370704710B5054B79
:101C3000044698470022A280E28022726272A27259
:101C4000E27210BD0317000870B500260446044D6B
:101C500040F8046BA847A66004F10C00A84770BDCB
:101C6000031700082DE9F34704463049304FB847C1
:101C7000304E2046B047304D002229784FF0010801
:101C80004B1C2B70DFF8CC90134604F1180A201877
:101C9000CDF80080C84725495046B8475046B04760
:101CA0002978002201EB080318302B70201800253A
:101CB0001346CDF80080C84784F8285084F829508E
:101CC00084F82A5084F82B50680120182C301B4BC4
:101CD00001359847402DF7D1403D182000FB0540C5
:101CE00000F502600C30164B01359847402DF4D1B9
:101CF000403D1C2000FB054000F562600C30114B9C
:101D000001359847202DF4D104F58C502C3004F582
:101D100010540D4B984704F15C000C4B984704F1AC
:101D20006C000B4B9847BDE8FC8700BFF821010809
:101D3000E11100089D120008FC020020AD17000808
:101D4000FD18000861170008291B0008491C00083D
:101D50002D1C0008F523000810B5064B04469847D3
:101D600004F12000044B984704F14800034B9847C6
:101D700010BD00BF011B000891190008E9190008F7
:101D80000C4A002310B513700B4A044613700B4A1B
:101D900004F5105413700A4A13700A4A13700A4B60
:101DA000984704F17800094B984704F17C00084BF0
:101DB000984710BDFD02002000030020FE02002015
:101DC000FF020020FC020020651C0008211C000806
:101DD000591D00082DE9F04193F900406425E60201
:101DE000361B96FBF5F6541EB04213F8244001DC76
:101DF00030B207E064B2E602341B94FBF5F4A04273
:101E0000A8BF20B200262AE093F90040E5022D1B6E
:101E1000642495FBF4F5A8421FDB93F9047003F1E9
:101E2000040C4FEAC728C7EB080797FBF4F7B84242
:101E300013DC93F90130401BDA02D31A9CF901201C
:101E400093FBF4F3D602B21A92FBF4F4E41A604363
:101E50007F1B90FBF7F5ED1805E001360433541EA7
:101E6000A642D1DB00256943642391FBF3F000B265
:101E7000BDE8F0810378FF2B1AD0FE2B1AD0FD2B82
:101E800001D1407817E03F2B05D80C4A5B019B1825
:101E90009A7952B200E0002290F9023090F90100E4
:101EA0006432C01A5043C82190FBF1F0C01802E020
:101EB000002000E0642040B2704700BF0808002006
:101EC00002780346FF2A17D0FE2A13D03F2A13D8E0
:101ED0000E4952015218917990F9020049B2884294
:101EE0000ADC907993F9012040B28242B4BF00200D
:101EF000012002E0012000E0002093F90330012BD3
:101F000004BFC0F10100C0B2704700BF0808002044
:101F100010B5A0B00346ADF102040022114818210B
:101F200001FB020101F50261183189880132402A62
:101F300024F8021FF2D1303A182101FB0201B1F856
:101F40003C4802F58E513431013200EB4101202A28
:101F50000C81F1D1044A4021D06A6A46984720B0EA
:101F600010BD00BFD00700205019002008B5184848
:101F7000184B98471648184B00F59A510831984766
:101F80001348164B00F58E51083198471048144BF2
:101F900000F59451083198470D48124B00F5A452B2
:101FA000083200F5006198470F48104B00F5CC51FE
:101FB000083198470C480E4B00F5D451083198472A
:101FC00009480C4B98470C480C4B984708BD00BF7C
:101FD000FC070020A5240008D928000829270008AC
:101FE00091280008F9290008FC0F00207D2B00082B
:101FF000E92B0008612C00088D0D0108111F000855
:1020000010B500230D4A342101FB0322FE2402F502
:10201000A452FD2182F8343082F8384082F83C1016
:10202000FD3982F83E10643182F83D1082F840306C
:102030000133402B82F84110E4D110BDD0070020BD
:10204000F8B58D498D4C8E48A0478E498E48A047E3
:102050008E498F48A0478F498F48A0478F499048A5
:10206000A047904B42F2B962DA6200212746844BC6
:10207000142202FB0132FE2402F59A52013182F849
:10208000384000206425013C102982F83E0082F887
:102090003D5082F83C4082F8420082F8415082F87C
:1020A0004040E4D102460C2000FB0230FE2400F543
:1020B0008E5080F838400021D13C013280F83E102B
:1020C00080F83D40D034102A80F83C40EBD10C2001
:1020D00000FB0130FE2400F5945080F838400022C7
:1020E000B33C013180F83E2080F83D40B2341029E5
:1020F00080F83C40EBD1342101FB0231FE2401F594
:10210000A45181F8384000209A3C013281F83E0009
:1021100081F83D409934402A81F83C40EBD100F5EC
:1021200006720332FE2103EB0212117200F5807277
:10213000013203EB0212013002F58C52FE396425A4
:10214000FD24102882F82E1082F82D5082F82C40A1
:1021500082F8321082F8315082F83040DFD101F538
:102160000A720332FE2003EB0212107201F588722C
:10217000013203EB0212013102F58C52FE38642564
:10218000FD24102982F82E0082F82D5082F82C4070
:1021900082F8320082F8315082F83040DFD10246B6
:1021A0002C2000FB0230082400F50E5080F834404B
:1021B000073C80F8354080F836404FF49674048729
:1021C00040F2DC5484874FF47A7400F13001C48704
:1021D00042F6E06048810021162000FB021000F565
:1021E0008E501C300131002403EB40001029048183
:1021F000F2D10132022AD3D1023A242101FB023169
:10220000082001F51051C873F7304873FF38887300
:102210000146122000FB021000F5905004300131FD
:10222000002403EB400010290481F2D10132022A7C
:10223000E3D10020182101FB003101300022FD24F0
:10224000402881F8422881F8412881F84048F1D19E
:1022500051015918383101200872901C40010024A6
:1022600018184C7284724472FD34047250B2022801
:102270001ADC262019E000BF88220108E1110008BD
:10228000D007002099220108982C00209E220108E6
:10229000A82C002077470108D82C0020A422010890
:1022A000E80700205019002027200132402AC87179
:1022B000CED12B3A83F83F20013283F85F200132E0
:1022C00083F87F20013283F89F20464C183AFD2185
:1022D00083F84A2083F8492083F8481083F86A205D
:1022E00083F8692083F8681083F88A2083F88920AE
:1022F00083F8881083F8AA2083F8A92083F8A8100F
:102300002F3984F8551084F8571084F859109C39E7
:1023100084F85B10313984F8542084F85610013168
:1023200084F85810013184F85A10911C4901002595
:1023300059188D71510101325918402A81F83E50C7
:102340008D87F2D1284B9847012384F87830274CA9
:10235000322684F8433084F84130033384F8423025
:10236000FB33257784F82450657784F82550A577CA
:1023700084F8265084F8283084F8293084F82A30EC
:1023800084F8203084F8213084F82230F93B84F836
:102390002C300E3384F83B300C3B84F8393004F198
:1023A000780084F83A50124984F8383084F8406054
:1023B000B8471A236020A087E387262384F830607B
:1023C00084F832303E3384F8315084F8365084F843
:1023D0003530993384F834307D3B84F82D3084F8DF
:1023E0002E50F8BDD02B002001200008502C0020DA
:1023F000AC220108F0B5002985B005DA2D24494248
:10240000047009B22C3C00E0002400250BE04FF0E2
:102410000A0C91FBFCF70CFB17110135303106F863
:102420000C1CEDB239B204AF092907EB0506EEDC4E
:10243000303106F80C1C691C03E0302605F80C6CE2
:102440000131C9B204AE994206EB0105F5D99142BA
:10245000F3D3002205F80C2C0A460DE09A4203D172
:102460002E2101550134E4B204AFB91811F80D1C46
:10247000013A01550134E4B2002AEFD1025505B00A
:10248000F0BD000010B50024E0B2044B9847044BA7
:1024900023F814000134202CF6D110BDA90801083E
:1024A00058040020F0B5002585B004462F4694F965
:1024B0001530EEB2042B24D1043B2375A37D013BE0
:1024C000DBB2632B01D90123A375E17DA37DA27C3F
:1024D00051B958B251B24118632901DC9B183DE053
:1024E0006423A374633B0AE050B259B2411A11F15C
:1024F000630F01DBD31A31E09C23A3749C3BE3758B
:1025000063E094F914208AB9022B5ED194F9163055
:10251000002B5ED1A37C5AB2632A04DC142701335A
:102520005743A37455E00123A37552E0754A012B6C
:1025300032F815703FB213D117F5027F01DA9B33E1
:102540000CE0B7F5027F01DD642307E007F5F877BB
:10255000033740F2E6339F4237D80023A37434E0B8
:10256000022B14D117F1640F05DAA37C5AB212F1D1
:10257000630F2ADB05E0642F27DDA37C5AB2632AB0
:1025800023DC4FF4FA7297FBF2F7FB18E6E7032B14
:102590001FD1642F07DD94F916308BB994F91220FE
:1025A0005AB9643309E017F1640F09DA94F9163067
:1025B00033B994F9122002B99C33A374012303E0C8
:1025C0006337C62F01D80023A37594F9123014275E
:1025D0005F43032E1DD84C4A05F590630F3302EB81
:1025E000C303DA8812B2BF1A002F07DD1A8912B2AC
:1025F000002A0EDDFA02D71B1B8907E009D09A8852
:1026000012B2002A05DA414A9B8857431BB297FB56
:10261000F3F7237F3F2B03D9FE2B01D0FD2B24D1D1
:102620003B4B04F11C00984794F91B30012B15D14A
:102630009B3364218DF804308DF805309C3B8DF878
:1026400008308DF809008DF80C1038B28DF80D1097
:10265000304F032201ABB847074606E0C302181A01
:10266000642390FBF3F000B23F1894F91A30012B69
:10267000264B08BF7F429F42B8BF1F4640F2FF7300
:102680009F42A8BF1F46244B33F8152012B2974231
:102690001DD0022E0BD9214A1670214A1278A2B100
:1026A00094F91520042A10D01E4A16700DE033F854
:1026B0001500282200B297FBF2F190FBF2F2914252
:1026C00003D0164A1670164A127823F8157094F93A
:1026D000143027827BB194F9153063B9143397FB1A
:1026E000F3F31BB2642BA8BF64236FF06302934221
:1026F000B8BF1346A37401352034402D7FF4D7AE04
:1027000005B0F0BD58040020D007002001F8FFFFFD
:10271000751E0008D51D000802030020E9010020F5
:10272000912C0020ED0100202DE9F04F0D4685B0E1
:1027300000242B5D2E193F2B79D8301D424B984732
:10274000012874D106F10800404B984782460028C2
:102750006DD02E5DDFF8209173014B44988F3C4F74
:1027600000B2B8473B493C4B98474FF07E513B4B3A
:102770008046984728B9404639493A4B984718B996
:1027800004E04FF07E5801E0DFF8D4802B195B782D
:10279000DFF8EC90013BDBB2012BDFF8E8B0324F01
:1027A00005D84046C847CDE90001404606E040460E
:1027B000C847CDE9000140464146D8474146D84781
:1027C0002A4A014640469047C847214BCDE90201BD
:1027D00050469847C8470022DFF8ACC0244BE0477A
:1027E00002460B46DDE90201B847DFF8A0C0024609
:1027F0000B46DDE90001E04711A3D3E90023B84708
:102800001C4A90471C4ADFF870C07301760163448C
:10281000961998873836B28840F2FF7312B29A42FE
:1028200004DCB288154B12B29A4200DAB3800C3441
:10283000C02C7FF47EAF05B0BDE8F08FAFF3008011
:102840000000000000FC9F40C11E0008751E00082B
:10285000550C000800E0FF44650E000875100008E4
:10286000000080BF391000087D040008E90A000854
:1028700000005940B1090008D007002001F8FFFF0F
:10288000D5030008FD0C0008D1060008150100085A
:10289000F8B504460E460025735D77193F2B12D814
:1028A000381D0B4B984701280DD10A4B07F1080042
:1028B0009847735D64215B01E318B3F9102042432C
:1028C00092FBF1F21A820C35C02DE5D1F8BD00BFA4
:1028D000C11E0008751E00082DE9F0470446884611
:1028E0000D46002708EB070673783F2B76D8281D86
:1028F0003E4B984701286CD1DFF8F8A005F108009D
:10290000D047814605F10C00D04718F807207378AE
:1029100092B95B01E318B3F910202B8A19B209EBC5
:10292000010C624503DD9944A5F810904BE0091AAB
:102930008A4248DA1B1A45E05B01E318B3F910300C
:10294000142B10DD03FB09F340F2FF7293FBF2F34B
:10295000B2785BB2002A28D0698A08B2101898426F
:1029600024DA521810E013F1140F11DA4343204A0D
:1029700093FBF2F3B2785BB242B1698A5B4208B270
:10298000801A984212DD8A1A6A820FE05B420CE0DC
:10299000B37853B16A8A11B2C81A002801DDD31A7C
:1029A00003E0CB424CBF9B1800236B822B8A6A8AC0
:1029B000D2180F4B2A8212B29A4203DB40F2FF7305
:1029C0009A4200DD2B8273782A8A5B01E3181A820F
:1029D00004E073785B01E3181B8A2B8214371435EB
:1029E000B7F5A07F7FF47EAFBDE8F087C11E000879
:1029F00001F8FFFF751E00082DE9F74F0B469046C2
:102A000082460E4601F5C0620021198218339342B6
:102A1000FAD14446002518F805303F2B00F29F807C
:102A2000201D534B9847012840F09980514B04F1E9
:102A300008009847237B81463F2B21D894F90D202D
:102A4000F2B14FF0180B0BFB036B18F80530BBF815
:102A500010C05B015344B3F91000082204F11403C1
:102A6000CDF804C04946444FB84794F90D30DDF81D
:102A700004C04343642293FBF2F39C44ABF810C0C0
:102A8000A37B3F2B21D894F90F20F2B14FF0180B04
:102A90000BFB036B18F80530BBF810C05B01534407
:102AA000B3F91000082204F11403CDF804C049461C
:102AB000314FB84794F90F30DDF804C04343642226
:102AC00093FBF2F39C44ABF810C0237C3F2B21D83E
:102AD00094F91120F2B14FF0180B0BFB036B18F8AF
:102AE0000530BBF810C05B015344B3F91000082255
:102AF00004F11403CDF804C049461F4FB84794F9B8
:102B00001130DDF804C04343642293FBF2F39C448C
:102B1000ABF810C0A37C3F2B21D894F91320F2B15D
:102B20004FF0180B0BFB036B18F80530BBF810C007
:102B30005B015344B3F91000082204F11403CDF8EB
:102B400004C049460C4FB84794F91330DDF804C06F
:102B50004343642293FBF2F39C44ABF810C034353A
:102B60003434B5F5506F7FF456AFBDE8FE8F00BF2B
:102B7000C11E0008751E0008D51D00082DE9F04192
:102B800004460E460025735D06EB05083F2B21D851
:102B900008F10400124B984701281BD1725D1827D9
:102BA00007FB0242138A19B2002902DD08F108006E
:102BB00002E073B108F10C000A4B9847735D642280
:102BC00007FB0347B7F91030434393FBF2F33B8213
:102BD00000E013821035B5F5807FD4D1BDE8F081D7
:102BE000C11E0008751E00082DE9F04104460E467E
:102BF0000025735D77193F2B28D8381D164B984751
:102C0000012823D1DFF8548007F10800C047735D25
:102C1000182202FB0342C3026421181AB2F91030D1
:102C200090FBF1F08342C8BF108207F10C00C0474F
:102C3000735D182202FB0343C2026421821A92FBD5
:102C4000F1F2B3F910109142B8BF1A821035B5F500
:102C5000807FCED1BDE8F081C11E0008751E00083E
:102C600070B5044600F5C066237DB4F910503F2BC3
:102C700003D9FE2B01D0FD2B0AD10F4B04F1140018
:102C80009847C3021B1A642293FBF2F31BB2ED18A0
:102C900094F91230012B094B08BF6D429D42B8BF19
:102CA0001D4640F6FE139D42A8BF1D4625821834DE
:102CB000B442D9D170BD00BF751E000802F6FFFFF7
:102CC000704700002DE9F047274CB4B0A0420746FA
:102CD000884645D32549264B02A89847254E02A889
:102CE000B0470022391B02AB0124234D0094181871
:102CF00009B21346A847DFF89890204902A8C847B0
:102D000002A8B04702AB0022009418180FFA88F10D
:102D10001346A847B246013C2E464D460EE01749E1
:102D200002A8A84702A8D0470123395D00220093DA
:102D300002AB18181346B0470134E4B24445EED351
:102D40000E4902A8A8470E4B002098470D4C02A937
:102D50000020A04700200C4B984700200B49A047BB
:102D6000002034B0BDE8F087D00700200826010815
:102D7000E11100089D120008F5230008263801081B
:102D8000290B0108750B0108210C01087547010882
:102D90009911000838B5084B9847084D0446A847D4
:102DA000844206D2A847041B04EBD4746010C0B25E
:102DB00038BD002038BD00BF79FE0008BF01010802
:102DC00038B5084B9847084D0446A847844206D2B8
:102DD000A847041B04EBD4746010C0B238BD0020B7
:102DE00038BD00BF9DFE0008BF01010838B5054B86
:102DF00005469847044B044628469847201AC0B217
:102E000038BD00BFBF0101089DFE000808B592F95A
:102E100000300BB1002300E00123137010460121A4
:102E2000014B9847012008BDC52C00082DE9F04F43
:102E3000DFF854928FB014468846C847884D06463E
:102E4000A8470121A6F10A02A0F10A0300260A20E0
:102E5000D2B2DBB20091834F0146019602960396EF
:102E6000B847C8478146A847FF21A9F10A02A0F147
:102E70000A030A20019102910391D2B20146DBB20A
:102E80000096B847DFF804A22046D047DFF8E0916B
:102E9000013099F800B0834502D8BBF10F0F01D97A
:102EA00089F80060DFF8D0C1FF26CDF814C02046B5
:102EB000E0476D4F22463346009601960F21B847F2
:102EC0006A4ADDF814C013789346002B7ED1B8F11E
:102ED000010F0DD1204699F800800693D047804518
:102EE000634E069B0CD208F1010886F800803AE098
:102EF000B8F1020F0AD199F800305D4E13B1013BD1
:102F0000337030E02046D04730702CE0A8F1030841
:102F10005FFA88F8B8F1010F25D899F8006046B932
:102F20002046D047411C89B22046524B9847012089
:102F30006AE106F1FF3814F808202B2A01D12D236D
:102F400002E02D2A03D12B2304F808300BE02046A1
:102F50000693D0478642069B03D9202204F8082016
:102F6000A3558BF8006099F800606EB94249434858
:102F700088470646A847FF23A0F11101009301935B
:102F80003046C9B23D4A10E02046D04786420FD9AC
:102F9000394A3B4890470646A847FF23A0F1110154
:102FA000374A009301933046C9B2B847002624E15E
:102FB000314B344898470646A847FF23A0F111013A
:102FC000009301933046C9B22E4AEEE72D48E04700
:102FD0000690A847069BA0F111010096184601969D
:102FE000C9B2284A3346B847B8F1010F0DD19BF852
:102FF0000030013BE25C2B2A10D02D2A12D0382A57
:1030000001D8013215E0302213E0B8F1020F12D1DD
:103010009BF80030013BE25C2B2A01D1023208E030
:103020002D2A01D1023A04E0302A01D9013A00E008
:103030003922E254BAE7A8F103085FFA88F8B8F138
:10304000010FB3D89BF800305A1EA15C202901D192
:103050002039A15489F8003000238BF80030A5E70F
:10306000C30101080DFC000815FF00088C030020B7
:1030700096030020C52C0008952D00081026010895
:103080001526010819260108BF0101089D12000834
:10309000A35D0021A01908908DF82C308DF82D101B
:1030A0005B4B5C48984799F800C002300CF1FF3345
:1030B000C0B29E42079040F09180A35D06FB00F8ED
:1030C000202B0CD1A84708F10F084108FF230093DB
:1030D00001935FFA88F0C9B24F4AB8473BE00EAAA5
:1030E00002F80C3D5FFA88F8CDF814C0CDF82480C2
:1030F0000692A84709994FF0FF0801F10F03410814
:10310000C9B2069AD8B2CDF800804346CDF8048003
:10311000B847A8470690A847079BDDF814C0069952
:103120000CFB03FC099A4308490802F10D0E00202C
:103130000CF10D02033905330090CDF80480CDF871
:103140000880CDF80C805FFA8EF0C9B2D2B2DBB243
:10315000DFF8C8C0E0479BF80030002B4BD0089840
:1031600003785A1ED2B22B2B8DF82C2001D10233BA
:1031700006E02D2B01D1023B02E02F2A02D8392391
:103180008DF82C30079906FB01F8A84708F10F08C5
:103190004108FF2306395FFA88F8009301930BAAD0
:1031A0004046C9B2B847089A13785A1CD2B22B2BA2
:1031B0008DF82C2001D1023306E02D2B01D1023BEA
:1031C00002E0392A02D930238DF82C30A847FF239A
:1031D0004108063100930193404609E0A847079B48
:1031E000410806FB03F2FF230F3200930193D0B294
:1031F000C9B20BAAB8470136F6B22046D047013013
:103200008642FFF445AF00200FB0BDE8F08F00BF4D
:1032100079FE0008EE2901081E2601080DFC0008B1
:103220002DE9F04186B006AC2B2304F8103D2A3B73
:1032300006468846114FB2F9001015460093092240
:10324000013B0DF10900B847FF23414622463046B5
:103250000B4EB0470B4E07462046B0472046B047BE
:10326000002803DA4FF0FF332B6002E02046B0471E
:103270002860384606B0BDE8F08100BFF52300089D
:103280002D2E0008D5100008F0B5012387B00646A2
:103290000D461446B2F9001003A805220093104F02
:1032A000013BB8472946FF23304603AA0D4DA847E6
:1032B0000D4D064603A8A847B0F5803F01DB00236B
:1032C00005E003A8A847002803DA4FF0FF33238066
:1032D00002E003A8A8472080304607B0F0BD00BF39
:1032E000F52300082D2E0008D5100008F0B50E4675
:1032F000B2F9001087B00029074614464FF00103C9
:10330000174D04DA009303A80522013B07E02B22A6
:103310008DF80C2000930DF10D00263A0023A847EC
:103320003146FF2303AA0F4D3846A8470E4D0646E7
:1033300003A8A847B0F5FA4F02DD4FF4FA4306E0C0
:1033400003A8A84710F5FA4F03DA48F200332380A8
:1033500002E003A8A8472080304607B0F0BD00BFB8
:10336000F52300082D2E0008D51000082DE9F04F98
:10337000DFF888928FB014468846C847924D0646BB
:10338000A8470121A6F10A02A0F10A0300260A209B
:10339000D2B2DBB200918D4F0146019602960396A0
:1033A000B847C8478146A847FF21A9F10A02A0F102
:1033B0000A030A20019102910391D2B20146DBB2C5
:1033C0000096B847DFF810B22046D847DFF80CA2C5
:1033D00001309AF80090814502D8B9F10F0F01D958
:1033E0008AF80060FF26DFF818922046C847784F19
:1033F00022463346009601960F21B847754ACB46C0
:103400001378002B78D1B8F1010F0FD10593204626
:10341000714A90479AF80080013080456F4E059BB5
:103420000CD208F1010886F8008032E0B8F1020FF2
:103430000CD19AF80030694E13B1013B337028E08B
:103440002046654B98470130307022E0A8F1030810
:103450005FFA88F8B8F1010F1BD89AF8006056B9E6
:10346000DFF874C12046E047411C89B220465C4B1E
:103470009847012095E105932046574A9047864298
:10348000059B04D9A219202102F8011CA355514B18
:103490001E709AF8006066B95248D8470646A84799
:1034A000FF23A0F11101009301933046C9B24D4AA8
:1034B00011E02046DFF820C1E04786420FD94A4894
:1034C000D8470646A847FF23A0F11101464A0093BA
:1034D00001933046C9B2B8470026A04659E1434897
:1034E000D8470646A847FF23A0F111010093019396
:1034F0003046C9B23D4AEEE73C48C8478146A84736
:10350000A0F11101009601964846C9B2374A3346E8
:10351000B847B8F1010F09D12E480378013BE25CAE
:103520007E2A01D801320DE020220BE0B8F1020F13
:103530000AD1284A1378013BE25C202A01D9013ADA
:1035400000E07F22E254C7E7A8F103085FFA88F899
:10355000B8F1010FC0D81F4803785A1EA15C20297A
:1035600001D12039A1541B4A8AF80030002313707E
:10357000B2E708EB0603079318F806304FF0000C8B
:103580008DF82C308DF82DC0194B1A4898479AF8B1
:1035900000C002300CF1FF339E42C4B240F0EC8018
:1035A00018F8063006FB04F9202B2BD1A84709F1A7
:1035B0000F094108FF23009301935FFA89F0C9B214
:1035C0000D4AB8475AE000BFC30101080DFC0008CE
:1035D00015FF0008A10300209D120008930300209E
:1035E000C52C000810260108152601081926010817
:1035F00079FE0008EE2901081E260108BF01010816
:10360000952D00080DF1380B0BF80C3D5FFA89F988
:10361000CDF814C0CDF81890A847069A4FF0FF09CE
:1036200002F10F0341085A46C9B2D8B2CDF8009052
:103630004B46CDF80490B847A8478346A847DDF825
:1036400014C0069B0CFB04FC03F10D0E4FEA5B0B50
:1036500043080CF10D020020ABF10301053300908B
:10366000CDF80490CDF80890CDF80C905FFA8EF06C
:10367000C9B2D2B2DBB2DFF838C1E0474A480378BA
:10368000002B00F084806342DBB2089306FB04F356
:103690000F33DBB2CDF824800693B0464FF000091B
:1036A00026461C4615E0023BC9EB03030DF1380B1F
:1036B0000BF80C3DA8474108FF23A2190C39D0B2E2
:1036C00000930193C9B25A46B84709F101095FFA5C
:1036D00089F9089A0798A418C145E4B20378E2D1A1
:1036E0000DF1380B013B0BF80C3D34464646DDF836
:1036F0002480A84741084FF0FF090639C9B25A464D
:103700004B46CDF80090CDF804900698B847079A3C
:10371000137801338DF82C30A84741080631CDF8D5
:103720000090CDF804905A464B460698C9B2B84767
:10373000A9F1FF09C34619E007980DF1380803788D
:1037400002334B4408F80C3DA84709EB06026243DC
:103750004108FF230F320C31D0B200930193C9B25C
:103760004246B84709F101095FFA89F9C6F10E032B
:103770009945E1DBD8460AE0A84774434108FF2396
:103780000F3400930193E0B2C9B20BAAB8470136D7
:10379000F6B24046054A904701308642FFF4E9AE52
:1037A00000200FB0BDE8F08FA10300209D1200089B
:1037B0000DFC000837B50B4B0D4693F838300A2B3B
:1037C00003D9811CFF23084C04E0084B084C1978EE
:1037D000FF234118009301930220C9B22A46A04753
:1037E0003EBD00BF502C002015FF0008E000002067
:1037F000CDFE00082DE9F341DFF85880064698F821
:1038000038300D460A2B104F104B114C08D9084682
:1038100098473A7898F83830D2438018073B08E048
:10382000084698473B78DFF83080DB43C01898F8AB
:103830000030F618F1B2FF232A46C0B2009301937C
:10384000A047BDE8FC8100BF34000020ED2D00083A
:10385000CDFE0008502C0020E000002070B50123B0
:1038600086B0144600220546009303A8134609B209
:10387000044EB047284603A92246034B984706B09A
:1038800070BD00BFF5230008F537000837B50E4BB3
:103890000C46054698470D4B013593F838200C4BE4
:1038A000083A19786FF012035B1A02EBD27205EB3B
:1038B0006201C01800230093E2B2C9B20133054C83
:1038C000C0B2A0473EBD00BFBF010108502C002080
:1038D00034000020F5F7000870B5054686B01C4698
:1038E000002922D1012A3E4B05D13E4903A8984721
:1038F0002846242162E0022A02D103A83A4923E0A3
:10390000032A02D103A8394955E0042A02D103A8A9
:10391000374906E0052A02D103A8364914E03649A2
:1039200003A8984728462B2148E0012926D1012ADF
:103930002B4B05D1314903A89847284625213DE066
:10394000022A03D12E4903A8984741E0032A05D152
:103950002C4903A89847284627212FE0042A02D1A2
:1039600003A8294906E0052A02D103A82749EBE765
:10397000274903A8984728462A211FE0022908D191
:10398000032A25D1234903A8154B98472846282107
:1039900014E0032908D1032A1AD11F4903A8104BA8
:1039A00098472846292109E004290AD1032A0FD182
:1039B0001A490B4B03A89847284626212246184B44
:1039C0000AE001230022009303A81346154EB047D6
:1039D000154B284603A92246984706B070BD00BF84
:1039E000E1110008242601082B26010833260108CE
:1039F0003A2601083D260108942601083C2B0108BF
:103A000045260108842E01084A2601084E26010891
:103A10008B260108552601085C260108632601084B
:103A20008D380008F5230008F537000870B501232C
:103A300086B0144600220546009303A8134609B237
:103A4000064EB04703A80649064B9847284603A9E7
:103A50002246054B984706B070BD00BFF52300080D
:103A60007626010899110008F537000837B5064B8E
:103A70000D461978054C4118FF230320C9B22A4688
:103A800000930193A0473EBDE00000204DFF0008D9
:103A900037B5064B0D461978054C4118FF23032016
:103AA000C9B22A4600930193A0473EBDE000002022
:103AB00015FF00082DE9F0410E46097888B03F292E
:103AC00005469046174C04D8174B490102A8C9185F
:103AD00005E00331C9B202291ED8144902A8144BCB
:103AE0009847144B30469847134E0746134902A88F
:103AF000B047134B02A8984701230022009302AB62
:103B000039B218180F4F1346B8470F4902A8B047EB
:103B1000284602A9424600E00C49A04708B0BDE88B
:103B2000F08100BFF5370008FC0700206826010877
:103B3000E1110008751E000899110008522C0108B7
:103B40009D120008F5230008762601086F2601085B
:103B50002DE9F0410E46097886B03F290546174603
:103B6000DFF86480104C12D8104B4901C918684620
:103B70000F4B98473046C0470E4B10B168460E4970
:103B800001E00E49684698472846694607E03046F6
:103B9000C04710B128460A4901E00A4928463A467A
:103BA000A04706B0BDE8F081F5370008FC0700200B
:103BB000E111000899110008782601087E26010805
:103BC000852601088E260108C11E0008F0B5DFF821
:103BD00070C085B00546184EF1B13278C71D00247B
:103BE000FFB20123C2F12E020093204629463B4634
:103BF000D2B2019402940394E0473278FF23C2F1D9
:103C00002E02009401930293039320462946D2B2D8
:103C10003B460A4CA0470DE03278C31DC2F12E028C
:103C2000012000900191029103910846D2B22946E9
:103C3000DBB2E04705B0F0BD340000200DFC000809
:103C40005DFA00082DE9F043054685B00C461D4F8E
:103C50001D4EDFF87C9011B3B847327805F10708A4
:103C6000D24300245FFA88F8012382182946009382
:103C700020464346D2B2019402940394C847B84701
:103C80003278FF23D2438218009401930293039366
:103C900020462946D2B243460C4CA0470EE0B84716
:103CA00032780121D2438218EB1D0091204629462B
:103CB000D2B2DBB2019402940394C84705B0BDE8C8
:103CC000F08300BFBF010108340000200DFC000894
:103CD0005DFA000838B50C46054622460449054BF6
:103CE000984728463D212246034B984738BD00BFE0
:103CF00010260108B53700088D38000808B50A46B7
:103D0000014B0249984708BDB53700081026010845
:103D1000012809D11848002303701078013988421E
:103D20000ADA0130107025E002280AD1124B02385D
:103D30001870137813B1013B13701BE00139117037
:103D400018E0032807D11978FF290CBF1278FF2249
:103D50001A7001220CE0632805D91A78FF2AF8D1DD
:103D600064381870F5E7042804D100221A70013273
:103D7000024B1A7000207047A80300209E0000200C
:103D80002DE9F04315463E4A89B012780446012ACF
:103D90008E463C4F3C4E20D1B7F8008040F6736C05
:103DA0001FFA88F8E04512D8DFF8E0C0DCF844805C
:103DB0004FF47A7CB8FBFCF90CFB198CBCF5FA7F4C
:103DC00005D9009205EB000C5B18FE321FE00121C3
:103DD00000912A197344013924E0B7F800C041F278
:103DE00018021FFA8CFC944517D9284AD2F844C00F
:103DF0004FF47A72BCFBF2F802FB18C2B2F5FA7FFC
:103E00000BD90122009205EB000C5B18013A0192DC
:103E1000029203925FFA8CF20AE0012100912A19C2
:103E20007344FE3101910291039120467146D2B252
:103E3000DBB2B0473988642389B2B1FBF3F1633B4D
:103E40000022009309B205A8114EB04705A8114BF6
:103E50009847114B2D1A197805EBD575C1F108015A
:103E600001EBD17104EB6504FF234910009301932A
:103E7000E0B2C9B205AA094CA04709B0BDE8F08379
:103E8000EE010020500400205DFA0008502C0020B4
:103E9000F523000879FE0008F000002015FF000857
:103EA00008B50146014B0248984708BDE1110008DA
:103EB000D80400202DE9F04F4B1EDBB2012B144635
:103EC00085B082466F4B704A0BD81878884208D16B
:103ED0006E4805786EB2022E01DC013505700620B1
:103EE00009E0127850B2002803DD6748013A0270F9
:103EF00002E0664A00201070012919700CD1634B52
:103F000022781B7859B2C1F156018A4201DA013395
:103F10000BE08BB156230FE0022911D15B4B2278C5
:103F20001B7859B28A4203DDDB43D218227004E0C9
:103F30000BB9563300E0002323702046012106E030
:103F4000042907D1237820465B4223700339504B64
:103F5000984707E0032905D1204602394C4B984782
:103F600001208CE0DFF83C81C0474A4F0546B84746
:103F700000266A1F431F4FF0010B0A21D2B2DBB2A9
:103F80000520DFF82891CDF800B00196029603963F
:103F9000C847C0470546B8476A1F431FFF250A2187
:103FA000D2B20520019502950395DBB20096C84771
:103FB000394B504698478146B84781082B460095B3
:103FC00001954846354DC9B25246A8472378344D2D
:103FD0005B450AD9B8472278A0F11001023A009651
:103FE0000A20C9B2D2B25B46A84723785BB1B84772
:103FF0002278410800230231013A00931320C9B20C
:10400000D2B20133A847C0470646B8470321760815
:10401000B0FBF1F1F31F06310026D8B2227801235C
:104020000096C9B2A8472378552B12D81D4B984744
:10403000184B8146984722784108A9F1220902319C
:10404000013200965FFA89F0C9B2D2B20123144E50
:10405000B0472378542B0ED8C0470646B84722787D
:10406000A0F110010023193E02320093F0B2C9B250
:10407000D2B20133A84750460B4B9847002005B0F9
:10408000BDE8F08FC8030020A2030020CD0300206C
:10409000C52C0008C3010108952D000815FF000874
:1040A000F5F70008BF010108A13E00080DFC00085B
:1040B00030B51D4C85B0A0470123A0F115020021A9
:1040C0001420D2B20093194D07330191029103914C
:1040D000A847A047164B044616489847273C8442F9
:1040E000154C0FDC154B134898472378114AC3F140
:1040F000080303EBD3735910FF2300930193C9B254
:104100000F4C0EE00F4B0B4898472378094AC3F138
:10411000080303EBD37359100B4CFF230093019357
:10412000C9B2A04705B030BDBF0101085DFA000863
:1041300079FE0008D8040020F0000020C12D0008FE
:10414000CDFE0008952D000815FF000870B5254E1E
:104150004EF66023716C88B0B1FBF3F101240222AA
:104160000023214D05A809B20094A8471F4905A8BE
:104170001F4B984705A81F4B9847726C4FF47A73F2
:10418000B2FBF3F23C23B2FBF3F103FB112305AACC
:1041900019B21018002302220094A84700200146FB
:1041A000142200940190029003900823124CA0471F
:1041B00005A8124B9847124BC0F11400197800EB78
:1041C000D070C1F1080101EBD171FF2340104910FB
:1041D00000930193C9B205AA0A4CC0B2A04708B027
:1041E00070BD00BF502C0020F52300080E260108EA
:1041F000991100089D1200085DFA00089DFE000854
:10420000F0000020CDFE00082DE9F04F2B4C89B0C6
:1042100007468B46A0472A4E0546B0474FF0010A95
:104220006A1F431F00250A21D2B2DBB20195029515
:1042300003950520DFF89480CDF800A0C047A04783
:104240000446B047621F431FFF240A21D2B2DBB2EB
:1042500000950520019402940394C047DFF8708014
:104260003846C0478146B04720FA0AF106393A4637
:104270002346009401944846C9B2DFF85890C847D5
:104280000FFA8BF12A462B46CDF800A005A80D4D5C
:10429000A84705A8C0470546B04720FA0AF10631ED
:1042A0002346009401942846C9B205AAC847384657
:1042B000054B984709B0BDE8F08F00BFBF0101086A
:1042C000C3010108F5230008A13E00080DFC000809
:1042D000952D000815FF00080129F8B5064614467B
:1042E00010D11568224B284698471DA3D3E9002317
:1042F000204FB84720B128464FF07E511E4B11E0A9
:104300001E4B13E0022917D11568194B2846984710
:1043100015A3D3E900231A4FB84730B1194B2846EB
:104320004FF07E519847206001E0174B23602046F4
:104330000421164B984707E0032905D110460131A7
:10434000124B98470120F8BD2068114B9847114B3C
:104350000146304698470020F8BD00BFAFF300800B
:1043600085EB51B8FE87C34085EB51B8FE87C3C0CB
:10437000D503000861090008ED0A0008F63F1CC6D5
:104380009D090008E90A0008F63F1C46C52C0008F4
:104390008910000809420008F8B54B1EDBB2012B5A
:1043A000154604462A4B2B4A0BD81878884208D168
:1043B0002948067877B2312F01DC023606700620D4
:1043C00009E0127850B2002803DD2248013A027059
:1043D00002E0214A00201070012919700CD11E4BF7
:1043E0002A781B7859B2C1F1FF018A4201DA013300
:1043F0000BE08BB1FF230FE0022911D1164B2A7875
:104400001B7859B28A4203DDDB43D2182A7004E0DC
:104410000BB9FF3300E000232B702846012106E092
:10442000042907D12B7828465B422B7003390B4BAC
:10443000984707E0032905D128460239074B9847DA
:104440000120F8BD20462978054B98470020F8BD8B
:10445000A6030020C6030020D4030020C52C0008BA
:1044600009420008F8B54B1EDBB2012B1546044685
:104470002D4B2E4A0BD81878884208D12C48067844
:1044800077B2312F01DC02360670062009E012787F
:1044900050B2002803DD2548013A027002E0244AA8
:1044A00000201070012919700FD1214B2A781B7838
:1044B00050B259B2C1F17F01884201DA01330FE0F5
:1044C0000BB9813313E07F2311E0022913D1184B7C
:1044D0002A781B7851B258B27E38884203DCDB431D
:1044E000D2182A7004E00BB97F3300E081232B70CF
:1044F0002846012106E0042907D12B7828465B4293
:104500002B7003390B4B984707E0032905D1284648
:104510000239084B98470120F8BD204695F9001054
:10452000054B98470020F8BDAF0300208E03002004
:10453000CF030020C52C000809420008F0B5184B35
:1045400085B093F83A300546072B02D9154B9847AA
:1045500024E0154FB8470123821F00240821D2B25E
:10456000009305201833114E019402940394B04730
:10457000B847821F0821D2B200940520FF341923C6
:10458000019402940394B047094B2846984700943D
:10459000019423460E212A46064CA04705B0F0BDE3
:1045A000502C0020A13E0008BF0101080DFC0008AE
:1045B000952D000815FF00082DE9F04F002291B05D
:1045C0000125DFF87C8107901346584C009508A818
:1045D00009B2A04708F5125494F83A30544F072B0B
:1045E000DFF86091DFF860A1DFF860B137D9514E94
:1045F000B04794F83A3005900693B8470746B0475D
:10460000069B059ADB43D218013F431E0020D1B21E
:10461000DBB2FAB20095019002900390C84708A857
:10462000D0470546B047444B94F83A201B7894F89D
:104630003A10CB1A03EBD373C2EB63014118FF238B
:104640002846C9B208AA00930193D847079B4FEAAE
:10465000431CE04408F12C00384B984763E0B8470E
:104660000026A0F1080208201B230146D2B20095C3
:10467000019602960396C847B847FF24A0F10802A6
:1046800008200146D2B21B230194029403940096A1
:10469000C847079B4FEA431C08EB0C0909F12C099A
:1046A0004846CDF818C0D0470B2123464A4600940F
:1046B0000194D84708A8D0471321234608AA00949C
:1046C0000194D847DDF818C00D20E04408F1380403
:1046D000E2792B4600960146DFF87480C047A37943
:1046E000642B06D1B8471C380096C0B20D21422277
:1046F00017E094F80690B9F1000F07D1B8471C38BD
:10470000CDF80090C0B20D2143220AE0A3795BB23C
:1047100013F1640F07D1B8471C380096C0B20D21C1
:1047200044222B46C04711B0BDE8F08FF5230008A6
:10473000BF010108C3010108F0000020A13E0008EC
:10474000D00700200DFC0008952D000815FF00087B
:10475000F5F700082DE9F043254F85B08946054659
:10476000B847244E0446B04700210091AB31019177
:10477000A4F10A022231FF24A0F10C030A20D2B2D4
:10478000DBB20291DFF8788001460394C047B84756
:104790000746B0470121009142310191223902912F
:1047A000A7F10C021239A0F10C030C200391D2B234
:1047B0000146DBB2C047104F2846B847DFF84480B7
:1047C00014212A46234600940194C0474846B8471E
:1047D0000746B04741082346009401943846C9B2C1
:1047E0004A46C0472846054B984705B0BDE8F083C8
:1047F000BF010108C3010108952D0008A13E000872
:104800000DFC000815FF00082DE9F04F8DB004469F
:104810009DF858006F4F0B92079309908946804688
:10482000B8476D4E6FF0070A96F83A306B4DC3EB00
:104830000A0A82445FFA8AFA4FEADA0C0CF1FF3C6A
:104840005FFA8CFCCDF810C0654B20469847A8470E
:104850000446B84796F83A30621E01210024C31A74
:10486000DFF88CB12046D2B2DBB20091073101945F
:1048700002940394D847B847079A96F83A30BAFB9F
:10488000F2FA511E6FF00802CDF820A0D21A07915B
:104890000AF1040102EB000A089A079BC2EB0A0A1C
:1048A00008FB0AFA9AFBF3FA8A44A8474D4A5FFAD2
:1048B0008AFA1178A24508BF4FF0010AC1F101013F
:1048C0004118C9B20591A8470690B847069B96F8CB
:1048D0003A2003F1FF3E6FF0010305999B1AC318BC
:1048E00001205FFA8EF2DBB20090084608210194A5
:1048F00002940394D847A8473A4A1178C1F10101BC
:104900004118C9B20591A8470690B847069B96F88A
:104910003A2003F1FF3E6FF0010305999B1AC3187B
:104920005FFA8EF20846DBB208210094FF3401944E
:1049300002940394D847A8472A490B78C3F103038C
:10494000C318DBB20A93B84796F83A600746A847FF
:10495000089A6FF007039B1B9B1ADB1908FB03F1F6
:10496000079BC21E91FBF3F101200A310AF10103FA
:10497000C9B20090DBB20A98D2B2019402940394B7
:10498000D84799F80030DDF810C0434584BF099935
:1049900089F80010E04508D999F80030634498453B
:1049A000C4BFCCEB080889F8008099F800300B9A56
:1049B00001339C440C4B82F800C01B780B4AC3F1B6
:1049C000080303EBD3735B10013313700DB0BDE824
:1049D000F08F00BFC3010108502C0020BF01010867
:1049E000A13E000834000020F0000020E00000207C
:1049F0000DFC00082DE9F04F8BB09B469DF8503020
:104A0000444F09928DF823300E46DCB20546B84774
:104A1000414B6FF0070993F83A209846C2EB090919
:104A200019EB00093D4B284648BF09F10709984793
:104A3000B84798F83A300025C31A4FF0010C082106
:104A400031222846DBB2DFF8E0A0CDF800C0CDF877
:104A500014C0019502950395D047B84798F83A30AD
:104A60000821C31A30222C20DBB20095FF350195B6
:104A700002950395D047B84798F83A3006900793C7
:104A8000B847079B98F83A706FF00B01069AC91A5D
:104A90006FF00C03DB1B89181B186143634391FB08
:104AA000FBF193FBFBF30A310D33DDF814C02D202D
:104AB0002F22DBB2C9B2CDF800C001950295039553
:104AC000D04733784FEAE909A34288BF9DF82330E5
:104AD00009F1FF395FFA89F988BF33704C4506D96F
:104AE00033784B449C42C4BFC9EB04043470337820
:104AF0000B4A01339944099B83F80090094B1B78BA
:104B0000C3F1080303EBD3735B10013313700BB0D5
:104B1000BDE8F08FC3010108502C0020A13E000821
:104B2000E0000020F00000200DFC00082DE9F04F0F
:104B300087B09DF840509DF844A09DF848B005907E
:104B400004911E4617460AEB03090BEB05083E4C81
:104B5000DAB901235FFA89F95FFA88F800930192C4
:104B6000029203924346304629464A46A047049B98
:104B7000012B66D1FE3301930293039300973046D5
:104B800029464A464346A0475BE0002701235FFAD7
:104B900089F95FFA88F800930197434602970397D3
:104BA000304629464A46A047049B012B09D1FE33D3
:104BB0000193029303930097304629464A464346A1
:104BC000A047BAF13C0F2FD906EB5A0AFF245FFA2F
:104BD0008AFAEB1C1D4F504629465246DBB2009420
:104BE00001940294B847A8F1030143465046C9B264
:104BF000524600940194029405EB5B08B8475FFAB3
:104C000088F8F21C30464146D2B2434600940194E3
:104C10000294B847A9F10300009401940294C0B231
:104C200041464A464346B847BBF1280F09D9FF23FE
:104C3000B01CA91C00930193C0B2C9B2059A044CE0
:104C4000A04707B0BDE8F08F5DFA000861FD0008DD
:104C5000CDFE00082DE9F04F814693B09DF87850C5
:104C60000D9199F9001008936943C823680891FBD6
:104C7000F3F19DF87CA04118C9B205914FEA5A01A1
:104C8000079199F90110079C01FB0AF191FBF3F3DD
:104C90009DF870809DF87460E318DBB211460990AE
:104CA0000693924801224346914C00960195CDF817
:104CB00008A0A0470998089900EB080301FB05F03C
:104CC00040F6FE7C90FBFCF01818FF27C0B20AEB00
:104CD00006030246CDF810C00097019702973146AF
:104CE000DBB2DFF818B2D847824C642108224B4669
:104CF0000898A0470AFB00F0079ADDF810C0931946
:104D000090FBFCF15918C9B205EB08020097019716
:104D100002974046D2B20B46D847FF3F03E0CDF89A
:104D200018C0CDF814B009EB070219F907B092F9D1
:104D300001C00BFB05FB0CFB0AFCC823099C079870
:104D40009BFBF3FB9CFBF3FCA34484443C2D5FFAE8
:104D50008BFB5FFA8CFC19D90CEB06030BEB0802FA
:104D6000D2B2DBB20024501E591E00940132FF342F
:104D70000133019402940394CDF810C0C0B2C9B2BB
:104D8000D2B2DBB25C4CA047DDF810C00599069AA0
:104D9000FF240CEB060301EB080091190BEB080252
:104DA000009401940294CDF810C0C0B2C9B2D2B23E
:104DB000DBB2524C0437A047202FDDF810C0AED133
:104DC0000D98002109EB800005900691C346B1467D
:104DD0000D9A069B9A427FD1059CC82394F9002026
:104DE00094F901C06A430CFB0AFC099892FBF3F2A8
:104DF00007998218D2B29CFBF3FC8C4402EB0B03A4
:104E00005FFA8CFCDBB20C920CEB0908DA1E033360
:104E10005FFA88F8DBB20A9308F10303FF24D2B2E9
:104E2000DBB20026A8F10301089210460B9300960E
:104E3000019402940394C9B20A9A2F4FCDF810C07E
:104E4000B847642D48D9059A012392F900102C4FD8
:104E5000324600930FA83346B8472A492A4B0FA879
:104E600098472A4B0FA89847059A012392F90110F9
:104E70000FAA0093101833463246B8470C9B099886
:104E8000234E8342DDF810C015D30799214B8C4582
:104E900009D30FA89847089AA8F10B01101A00949B
:104EA0000194C0B214E00FA89847089B0094181A08
:104EB0000194C0B205E00798844504D20A98009492
:104EC00001940B9905E00A98A8F10B010094019454
:104ED000C9B20FAA2346B04706994B1CDBB2082B78
:104EE00006937FF475AF13B0BDE8F08FF726010885
:104EF0002D4B0008D51D00085DFA000861FD000873
:104F0000F523000898260108991100089D12000851
:104F100015FF000879FE00082DE9F0430446994684
:104F200010F8043B85B03F2B0E4617469DF83080A5
:104F3000134B144D13D898470246204610F8143BE3
:104F400011495B015B18B3F804E0FF21009601975B
:104F5000CDF80890CDF80C800FFA8EF30BE098474F
:104F6000009602460197CDF80890CDF80C8004F128
:104F70001400FF210023A84705B0BDE8F08300BF5F
:104F8000C11E0008554C000808080020F7B50C4663
:104F900006461F4608460F4B114698470E4D0F49CF
:104FA0002046A84720460E4B984700220123009335
:104FB0003946134620180B4FB8470B492046A847DF
:104FC00020460A4B9847073000F0F800B04238BF3F
:104FD0003046FEBDE1110008991100089A2601082B
:104FE0009D120008F5230008092701089DFE00080E
:104FF0002DE9F04F85B098469DF838B000238146E2
:10500000039194461C462349342202FB031202F505
:10501000A452303212798A464A4501D10134E4B2B1
:105020000133402BEFD1002C2FD000252E462746F0
:1050300034226A430AEB020303F5A45330331B798D
:105040004B451DD1039B1348C8EB0301BBFBF7F392
:105050008018023B0CF10102B218DBB200F5A4503B
:105060000093CDF808C043463430C9B2D2B20A4CDE
:10507000A047082393FBF7F3F618DDF808C0F6B253
:105080000135402DD4D1092000E0204605B0BDE80F
:10509000F08F00BFD0070020194F000810B5002383
:1050A0000C4A342101FB032101F5A45292F840403F
:1050B0003832844208D0927A824205D001F5A65255
:1050C0001179814218BF92790133402BE8D1002039
:1050D00010BD00BFD00700202DE9F04F8DB007466E
:1050E0009DF858009B460390624B894616469DF8F2
:1050F0005CA09847604B614A1978342303FB07236F
:1051000003F5A45393F8344090463F2C00F2AE8050
:1051100093F84020411A01EBD171CBEB6104383395
:105120003F2AE4B219D81A7A182101FB02825B7A6D
:1051300002F50262204604A90C325BB2504CA04733
:10514000FF230446C0EB09004E4D00930193C0B20B
:10515000314604AAA847082500E00025342303FBB4
:10516000078303F5A45393F8422038333F2A1CD811
:105170009A7A4249182000FB0212DB7A02F5026299
:10518000204604A90C325BB23D4CA047A919044645
:10519000C0EB0900FF23DFF8ECC0C0B2C9B204AA1B
:1051A00000930193E0470835EDB2342303FB0783F6
:1051B00003F5A6531A793F2A1CD81A792F491820CB
:1051C00000FB02125B7902F50262204604A90C3250
:1051D0005BB22B4CA047A9190446C0EB0900FF2382
:1051E000DFF8A0C0C0B2C9B204AA00930193E0479F
:1051F0000835EDB2342303FB078303F5A6539A79F0
:105200003F2A1AD89A791D49182000FB0212DB792F
:1052100002F50262204604A90C325BB2184CA0478A
:10522000A9190446C0EB0900FF23DFF858C0C0B23B
:10523000C9B204AA00930193E047342303FB078714
:1052400003980634E4B2C4EB0909831EDBB2CBEB4E
:105250000901721C07F5A45000933430C9B2D2B2D0
:105260005B46094D0934A847E0B200E000200DB0CC
:10527000BDE8F08FBF01010834000020D0070020F6
:105280008D4F0008CDFE0008194F00082DE9F04FA2
:1052900095B09DF878C09DF87C509DF880900D9059
:1052A0000C920993CDF800C00122634CCDF818C0D0
:1052B0000195CDF808906148A047DDF818C04FEA85
:1052C0005903099C6A080B93634402EB0408002706
:1052D000DBB20A925FFA88F8079308973C46CDF84C
:1052E0004CC02E4678E0DFF884B12046D84705460A
:1052F0003046D847DFF878A14FF07C51D047504B6B
:10530000014628469847054609FB04F04D4B90FBA3
:10531000F6F09847CDE90E0129462846D0472946A0
:10532000D047494B01460593284698478446474A4B
:105330000B98CDF818C09047DDF818C001466046BC
:10534000D047059B014628469847414DA847CDE9DF
:1053500010010D98D847A84700223E4B3E4DA84764
:105360003E4D02460B46DDE91001A8473C4D024682
:105370000B46DDE90E01A8473A4B9847DDF81CC003
:10538000089D5FFA80FA07EB0C0105EB080004EBBF
:105390000802FF250AEB0C03009501950295C0B2A7
:1053A000C9B2D2B2DBB2DFF8C0C0E047089A079BAF
:1053B000C2EB0800D91BC4EB0802CAEB030300953B
:1053C00001950295DBB2C0B2C9B2D2B2264DA84750
:1053D000631C08945746DCB2DDF828C0644582D3CC
:1053E0000C9A354602FB06F0C826DDF84CC090FB4F
:1053F000F6F08044FF245FFA88F009EB0C03614665
:105400000246009401940294DBB2174FB847DDF8CE
:1054100030C0079A0CFB09F1099B91FBF6F151187A
:10542000C9B2EA181846009401940294D2B20B460D
:10543000B84715B0BDE8F08F2D4B00089C26010839
:10544000650E0008B1030008E90A0008550C0008C1
:10545000D503000800005940D10600087D0400086B
:1054600019010008010A000861FD00084D0C000840
:10547000FD0C00082DE9F04F8BB09DF854509DF8BD
:1054800058809DF85C709DF860B0089109921946AB
:1054900001222B46CDF800800197CDF808B0354C9D
:1054A0009DF950A0A047089A4FEA5B0C02FB0CF153
:1054B00005EB5703DBB20CEB080606936FF06303B2
:1054C000F6B291FBF3F17118FF24DFF8AC90284697
:1054D000069A3346C9B2CDF814C0009401940294E0
:1054E000C847DDF814C0099A7B19DBB2079302FBA9
:1054F0000CF34FF0640C93FBFCF3F3180698314661
:10550000079ADBB2CDF814C0009401940294C84706
:105510000AFB07F0C82390FBF3F0069B41461818DE
:10552000C0B20BEB08030246DBB200940194029474
:10553000C847BAF1000FCBBF099A089B02FB0AFAD1
:1055400003FB0AFADDF814C0C8239AFBFCFC4FFAEF
:105550008CFC0BFB0CFC9CFBF3FC66443733F1B278
:105560000093019302932846079A0B46C8470BB055
:10557000BDE8F08F2D4B000861FD00082DE9F04FCC
:105580009946454B8BB0064605930846BDF950A099
:105590009DF854509DF858809DF85C709DF860B05F
:1055A00014469847059B0890204698473B4C099025
:1055B0004946304601222B46CDF800800197CDF8B0
:1055C00008B0A047089A4FEA5B0C0CFB02F105EB10
:1055D0005703DBB20CEB080606936FF06303F6B2D9
:1055E00091FBF3F1FF247118DFF8B4902846069A76
:1055F0003346CDF814C0009401940294C9B2C84750
:10560000DDF814C0099A7B19DBB207930CFB02F397
:105610004FF0640C93FBFCF3F318CDF814C006981C
:105620003146079A009401940294DBB2C8470AFB02
:1056300007F040F6FE7390FBF3F0069B4146181806
:10564000C0B20BEB08030246DBB200940194029453
:10565000C847BAF1000FCBBF099A089B0AFB02FAB0
:105660000AFB03FADDF814C040F6FE739AFBFCFC5B
:105670000FFA8CFC0BFB0CFC9CFBF3FC6644FF2339
:10568000F1B20093019302932846079A0B46C8474C
:105690000BB0BDE8F08F00BF751E00082D4B000851
:1056A00061FD00082DE9F04F8DB0BDF958C00646E8
:1056B0009DF86800CDF814C00990534F08469DF836
:1056C0005C809DF860A09DF8649014461D46B84724
:1056D0000A902046B84709990B90CDF804900291A2
:1056E0003046294601224346CDF800A0474CA0474A
:1056F0000A9B4FEA590B0BFB03F20BEB08076FF009
:105700006303FFB2099892FBF3F20A99BA184008B2
:10571000D2B2079200FB01F200EB0A06F6B292FB4E
:10572000F3F3F318FF24DBB2394D06900893079882
:1057300019463A463346009401940294A8470899C2
:105740004046079A0B46009401940294A8470B9A8E
:1057500006980BFB02F34FF0640B93FBFBF3FB1873
:10576000DBB2079300FB02F393FBFBF3F318DBB20E
:10577000069338463146079A009401940294A8474C
:10578000069909EB0803DBB2089307981A460094C0
:105790000B4601940294A847DDF814C040F6FE734E
:1057A0000CFB09F9099999FBF3F94F44F8B201EBA5
:1057B0000A030246DBB25146009401940294A847C2
:1057C000DDF814C00998BCF1000FCBBF0B9A0A9BFF
:1057D0000CFB02FC0CFB03FC9CFBFBFB0FFA8BFBA2
:1057E00000FB0BFB40F6FE739BFBF3FB5E44FF23C9
:1057F000F1B20093019302934046089A0B46A847E2
:105800000DB0BDE8F08F00BF751E00082D4B0008DD
:1058100061FD00082DE9F04F8DB0064609929DF814
:1058200058009DF85C200A930023884608900B924C
:105830001D46FF2E09D1484A0C2101FB032202F527
:1058400094523032127942450FD0B8F1FF0F0ED189
:10585000DAB296420BD1404A0C2101FB062202F536
:105860009452303212793F2A01D80135EDB201331A
:10587000102BDED1002D6BD00024A1462F46FF2E29
:1058800009D1354B0C2202FB043303F5945330331A
:105890001B7943450FD0B8F1FF0F54D1E3B29E42BC
:1058A00051D12D4B0C2202FB063303F594533033B8
:1058B0001B793F2B47D84FF00C0B0BFB04FBDFF899
:1058C00098A00BF594530AEB03023C32234D069348
:1058D00010460792A847079A014607911046A84725
:1058E000069B0546534403F138001D4B9847D344AB
:1058F0000BF59452303212790346520192449AF8D1
:105900003E20DDF824E0089852B20092C0EB0E026F
:105910000A98D2B20192421C4A44D2B20292DDF8F5
:105920002CE0089A0F480392BEFBF7F2023AD2B27B
:10593000049207992A460C4DA847082393FBF7F3D6
:1059400099445FFA89F90134102C98D1092000E0BC
:1059500028460DB0BDE8F08FD0070020751E000866
:10596000C11E0008A1260108755400082DE9F04F5A
:1059700089B006469DF84C0006939DF848A0002388
:105980008846059207901D46FF2E09D1424A0C21F8
:1059900001FB032202F58E523032127942450FD0BC
:1059A000B8F1FF0F0ED1DAB296420BD13A4A0C2170
:1059B00001FB062202F58E52303212793F2A01D8BD
:1059C0000135EDB20133102BDED1002D60D0002463
:1059D000A1462F46FF2E09D12F4B0C2202FB043388
:1059E00003F58E5330331B7943450FD0B8F1FF0FC9
:1059F00049D1E3B29E4246D1274B0C2202FB06332B
:105A000003F58E5330331B793F2B3CD84FF00C0BF2
:105A10000BFB04FB204D0BF58E53E8181F4A049333
:105A20003C309047049B8446EB1803F13800CDF8D6
:105A300010C01B4B9847AB440BF58E5330331B798A
:105A400001465B01ED1895F83E20059DDDF810C07C
:105A5000CAEB0503069DDBB2681C4844079DC0B233
:105A60000090A81E90FBF7F0C0B20290CDF804A001
:105A70005FFA8CF052B20B4DA847082393FBF7F363
:105A800099445FFA89F90134102CA3D1092000E070
:105A9000284609B0BDE8F08FD0070020751E000829
:105AA000C11E00088D5200082DE9F04F8DB006464A
:105AB00009929DF858009DF85C200A9300238846BF
:105AC00008900B921D46FF2E09D1494A142101FB73
:105AD000032202F59A523032527942450FD0B8F182
:105AE000FF0F0ED1DAB296420BD1414A142101FBCD
:105AF000062202F59A52303252793F2A01D80135F6
:105B0000EDB20133102BDED1002D6CD00024A14664
:105B10002F46FF2E09D1364B142202FB043303F526
:105B20009A5330335B7943450FD0B8F1FF0F55D10D
:105B3000E3B29E4252D12E4B142202FB063303F5F0
:105B40009A5330335B793F2B48D84FF0140B0BFB43
:105B500004FBDFF89CA00BF59A5303F13802524482
:105B6000244D0693101D0792A847079A01460791F6
:105B700002F10800A847069B0546534403F138008C
:105B80001D4B9847D3440BF59A5230325279034655
:105B9000520192449AF83E20DDF824E0089852B26F
:105BA0000092C0EB0E020A98D2B20192421C4A4403
:105BB000D2B20292DDF82CE0089A10480392BEFBA4
:105BC000F7F2023AD2B2049207992A460C4DA8473E
:105BD000082393FBF7F399445FFA89F90134102CF9
:105BE00097D1092000E028460DB0BDE8F08F00BF36
:105BF000D0070020751E0008C11E0008AA26010853
:105C0000755400082DE9F04F8DB00A939DF85C3073
:105C10009DF858A00B9300230646884609921D461E
:105C2000FF2E08D103F506724049033201EB021240
:105C3000127942450ED0B8F1FF0F0DD1DAB296427B
:105C40000AD106F506723949033201EB02121279C4
:105C50003F2A01D80135EDB20133102BE0D1002DE0
:105C600060D00024A1462F46FF2E08D104F506730C
:105C70002E4A033302EB03131B7943450ED0B8F1D0
:105C8000FF0F4AD1E3B29E4247D106F50673274A79
:105C9000033302EB03131B793F2B3ED82201234D24
:105CA00002F50652383204F5067B52190BF1030B4C
:105CB00002F1080105EB0B1B04321D4B0891079202
:105CC0000BF10800984703469BF804004FF0180EAC
:105CD0000EFB005000F5026070448088099D00B200
:105CE0000090CAEB05000A9DC0B20190681C4844B0
:105CF0000B9DC0B20290B5FBF7F00238C0B2049021
:105D0000CDF80CA00B480899079A0B4DA84708231B
:105D100093FBF7F399445FFA89F90134102CA3D16E
:105D2000092000E028460DB0BDE8F08FD007002024
:105D3000C11E0008B12601087D5500082DE9F04F6D
:105D40008DB00A939DF85C309DF858A00B9300230A
:105D50000646884609921D46FF2E08D103F50A72B1
:105D60004049033201EB0212127942450ED0B8F1DC
:105D7000FF0F0DD1DAB296420AD106F50A723949FF
:105D8000033201EB021212793F2A01D80135EDB23C
:105D90000133102BE0D1002D60D00024A1462F4606
:105DA000FF2E08D104F50A732E4A033302EB0313C6
:105DB0001B7943450ED0B8F1FF0F4AD1E3B29E42A2
:105DC00047D106F50A73274A033302EB03131B7905
:105DD0003F2B3ED82201234D02F50A52383204F5FA
:105DE0000A7B52190BF1030B02F1080105EB0B1BA7
:105DF00004321D4B089107920BF1080098470346A7
:105E00009BF804004FF0180E0EFB005000F50260E6
:105E100070448088099D00B20090CAEB05000A9D7D
:105E2000C0B20190681C48440B9DC0B20290B5FB03
:105E3000F7F00238C0B20490CDF80CA00B480899D6
:105E4000079A0B4DA847082393FBF7F399445FFA91
:105E500089F90134102CA3D1092000E028460DB0A7
:105E6000BDE8F08FD0070020C11E0008B52601084C
:105E7000A55600082DE9F04F8FB081469DF86400CB
:105E800090460022079106901346AC48342101FB4E
:105E9000020101F5A45191F838404C4503D0383146
:105EA0000979494501D101339BB20132402AECD135
:105EB000403ADFF888C20C2101FB02C101F58E5186
:105EC00091F83800484503D038310979494501D166
:105ED00001339BB20132102AEBD1103A97480C21C2
:105EE00001FB020101F5945191F83800484503D0B7
:105EF00038310979494501D101339BB20132102A69
:105F0000ECD1103ADFF834C2142101FB02C101F5D3
:105F10009A5191F83800484507D091F83C00383143
:105F2000484502D0097A494501D101339BB201327B
:105F3000102AE7D1103A02F506718048033100EBD0
:105F40000111097A49450ED002F58071013100EB4B
:105F5000011101F58C5191F82C002831484502D0EF
:105F6000097A494501D101339BB20132102AE2D1AD
:105F7000103A02F50A71DFF8C4C103310CEB0111CC
:105F8000097A49450ED002F5887101310CEB0111F7
:105F900001F58C5191F82C002831484502D0097A3E
:105FA000494501D101339BB20132102AE1D1002BC6
:105FB00000F02685042B28BF0423049304980323B0
:105FC00093FBF0F3023BDBB24FF0000B079DCA4698
:105FD00005931C465E46C146584A342707FB0B27EB
:105FE00007F5A45797F838303037534533D1544923
:105FF000544B08A898473979504B490159182C310E
:10600000514B08A89847514F08A8B847A5F10A0373
:10601000181A04EB0901FF2300930193C9B208AADF
:10602000DFF83C81C0B2C047DDF810C0062393FB07
:10603000FCF308A8E418B847B042E4B203D908A8B2
:10604000424B98470646062C05D90F3DAD1B059CD3
:1060500005F0FF050026342000FB0BF0374A02EB69
:10606000000C0CF5A45C9CF83C30534548D10DF174
:106070003808002708F8187D0CF13C00CDF80CC05A
:10608000334B984701233A460146009340463B462E
:10609000304FB8472C4F30494046B847DDF80CC068
:1060A00040469CF83410DFF894C0490161442C311B
:1060B000B847264F4046B847A5F10A03181A04EB23
:1060C0000901FF2300930193C9B24246DFF890C053
:1060D000C0B2E0470498062393FBF0F308A8E41845
:1060E000B847B042E4B203D908A8184B984706460F
:1060F000062C05D90F3DAD1B059C05F0FF050026BC
:106100000BF1010BBBF1400F7FF466AFABF1400B1D
:106110000A4A0C2707FB0B2707F58E5797F83830EC
:106120003037534549D10D49064B08A8984739796E
:10613000024B490159182C3114E000BFD007002050
:10614000BE260108E1110008991100089DFE000813
:10615000751E0008F5230008BD260108C5260108A4
:10616000CDFE0008AA4B08A89847AA4F08A8B84730
:10617000A5F10A03181A04EB0901FF230093019308
:10618000C9B208AADFF8B082C0B2C047DDF810C0BB
:10619000062393FBFCF308A8E418B847B042E4B226
:1061A00003D908A89B4B98470646062C05D90F3DF6
:1061B000AD1B059C05F0FF0500260C2000FB0BF035
:1061C000954A02EB000C0CF58E5C9CF83C30534574
:1061D00048D10DF13808002708F8187D0CF13C0073
:1061E000CDF80CC08D4B984701233A4601460093E9
:1061F00040463B468A4FB847854F8A494046B84794
:10620000DDF80CC040469CF83410DFF80CC24901A0
:1062100061442C31B8477F4F4046B847A5F10A0387
:10622000181A04EB0901FF2300930193C9B24246F7
:10623000DFF804C2C0B2E0470498062393FBF0F3F2
:1062400008A8E418B847B042E4B203D908A8714BD3
:1062500098470646062C05D90F3DAD1B059C05F059
:10626000FF0500260BF1010BBBF1100F7FF450AFBF
:10627000ABF1100B684A0C2707FB0B2707F5945767
:1062800097F838303037534533D16749674B08A802
:1062900098473979604B490159182C315C4B08A853
:1062A00098475C4F08A8B847A5F10A03181A04EBF1
:1062B0000901FF2300930193C9B208AADFF878818E
:1062C000C0B2C047DDF810C0062393FBFCF308A85A
:1062D000E418B847B042E4B203D908A84D4B984738
:1062E0000646062C05D90F3DAD1B059C05F0FF05A4
:1062F00000260C2000FB0BF0474A02EB000C0CF5CB
:10630000945C9CF83C30534548D10DF13808002787
:1063100008F8187D0CF13C00CDF80CC03F4B9847B5
:1063200001233A460146009340463B463C4FB8475E
:10633000374F3F494046B847DDF80CC040469CF80F
:106340003410DFF8D4C0490161442C31B847314FD3
:106350004046B847A5F10A03181A04EB0901FF23C8
:1063600000930193C9B24246DFF8CCC0C0B2E04707
:106370000498062393FBF0F308A8E418B847B0424A
:10638000E4B203D908A8234B98470646062C05D942
:106390000F3DAD1B059C05F0FF0500260BF1010B21
:1063A000BBF1100F7FF466AFABF1100B1A4B142743
:1063B00007FB0B3707F59A5797F8382030375245C7
:1063C00049D11C49194B08A898477979124A4901C3
:1063D00051182C310E4B08A898470E4F08A8B84703
:1063E000A5F10A03181A04EB0901FF230093019396
:1063F000C9B208AADFF84080C0B2C047DDF810C0BB
:10640000062393FBFCF308A8E418B847B04215E054
:10641000991100089DFE0008D0070020751E000895
:10642000F5230008C4260108CC260108E111000864
:10643000CB260108D2260108CDFE0008E4B203D91C
:1064400008A8A74B98470646062C04D90F3DAD1B5C
:10645000059C05F0FF05142000FB0BF0A14A02EBA0
:10646000000C0CF59A5C9CF83C30534548D10DF17A
:106470003808002708F8187D0CF13C00CDF80CC056
:10648000994B984701233A460146009340463B46C4
:10649000964FB847964F97494046B847DDF80CC02D
:1064A00040469CF83510DFF83CC2490161442C316C
:1064B000B8478B4F4046B847A5F10A03181A04EBBA
:1064C0000901FF2300930193C9B24246DFF834C2A9
:1064D000C0B2E0470498062393FBF0F308A8E41841
:1064E000B847B042E4B203D908A87D4B98470646A6
:1064F000062C05D90F3DAD1B059C05F0FF050026B8
:10650000142000FB0BF0774A02EB000C0CF59A5CB0
:106510009CF84030534549D10DF138080027101838
:1065200008F8187D704BCDF80CC000F59C509847CA
:1065300001233A460146009340463B466B4FB8471D
:106540006B4F6C494046B847DDF80CC040469CF89C
:106550003510DFF890C1490161442C31B847604FD4
:106560004046B847A5F10A03181A04EB0901FF23B6
:1065700000930193C9B24246DFF888C1C0B2E04738
:106580000498062393FBF0F308A8E418B847B04238
:10659000E4B203D908A8524B98470646062C05D901
:1065A0000F3DAD1B059C05F0FF0500260BF1010B0F
:1065B000BBF1100F7FF4FAAEABF1100B0BF50677C1
:1065C000484A033702EB07173B7A534532D14A4911
:1065D0004A4B08A898473979424B490159182C3140
:1065E000434B08A898473E4F08A8B847A5F10A03AF
:1065F000181A04EB0901FF2300930193C9B208AAFA
:10660000DFF80081C0B2C047DDF810C0062393FB5D
:10661000FCF308A8E418B847B042E4B203D908A8CC
:106620002F4B98470646062C04D90F3DAD1B059C01
:1066300005F0FF050BF580700130DFF8A8C0000100
:106640000CEB000303F58C5328331B79534563D1BE
:1066500060440DF13808002700F58C5008F8187DCB
:106660002C30CDF80CC0204B984701233A46014608
:10667000009340463B461D4FB8471D4F20494046BA
:10668000B847DDF80CC00BF5067303330CEB0313AE
:106690001B7940465B019C440CF12C01B847104F1C
:1066A0004046B847A5F10A03181A04EB0901FF2375
:1066B00000930193C9B24246DFF848C0C0B2E04738
:1066C0000498062393FBF0F308A8E418B847B042F7
:1066D000E4B219D908A8024B9847064614E000BF57
:1066E0009DFE0008D0070020751E0008F523000855
:1066F00099110008D1260108D8260108E1110008E7
:10670000D7260108CDFE0008062C05D90F3DAD1B8C
:10671000059C05F0FF0500260BF580700130DFF8C1
:10672000CCC200010CEB000303F58C5328331B7A19
:1067300053454DD160440DF13808002700F58C50C9
:1067400008F8187D3030CDF80CC0A34B98470123D2
:106750003A460146009340463B46A04FB847A04FFB
:10676000A0494046B847DDF80CC00BF5067303336B
:106770000CEB03131B7940465B019C440CF12C018C
:10678000B847994F4046B847A5F10A03181A04EBD9
:106790000901FF2300930193C9B24246DFF85CC2AE
:1067A000C0B2E0470498062393FBF0F308A8E4186E
:1067B000B847B042E4B203D908A88B4B98470646C5
:1067C000062C05D90F3DAD1B059C05F0FF050026E5
:1067D0000BF1010BBBF1100F7FF4F0AEC846ABF12B
:1067E000100B0BF50A77814A033702EB07173B7A48
:1067F000534532D17E497F4B08A8984739797B4B66
:10680000490159182C31764B08A89847764F08A8AB
:10681000B847A5F10A03181A04EB0901FF230093F6
:106820000193C9B208AADFF8D481C0B2C047DDF82D
:1068300010C0062393FBFCF308A8E418B847B04245
:10684000E4B203D908A8684B98470646062C04D939
:106850000F3DAD1B059C05F0FF050BF58870013061
:10686000DFF888C100010CEB000303F58C532833DB
:106870001B7953454DD160440DF13808002700F5D0
:106880008C5008F8187D2C30CDF80CC0524B98472E
:1068900001233A460146009340463B464F4FB847D6
:1068A0004F4F55494046B847DDF80CC00BF50A7309
:1068B00003330CEB03131B7940465B019C440CF142
:1068C0002C01B847484F4046B847A5F10A03181AAB
:1068D00004EB0901FF2300930193C9B24246DFF89C
:1068E0001CC1C0B2E0470498062393FBF0F308A84C
:1068F000E418B847B042E4B203D908A83A4B984725
:106900000646062C05D90F3DAD1B059C05F0FF057D
:1069100000260BF588700130DFF8D0C000010CEBC9
:10692000000303F58C5328331B7A53454DD1604443
:106930000DF13808002700F58C5008F8187D30302C
:10694000CDF80CC0244B984701233A4601460093EA
:1069500040463B46214FB847214F27494046B8475C
:10696000DDF80CC00BF50A7303330CEB03131B7932
:1069700040465B019C440CF12C01B8471A4F40463D
:10698000B847A5F10A03181A04EB0901FF23009385
:106990000193C9B24246DFF864C0C0B2E047049830
:1069A000062393FBF0F308A8E418B847B042E4B21A
:1069B00003D908A80C4B98470646062C05D90F3D6D
:1069C000AD1B059C05F0FF0500260BF1010BBBF18B
:1069D000100F7FF406AF14E0751E0008F5230008C1
:1069E00099110008D72601089DFE0008D007002055
:1069F000DE260108E1110008E3260108CDFE0008AB
:106A0000079D079A551BE8B20FB0BDE8F08F00BF95
:106A1000012908B5104605D113785AB2632A0ADC59
:106A2000013307E002290BD113785AB212F1630F38
:106A300001DB013B03700121074B9847002008BD93
:106A40000339C9B2012904D80121034B9847012019
:106A500008BD002008BD00BFC52C00082DE9F0438B
:106A6000464B05461E7889B0FF2E084690461C46C8
:106A700063D1434E03213246424CA0473378424C07
:106A8000009328462146414D0DF11F020323A847DC
:106A9000B146247808254BE0022C45D899F800101F
:106AA00028460B1B594241EB0301394B9847012CF7
:106AB000334E0AD0022C1DD031782846D1F1010185
:106AC00038BF0021334B98472EE03349334B03A89E
:106AD0009847334B03A89847002203AB98F900105E
:106AE0001818009413462F4FB8473278284603A948
:106AF000012A14E02C49294B03A89847284B03A8E6
:106B0000984701230022009303AB98F9011018184D
:106B1000244F1346B8473278284603A9022A14BFE7
:106B200000220122214B984708350134EDB2E4B22E
:106B30009DF81F30A342AFD81CE0012E09D002D32C
:106B4000022E17D108E01A4A01201070FF221A7095
:106B500011E0184B586802E0164B01329868FF2389
:106B6000154DA847012805D1114B1870FF2323703C
:106B7000013800E0002009B0BDE8F083D401002016
:106B8000C4030020113D000890030020F5490008CF
:106B9000CD3B0008FD3C0008432C0108E111000832
:106BA0009D120008F5230008EA260108913A000822
:106BB0009E000020E4000020116A00082DE9F04F3B
:106BC000814B8DB093F800808246B8F1FF0F0E46DE
:106BD00014461D4665D17D4F08463A4611217C4E2C
:106BE000B047DFF818823B7841460093794E8146E2
:106BF0000DF12F0250461123B04798F800604FF076
:106C0000080831E0397840468B1B594241EB0301BB
:106C1000714B98473A783EB9D2F10101404638BFEE
:106C200000216E4B984719E0082E09D8C6EB020CDC
:106C3000DCF100024046314642EB0C02684B0CE0AE
:106C4000684BC6EB020EA6F1090153F82110DEF1E4
:106C50000002654B404642EB0E02984708F10808D7
:106C600001365FFA88F8F6B29DF82F30B342C9D8E2
:106C70005E4B3E7898475E4B07469847013E32236D
:106C8000333F0938F6B20093FFB22A3BC0B20193FA
:106C900003903146029720460122083B554EB047EB
:106CA00060E1B8F1000F05D1534A01201070FF22B6
:106CB0001A707AE1B8F1090F0ED100231A460721A4
:106CC00092FBF1F16439C832E018E1540433B2F5B3
:106CD000C86F4170F3D148E1B8F10A0F0ED100231B
:106CE0006422E118E2540433202B4A70F8D17C333B
:106CF000237063709C3B2371637136E1B8F10B0F15
:106D00001BD100226423A118A3540432202A4B7003
:106D1000F8D17C3222706270627133322272CF3AC3
:106D2000CE2162723120627332322274217120735B
:106D3000637423756375313A18E1B8F10C0F0BD108
:106D40000023E21892F90110043301EBD1714910CC
:106D5000202B5170F5D108E1B8F10D0F08D10023B7
:106D6000E218517804334942202B5170F8D1FCE0ED
:106D7000B8F10E0F12D10023E21851780139517089
:106D800049B211F1640F01DA9C2102E0642901DDAE
:106D9000642151700433202BEED1E6E0B8F10F0FDF
:106DA0002ED10023E21851780131517049B211F10E
:106DB000640F01DA9C2102E0642901DD6421517035
:106DC0000433202BEED1D0E03801002087030020CF
:106DD000113D0008F5490008CD3B0008FD3C0008C6
:106DE0006D3A00087C000020913A0008BF010108BC
:106DF000C3010108554C00089E000020D803002064
:106E0000B8F1100F6A4FDFF8C091DFF8C0B16ED152
:106E1000DFF8A881FF23674E67484246B04798F8DD
:106E20000030099046460BB9013333703378402B5C
:106E300002D9624B40221A7095F800C096F800A063
:106E40000CF1FF3C5FFA8CFCDFF884813423CDF831
:106E500014C00AF1FF3A03FB0A8AB8470690C847F4
:106E60000790B8470890B8470746C847069A079B57
:106E7000D208D2B200920522B3FBF2F303EB430334
:106E8000DBB20899019383080139013BDDF814C096
:106E90000AF5A65AA1EB9707DBB20AF1080A039399
:106EA000043A0023FFB2504661460297D847099B37
:106EB000012B5FD10022134630780D21013801FBF0
:106EC000003000F5A66008EB8000007AA05430780E
:106ED000013801FB003101F5A66108EB8101487A18
:106EE0000133A1180432082B4870E5D13DE0B847C2
:106EF0000746C847322309380093333F2A3BC0B2C4
:106F000008F1FF3101220193FFB2083B0390C9B29F
:106F100020460297D8472B785046013B04EB83026A
:106F20003146DBB2264FB847012E81460DD12346AC
:106F300004F11C011A7893F9046050B28642B8BF7C
:106F40001A7104338B42F5D10CE0022E0AD10023D2
:106F5000E2181279E05651B28842C8BFE2540433B5
:106F60001C2BF5D1B9F1010F04D10122154B1A7078
:106F7000FF232B700023E25612F1640F01DA9C22EA
:106F800002E0642A01DD6422E254E21892F9011061
:106F900011F1640F01DA9C2102E0642901DD642112
:106FA00051700433202BE6D100200DB0BDE8F08FE6
:106FB000BF01010899430008ED2601089E03002047
:106FC0005D6A00089E000020C3010108554C0008BE
:106FD000D00700202DE9FF474B4E824635781446F6
:106FE000FF2D69D1DFF834810846424643213346FC
:106FF000464FB847DFF84C9198F800300DF10F027A
:107000000093434F432350464946B847414B4746B8
:107010001A78FF2A04D01B780127237035706FE09F
:1070200099F80040082541E0397828460B1B594261
:1070300041EB0301384B394E98473CB9327828462A
:10704000D2F10102364938BF00220FE0012C04D1F1
:10705000327828463349012A05E0022C08D13278DB
:1070600031492846022A14BF002201222F4B18E082
:10707000422C17D832782846C4EB020CDCF100020F
:1070800042EB0C022A49294B98473278294B61017F
:10709000C4EB020EC918DEF10002274B284642EB72
:1070A0000E02984708350134EDB2E4B29DF80F3076
:1070B000A342B9D8002723E0204A214B2DB9FF2154
:1070C000012721701770317017E0012D09D1FE21C1
:1070D00021701570FF2232702046294698472F46AE
:1070E0000EE0022D4FF0010702D1FD21217001E0D9
:1070F000033D25701770FF223270204639469847AD
:10710000384604B0BDE8F0879C000020113D00081F
:1071100009480008E9010020453C0008D50300208B
:10712000FD2601080C2701081C270108B5370008B7
:10713000282701089C070020F53700089E00002042
:10714000C52C000884030020F0B5334B06461046DA
:107150001A7885B0FF2A4CD1304C0846224641218E
:107160002F4DA84723782F4D0093304629462E4EA9
:107170000DF10F024123B0472D78082633E0217826
:1071800030464B1B594241EB0301284B234F984794
:1071900045B93A783046D2F10102254938BF00227C
:1071A000244B1BE0402D1AD83A783046C5EB020C30
:1071B000DCF1000242EB0C021F491E4B98471F4BAB
:1071C0006A1E182101FB02313A780431C5EB020E28
:1071D000DEF100021A4B304642EB0E0298470836A9
:1071E0000135F6B2EDB29DF80F30AB42C7D80020A2
:1071F0000FE014490124144D1AB9FF3202700C70CB
:1072000003E0013A02700C70FF221A702146A84771
:10721000204605B0F0BD00BF3901002082030020E8
:10722000113D0008AC03002009480008453C000857
:107230002E270108B537000833270108F80F002072
:10724000F53700089E000020C52C00082DE9F04FFE
:10725000137889B0FD2B074614460BD003F1020AC0
:107260005FFA8AFABAF1010F94BF4FF0020A4FF0A9
:10727000040A01E04FF0030A8B4D95F80180B8F144
:10728000FF0F40F0DC8008462A4651466B1C874EB3
:10729000B0472B7886490DF11F0238460093854E82
:1072A0005346854FB047B847DFF86CB20646D8471B
:1072B0008146B8470122A6F10801009200264A46FD
:1072C000DFF8589203460196029603963046C9B2FB
:1072D000DFF8E8C1E04799F83A30002B3AD0B847D8
:1072E00099F83A3004900593D8478346B847059BF0
:1072F000049ADB43D2180BF1FF3B431E01213046B9
:1073000000910196D1B202965FFA8BF20396DBB23E
:107310006A4EB0476A4E2B7856F82300694B98475F
:107320008346B847684B99F83A201B7899F83A1089
:10733000CDF80080CB1A03EBD373C2EB63012B783B
:107340004118CDF8048056F823205846C9B2434668
:107350005E4EB047564B08261F786BE029783046C2
:10736000CB1B594241EB0301594B984757455DD21E
:1073700023785849FD2B584B0DD1022F0BD14A4A87
:10738000304612780969A2F1020CDCF1000242EBEE
:107390000C02984734E02A783046C7EB020EDEF143
:1073A000000242EB0E0251F827109847022F27D017
:1073B0003D4B032F1A7829D0012F484B2FD194F839
:1073C00000E0BEF1FF0F02D1304645490AE0BEF1B0
:1073D000FE0F02D13046434904E0BEF1FD0F03D158
:1073E00041493046012A1DE0BEF13F0F05D83F4913
:1073F0004FEA4E1E30467144F4E730463C49F1E70F
:107400002A78304694F90110022A03E094F9021018
:107410003046032A14BF00220122364B05E03649CC
:107420003046BA4214BF002201229847083601377D
:10743000F6B2FFB29DF81F30BB428FD87DE0B8F1A5
:10744000030F7AD8DFE808F0020D246C2B4B0126DD
:107450001E70FF236B7020460421294B984730464D
:107460006CE01C4B274E58682246FF23B047264F3E
:1074700006463B78FF2B5AD0244B98473878244B4C
:107480009847002801DD642300E09C2363704EE0F0
:10749000FD2B104B04F101020CBF186998681D4EBA
:1074A000FF23B04742E000BF4C010020113D00081F
:1074B0008903002009480008C30101085DFA00089B
:1074C000C0010020952D0008F000002015FF0008E5
:1074D000453C000800000020B5370008F5370008DB
:1074E000FD2601080C2701081C270108FC070020C5
:1074F0003A2701082D3A0008F92901089E000020CA
:10750000C52C0008D56F0008E9010020B906010864
:10751000A908010865440008BF010108502C00209B
:10752000084BA21CD868084CFF23A0470646012E32
:1075300003D1064B1E70FF236B70002009B0BDE81D
:10754000F08F00BF00000020654400089E0000206E
:107550002DE9F04F137891B0FD2B0746154601D168
:107560000233137095F800A0974C0AF1020A94F8C0
:1075700005805FFA8AFABAF1010F94BF4FF0020A50
:107580004FF0050AB8F1FF0F40F0F0800846221DC9
:107590005146631D8D4EB04723798D490DF13F0251
:1075A000384600938B4E53468B4FB047B847DFF8B1
:1075B0009CB20646D8478146B8470122A6F1080189
:1075C000009200264A46DFF888920346019602960A
:1075D00003963046C9B2DFF804C2E04799F83A3062
:1075E000002B3AD0B84799F83A3004900593D84721
:1075F0008346B847059B049ADB43D2180BF1FF3B47
:10760000431E0121304600910196D1B202965FFAE5
:107610008BF20396DBB2714EB047714E237956F868
:107620002300704B98478346B8476F4B99F83A2030
:107630001B7899F83A10CDF80080CB1A03EBD3737E
:10764000C2EB630123794118CDF8048056F823205A
:107650005846C9B24346654EB0475D4B08261F7871
:107660007EE021793046C7EB010CDCF1000141EBF3
:107670000C015F4B984757456ED2534B30461A79F1
:107680005C4BC7EB020EDEF1000253F8271042EB11
:107690000E02594B98477B1E032B52D8DFE803F0AC
:1076A00002353B452978DFF88481FF2903D122790F
:1076B0003046524922E0FE2903D122793046504912
:1076C0001CE0A1F14003DBB2BD2B14D94D4B4901A5
:1076D000C91807A84C4B98474C4B284698474C4B29
:1076E00010B107A84B4901E04B4907A898472279F8
:1076F000304607A902E0227948493046A2F1010349
:107700005A4242EB0302C04726E02279304695F9FF
:107710000110022A04E0227995F902103046032A6A
:1077200014BF002201223E4B15E022793046A2F11F
:10773000040CDCF1000295F9031042EB0C02394B0A
:1077400009E022793849C7EB020EDEF10002374B1F
:10775000304642EB0E02984708360137F6B2FFB2C8
:107760009DF83F30BB423FF67CAF80E0B8F1040F9C
:107770007DD8DFE808F0030E20236F002C4B012694
:107780001E70FF236371284604212A4B9847304618
:107790006EE0184B284E58682A46FF23B047274B07
:1077A00006461B78FF2B5CD0254B984764236B70F3
:1077B000503BAB7055E023486A1C02E00D4BAA1CFD
:1077C000D868FF23204D4AE04C010020113D0008FD
:1077D0009403002009480008C30101085DFA00086D
:1077E00068000020952D0008F000002015FF00081B
:1077F000453C0008CC000020B53700088E26010863
:1078000085260108FC070020E1110008C11E0008C0
:1078100099110008782601087E2601083A270108F8
:107820002D3A00085D380008F9290108F5370008ED
:107830009E000020C52C0008D56F0008E90100203B
:10784000B9060108D400002065440008BF01010802
:10785000502C0020084BEA1C084D1869FF23A8474C
:107860000646012E03D1064B1E70FF2363710020D4
:1078700011B0BDE8F08F00BFCC0000200D2E000835
:107880009E0000202DE9F04F894D8FB0894E804633
:10789000B0472B78FF2B40F086814FF00A0CA0F107
:1078A0000A0797FBFCF7CDF810C0FFB28248834B64
:1078B00098474FEA470A824C402191FBFAF1224651
:1078C0002B46013140467F4DDFF80882A847C0476C
:1078D0000C3800EBD070401080B20690B04724788E
:1078E000A0F10905C047640095FBF7F57C43074606
:1078F000B0470121431E7A1E0020009101900290A2
:1079000003900731D2B2DBB26F4EB04706990698AA
:10791000C9B2E4B2400801F108035FFA80F9DBB2B2
:1079200004F1010BDDF810C0544409F10408EAB277
:107930000134994408350D9409905FFA88F80A914A
:1079400007935FFA89F90B92EDB2644620E1059E38
:107950005E4A7301D31838339B796FF063015BB2D1
:107960008B42B8BF0B46069F642BA8BF642303FB62
:1079700007F0C921DDF824C090FBF1F1614489B220
:10798000002B0C914FF0010301F104020DDD009377
:10799000FE330193643B0293963B0393404621469A
:1079A000D2B22B46484EB0470BE00093FF23019321
:1079B000FA3B02930393D0B2214642462B46424FF4
:1079C000B84704F1020AFF269B275FFA8AFA40466D
:1079D000214642465346DFF800C1009601970297C0
:1079E000E047AB1EDBB219460893404642462B46A1
:1079F000DFF8E4C0009601970297E0470C99DFF8A2
:107A0000D8C0081DC0B202465146089B0096019797
:107A10000297E04705982D4942018A182C321046FA
:107A200004922B4B9847A8EB50005146049A3346DA
:107A3000DFF8A8C000960196C0B2E0470A9800237C
:107A4000021D009304202146D2B22B46DFF878C0F5
:107A5000019602960396E0471C484FEA4B13C31861
:107A600038339B796FF063025BB29342B8BF134621
:107A7000069A642BA8BF642303FB02F1DDF824C03F
:107A8000C92291FBF2F26244079892B2002B059250
:107A90004FF00103024423DD009304330196039366
:107AA000029748462146D2B22B46074EB04722E005
:107AB00035000020C301010841270108A13E00084C
:107AC00092030020113D00080DFC0008D0070020A3
:107AD0009DFE0008BF01010861FD0008CDFE000801
:107AE0000093052302930393D0B2019621464A46A0
:107AF0002B46324FB847FF269B2721460096019719
:107B0000029748464A465346DFF8B4C0E0472B4642
:107B1000DFF8ACC0009601970297484608994A469C
:107B2000E0470799059A089B8818C0B2024600965C
:107B3000019702975146224FB847DFF894C04FEAA9
:107B40004B1767442C3738461E498847A9EB50002D
:107B50003A4633460096019651461B4FC0B2B8478D
:107B6000DDF828C000234FEA4C020832009301964A
:107B70000296039621462B46079802F0FE020F4E0E
:107B8000B0470B9F0BF1020BE419ED19E4B2EDB213
:107B9000DDF834C0E3450CD00BF1FF303F280590F1
:107BA0007FF7D5AE05E0094B01201870FF232B703D
:107BB00000E000200FB0BDE8F08F00BF0DFC000812
:107BC00061FD00089DFE0008CDFE00089E0000201B
:107BD000D00700202DE9F04F904D91B0904E804697
:107BE000B0472B78FF2B40F096814FF00A0CA0F1A4
:107BF0000A0797FBFCF7CDF818C0FFB289488A4BFB
:107C000098474FEA470A894C402191FBFAF12246F6
:107C10002B4601314046864DDFF82082A847C047F9
:107C20000C3800EBD070401080B20890B047247838
:107C3000A0F10905C047640095FBF7F57C430746B2
:107C4000B0470121431E7A1E00200091019002904E
:107C500003900731D2B2DBB2764EB047089908984C
:107C6000C9B2E4B2400801F108035FFA80F9DBB25F
:107C700004F1010BDDF818C0544409F10408EAB21C
:107C80000134994408350F940B905FFA88F80C91F1
:107C900009935FFA89F90D92EDB2644630E1664AC4
:107CA000079E182303FB062303F5026318339B8802
:107CB00014211BB293FBF1F378398B42B8BF0B460A
:107CC000089F642BA8BF642303FB07F0C921DDF8DC
:107CD0002CC090FBF1F1614489B2002B0E914FF062
:107CE000010301F104020DDD0093FE330193643BB7
:107CF0000293963B039340462146D2B22B464D4E0B
:107D0000B0470BE00093FF230193FA3B02930393E8
:107D1000D0B2214642462B46464FB84704F1020AEC
:107D2000FF269B275FFA8AFA404621464246534681
:107D3000DFF80CC1009601970297E047AB1EDBB25B
:107D400019460A93404642462B46DFF8F4C0009697
:107D500001970297E0470E990A9B081DC0B20246A0
:107D60005146DFF8DCC0009601970297E04707987C
:107D7000314B182101FB003202F502620C32104631
:107D80000692DFF8C0C0E047A8EB50005146069AC3
:107D90003346DFF8B4C000960196C0B2E0470C98B5
:107DA0000023021D009304202146D2B22B46DFF8A7
:107DB00084C0019602960396E0471F49182000FBF5
:107DC0000B1C0CF502631B189B8814221BB293FB3F
:107DD000F2F3783A9342B8BF1346089A642BA8BFCF
:107DE000642303FB02F1DDF82CC0C92291FBF2F2FF
:107DF0006244099892B2002B07924FF001030244AB
:107E000024DD0093043301960393029748462146EC
:107E1000D2B22B46074EB04723E000BF9D000020A2
:107E2000C301010850270108A13E0008C203002039
:107E3000113D00080DFC0008D0070020BF0101081B
:107E400061FD00089DFE0008CDFE0008009305239B
:107E500002930393D0B2019621464A462B46334FF4
:107E6000B847FF269B272146009601970297484670
:107E70004A465346DFF8B8C0E0472B46DFF8B0C0AB
:107E800000960197029748460A994A46E0470999A1
:107E9000079A0A9B8818C0B202460096019702977B
:107EA0005146234FB847DFF898C0182707FB0BC788
:107EB00007F502670C3738461E498847A9EB500082
:107EC0003A4633460096019651461B4FC0B2B8471A
:107ED000DDF830C000234FEA4C02083200930196CF
:107EE0000296039621462B46099802F0FE020F4E99
:107EF000B0470D9F0BF1020BE419ED19E4B2EDB29E
:107F0000DDF83CC0E3450CD00BF1FF303F28079073
:107F10007FF7C5AE05E0094B01201870FF232B70D9
:107F200000E0002011B0BDE8F08F00BF0DFC00089C
:107F300061FD00089DFE0008CDFE00089E000020A7
:107F4000D00700202DE9F04FAD4F93B0A7F51050AA
:107F5000AC4B97F878A097F879B097F87A60984783
:107F6000A94B984701238DF84130DB188DF842303A
:107F700001338DF8433001338DF8443001338DF8EF
:107F8000453001334FF000088DF84630013387F853
:107F900078A08DF8408087F879B08DF8473087F861
:107FA0007A609A4C4FEA481020182C309849994D25
:107FB00008F10108A847B8F1400FF2D1A8F1400834
:107FC000182000FB084000F502600C30904908F1D1
:107FD0000108A847B8F1400FF2D14FF0000E34204D
:107FE00000FB0E40FF2200F5A45080F8342000F181
:107FF0003001383002724FF0FE0C9B3A42720EF1A3
:10800000010E81F808C0FD2101714271643ABEF190
:10801000400F7E4B8271E2D183F84A2083F84920D9
:1080200083F8481083F86A2083F8692083F8681081
:1080300083F88A2083F8892083F8881083F8AA209F
:1080400083F8A92083F8A810CE2387F8553087F845
:10805000573087F859309C3B87F85B30313B87F8C5
:10806000542087F85630013387F85830013387F8A9
:108070005A30694B102E00F25B87DFE816F01100D2
:10808000110011001100110011000803080308037A
:1080900059075907DB05DB0559079C0663069C0653
:1080A0000022711E84F8282010460132042908D8C5
:1080B000DFE801F007030303060084F8280002E06C
:1080C000022284F82820554853F82610A847BAF110
:1080D000020F18D0BAF1030F1ED0BAF1000F4FF003
:1080E00003080CBF4FF0020C4FF0010CCDF82080BC
:1080F000CDF818C00CBF4FF001084FF0020818BFB0
:108100004FF0000A0EE00020032108904FF0010814
:10811000CDF818A0079107E00022012308924FF044
:1081200002080693CDF81CA0079F3D49780120184E
:108130002C30A847DDF818A03A494FEA4A10201819
:108140002C30A8474FEA4810201837492C30A84750
:10815000DDF820C035494FEA4C1020182C30A847D4
:1081600033493448A8479DF842003349400120185C
:1081700000F5B670A84731493148A847314932481F
:10818000A84732493248A84732493348A8473348BC
:108190003349A84700220123BBF1030F72D8DFE85F
:1081A0000BF0020E20618DF8413002238DF8423031
:1081B00001338DF843308DF8402001331CE08DF8F9
:1081C000403002238DF84130023B8DF842300333BA
:1081D0008DF8433001338DF8443003338DF845304A
:1081E00050E08DF8413003238DF84230013B8DF88B
:1081F00043308DF8402002338DF844300133EDE7F1
:10820000D02B0020651C000841200008D00700206A
:108210003A270108E1110008F4000020E8070020D7
:1082200060270108652701081B2201086A27010849
:10823000702701087C080020782701089C26010887
:10824000FC090020A12601085C0A00208127010802
:108250003C0A002084270108BC090020DC0900201A
:108260008B2701088DF8443002238DF8413001330B
:108270008DF8453001338DF8433001338DF84020BF
:108280008DF842309DF840104FF0180909FB01FAB3
:1082900004EB0A0000F5026009910C307949A84707
:1082A0009DF8412078490B9209FB02F2A01800F5D5
:1082B000026003920C30A8479DF842B0734909FB55
:1082C0000B4000F502600C30A8479DF84330704920
:1082D00009FB034000F502600D930C30A8479DF8A0
:1082E00044C06C4909FB0CF3E01800F502600493EC
:1082F000CDF828C00C30A8479DF84500664909FB19
:1083000000FC0C9004EB0C0000F50260CDF814C0EA
:108310000C30A8479DF84610604F09FB014000F55E
:1083200002600E910C305E49A8479DF847005D49F8
:108330000F9009FB004000F502600C30A84707F5DC
:108340000E60A2440C305849A8470AF50265002087
:10835000FD214D44A87268722972049BE31803F54D
:1083600002634B44987258721972039AA21802F56C
:1083700002624A44907250721172DDF814C0644473
:1083800004F502644C44A07260722172079A07F5EA
:10839000A45484F83420099B07F5A6521370642373
:1083A00053700A9D4FF09C0C09F1E609957082F814
:1083B00003C084F8389084F83C1084F83EC084F8F8
:1083C0003D30DDF818A0012E82F828A00B9C82F821
:1083D000344082F835300C9D82F8365082F83730C0
:1083E00082F82C9082F8301082F832C082F8313056
:1083F000DDF820A007F5A85282F81CA00D9C08F11A
:10840000020A82F8284007F5A95482F8293084F836
:10841000009082F8241007F5AC5482F826C082F848
:10842000253007F5AE5241D84FEA4A1A5744012584
:108430000426BD7102F8706CDDF838A002F864AC57
:1084400002F8633C02F86C9C02F8681C02F866CCE7
:1084500002F8673C84F8048084F810B0637484F8F0
:108460000890217384F83860DDF824C082F804C0D5
:1084700053710A9D9571D37184F83C90117090707E
:108480005370C3E091270108982701081B220108B7
:108490006A2701089F270108A6270108D0070020A6
:1084A00070270108842701088B2701084FEA4A1A20
:1084B00007EB0A054FF0010A85F806A00D95C74D98
:1084C0004FF00E0A85F8108085F81CB06B7785F8A0
:1084D0001490297685F81AC06B7684F804A00F9D55
:1084E00025740825637484F80890217384F80EC0FD
:1084F000637384F8388015710735537184F83C50E4
:10850000117082F802C053700D9DFF242C720BF184
:108510000A0507F50654A84607F5075584F834B050
:1085200084F8389084F83C1084F83E0084F83D309C
:1085300085F800804B2584F842304FF0EC0884F831
:10854000415007F50A5484F834B084F838A084F810
:10855000398084F83AC084F83C1084F83E0084F8EE
:108560003DC007F50B5C8CF800104FF0140C84F83C
:108570004200042E84F8413084F844B084F848A0C6
:1085800084F849C00CF1A60C84F84A8084F84C1099
:1085900084F84E0084F84DC084F8501084F85200DE
:1085A00084F8513032D1122482F83040079E82F88C
:1085B0002C60DDF82C80B52682F8388082F839509E
:1085C000DDF830A082F83AA082F83B6082F83410DF
:1085D00082F8360082F8353007F5B05282F8244030
:1085E000DDF818C007F5B15787F800C0099C82F87C
:1085F0002C4082F82D500A9E82F82E6082F82F506F
:1086000082F8281082F82A0082F82930744A079FDD
:10861000FD2100242D20102582F8347082F8385076
:1086200082F83C1082F83E4082F83D00DDF8188068
:10863000134603F8408F1D7119729C725872DDF851
:1086400020A083F80CA01D7419759C7558751334FF
:10865000053082F8F47082F8F84082F8FC1082F855
:10866000FE00193082F8FD0002F5807382F8008167
:1086700082F8044182F8081114229A72587283F821
:108680000CA01C7419759A75587500F08ABC0422E8
:1086900084F82820534853F82610A847BAF1020F4F
:1086A00016D0BAF1030F1BD0BAF1000F4FF0030C34
:1086B000CDF818C00CBF4FF001084FF002080CBFF6
:1086C0004FF002094FF0010918BF4FF0000A0DE00A
:1086D0000020D14606904FF001084FF0030A05E054
:1086E000002106914FF002084FF001094FEA4A10AD
:1086F00020182C303C49A8474FEA491020182C304C
:108700003A49A8474FEA481020182C303849A84762
:10871000069A3849500120182C30A8473649374866
:10872000A84737493748A84737493848A8473849FC
:108730003848A84738493948A84739493948A847E7
:108740000AF102035B01E318187A37494001201847
:108750002C30A84709F102035B01E318187A33496A
:10876000400120182C30A84708F102035B01E318F0
:10877000187A2F49400120182C30A847069F2D4910
:10878000BB1C5B01E318187A0027400120182C302D
:10879000A84784F8E070284984F8DE702748A84785
:1087A00084F80071264984F8FE702648A84784F8AA
:1087B0002071254984F81E712448A84784F8407127
:1087C000234884F83E712349A8470523BBF1030FD2
:1087D00067D8DFE80BF058414B5800BF101D002050
:1087E00090190020E8070020AD270108B2270108F2
:1087F000B72701086A2701089C260108FC09002008
:10880000A1260108DC090020812701083C0A00207C
:1088100084270108BC090020BD2701085C0A00204C
:10882000C22701087C080020CD270108D7270108AE
:10883000E1270108EC270108F82701089C0800201F
:1088400007280108BC08002016280108DC080020C1
:10885000FC0800202128010801228DF84130022364
:108860008DF842308DF840209B1808E08DF840309C
:1088700001238DF84130DB188DF8423001338DF83B
:108880004330033B0BE001238DF84130DB188DF8BA
:10889000423001338DF843308DF8407001338DF84C
:1088A00044309DF840304FF0180B0BFB034C0CF597
:1088B000026C0CF10C0C60460493CDF814C0D14945
:1088C000A8479DF84120D04F0BFB02F0211801F57D
:1088D00002610C310392099007910846CB49A847E1
:1088E0009DF842100BFB01F00A90201800F5026081
:1088F00008910C30C649A8479DF84300C5490BFBB9
:1089000000F00B90201800F502600C30A8479DF88D
:1089100044100BFB01FB04EB0B0000F502600C3074
:10892000BD49A84707F50A600430BC49A847062E90
:1089300007F5A65407F5A45607F5A855039A049B16
:10894000DDF814C05ED108F10200400101213818A1
:108950008171DDF828C007EB0C0080F83E18DDF8C7
:1089600024C007EB0C0080F83E18DDF82CC007EBA4
:108970000C005F4480F83E1887F83E18563186F8A0
:1089800034A0237061705231A2704FF0FE0CE17080
:10899000FD274539002086F838C086F83C7086F8F7
:1089A0003E0086F83D10CE2684F8289084F83430B6
:1089B00084F8356084F8362084F83760089E84F89F
:1089C000386084F8391084F82CC084F8307084F84A
:1089D000320084F8311085F81C8085F8283085F83D
:1089E000291085F82A2085F82B1085F82C6085F849
:1089F0002D1084F860C085F8247085F8260085F86D
:108A0000251038E0604603920493854F8549B847A6
:108A100085490798B84786F834A0049BFE27237041
:108A2000FD2064230021637086F8387086F83C00CE
:108A300086F83E1086F83D3084F82890DDF820C096
:108A400084F834C084F8353084F82C7084F8300011
:108A500084F8321084F8313085F81C80039A85F848
:108A60002820724A85F82930177085F8240085F887
:108A7000261085F825306E4A642182F810809DF812
:108A800043C0FE26082382F81CC051771675137662
:108A9000DA339376C43B537682F844809DF8447071
:108AA000FD20002582F8507082F8511082F848604D
:108AB00082F84C0082F84E5082F84D10DDF8188094
:108AC000042402F5546382F8788082F884C082F826
:108AD00085104FF0130C82F87C6082F8800082F8D9
:108AE000825082F8811082F8AC40013482F8B8409C
:108AF00082F8B91082F8B06082F8B40082F8B650FB
:108B000082F8B51083F8347083F838C0ACF10C0CDF
:108B100083F83CC00CF1210C83F83EC00CF1B00C82
:108B200083F83DC04FF00E084FF0140C82F8800D12
:108B300083F8425083F8411083F8447083F84880EA
:108B400083F849C00CF1D80C83F84AC083F84C4034
:108B5000013483F84E5083F84D1083F8504096341A
:108B600083F8525083F8514083F8547083F858804A
:108B700083F859C083F85A4083F85C0083F85E504C
:108B800083F85D1083F8600083F8625083F86140D9
:108B90009DF8401002F5446383F83410322183F8C5
:108BA000386083F83C0083F83E1083F83D1082F86B
:108BB000800C83F8421083F841109DF8412083F81F
:108BC000442083F8486083F84C0083F84E1083F803
:108BD0004D1083F8500083F8521083F851109DF81F
:108BE000422083F8542083F8586083F85C0083F8AF
:108BF0005E1083F85D1083F8600083F8621083F8DC
:108C00006110CEE12F280108D00700203628010886
:108C1000B22701086A2701081B220108C2270108A0
:108C2000E1110008AD270108B7270108F01C00205A
:108C3000101D00200D2253F8261084F82820A84883
:108C4000A847A849A848A847A849A948A847A949A2
:108C5000A948A847A949AA48A847AA49AA48A8478D
:108C60009DF84090182606FB094000F50260A749D0
:108C70000C30A8479DF84180A54906FB084000F547
:108C800002600C30A8479DF84270A24906FB0740DD
:108C900000F502600C30A8479DF843A09E4906FBF2
:108CA0000A4404F502600C30A8479C49012381F86E
:108CB00034300B4603F8408F6422FD249C20FE25AF
:108CC000183E5A709F70DA7083F804A05A7181F8C8
:108CD000385081F83C4081F83E6081F83D2083F8AF
:108CE000286083F8349083F8352083F82C5083F87B
:108CF000304083F8320083F8312081F89C600323F0
:108D000081F8A88081F8A92081F8AA70122781F83B
:108D1000AB0081F8A07081F8A44081F8A60081F82A
:108D2000A52081F8D0309DF8443081F8DC3081F8FE
:108D3000DD2081F8D45081F8D84081F8DA0081F83C
:108D4000D9202EE1132284F82820D96B6448A84743
:108D5000002101200A463E2926DC342606FB024675
:108D6000642506F5A45300F1010C06F5A65683F818
:108D7000342083F8401083F8415083F8420083F890
:108D8000435086F804C000F1020C757186F806C0E5
:108D9000F571FE2683F83860013E83F83C60FD3EA5
:108DA00083F83E6083F83D50013204300431402A9C
:108DB000C0B2D0D1F5E0132284F82820484853F8F7
:108DC0002610A84700274FEA471804EB080A0AF1C3
:108DD0002C0A53495046A8475046DFF84CA1D047CB
:108DE00040444FF0010C0022791C2018CDF800C03F
:108DF0002C301346CDF814C009B2DFF830B1D84793
:108E0000A044002288F84020102E5FFA87F9DDF890
:108E100014C004D1043288F8412088F842C0B9F166
:108E20000F0F21D80C2303FB0743FF2003F58E52BD
:108E300082F83490FD2182F83800FF3882F83C1027
:108E400082F83E002D3082F83D0003F59453322223
:108E5000D13083F8349083F8380083F83C1083F8DD
:108E60003E20921883F83D200137402FABD10023DC
:108E7000342202FB034202F5A45282F8343064210A
:108E800082F84030FE26013382F84110FD2082F83E
:108E90003860FE3E402B82F83C0082F83E6082F84B
:108EA0003D10E5D14FF0180808FB06F804EB080761
:108EB00007F502670C371B493846A8473846D047A4
:108EC0004044201801230022013600F5026000937F
:108ED0000C3031B21346D847402EE3D161E000BFD9
:108EE000E80700203D280108FC070020452801086C
:108EF0001C0800204E2801083C08002052280108C8
:108F00005C0800205C2801083C0A00206528010854
:108F10006B2801087228010879280108501C0020DC
:108F200080280108892801089D120008F5230008FF
:108F3000052253F8261084F828201C48A8471C490D
:108F40001C48A8471C491D48A8471D491D48A8475B
:108F50001D481E49A8470D2E05D11023FB73093B60
:108F60007B73073BBB730023342202FB0342FE20CA
:108F700002F5A452FD2582F8343082F8380082F8D8
:108F80003C50613D82F83E50383D82F83D5082F8B9
:108F90004030013302F13001102B82F84150087249
:108FA000E2D1012013B0BDE8F08F00BFE807002038
:108FB0003D280108FC070020452801081C08002066
:108FC0004E2801083C0800205C0800209028010879
:108FD0002DE9F043324D87B06B780646FF2B2C46C7
:108FE00050D12A466B1C08462E4D1121A8472378E4
:108FF0002D4D0DF117022946304600932B4E1123BB
:109000002B4FB047B8472B4B814693F83A802A4BF9
:1090100098470646B847C8EB0908034601220020D6
:109020000092019032460290244E03905FFA88F13C
:10903000B0472D7808261FE0217830464A1B514260
:1090400041EB02011E4B9847102D11D8144B3046AE
:109050001A781C4B53F82510531B5A4242EB03025B
:10906000194B9847194B30465957FF22184B9847D0
:1090700008360135F6B2EDB29DF81730AB42DBD8B9
:10908000002009E013701046124B01219847124B43
:1090900001201870FF236B7007B0BDE8F08300BF9C
:1090A000B4000020113D0008A40300200948000876
:1090B000C3010108502C0020BF0101085DFA00081F
:1090C000453C0008F4000020B53700088024010862
:1090D0008D380008C52C00089E0000202DE9F043C3
:1090E000314D87B06B780646FF2B2C464ED12A4671
:1090F0006B1C08462D4D0421A84723782C4D0DF1FB
:1091000017022946304600932A4E04232A4FB047BF
:10911000B8472A4B814693F83A80294B9847064630
:10912000B847C8EB090803460122002000920190CD
:1091300032460290234E03905FFA88F1B0472D78B3
:1091400008261DE021783046C5EB010CDCF100015A
:1091500041EB0C011C4B9847032D0DD8124B3046A8
:109160001A781A4BC5EB020EDEF1000253F82510F7
:1091700042EB0E02164B984708360135F6B2EDB2B7
:109180009DF81730AB42DDD8002009E0137010467F
:10919000104B01219847104B01201870FF236B7072
:1091A00007B0BDE8F08300BFCA000020113D0008F1
:1091B000D603002009480008C3010108502C0020F4
:1091C000BF0101085DFA0008453C0008B800002016
:1091D000B5370008C52C00089E0000202DE9F0439B
:1091E0002F4D87B06B780646FF2B2C464AD12A4676
:1091F0006B1C08462B4D0421A84723782A4D0DF1FE
:109200001702294630460093284E0423284FB047C2
:10921000B847284B814693F83A80274B9847064633
:10922000B847C8EB090803460122002000920190CC
:1092300032460290214E03905FFA88F1B0472D78B4
:10924000082619E0217830464A1B514241EB0201C1
:109250001B4B9847032D0BD8114B30461A78194BEE
:1092600053F82510531B5A4242EB0302164B984702
:1092700008360135F6B2EDB29DF81730AB42E1D8B1
:10928000002009E013701046104B01219847104B45
:1092900001201870FF236B7007B0BDE8F08300BF9A
:1092A000D7010020113D0008A9030020094800084B
:1092B000C3010108502C0020BF0101085DFA00081D
:1092C000453C00083C010020B5370008C52C0008CB
:1092D0009E0000202DE9F043314D87B06B780646A3
:1092E000FF2B2C464ED12A466B1C08462D4D0521DE
:1092F000A84723782C4D0DF11702294630460093DC
:109300002A4E05232A4FB047B8472A4B814693F887
:109310003A80294B98470646B847C8EB09080346E8
:10932000012200200092019032460290234E0390C9
:109330005FFA88F1B0472D7808261DE02178304685
:10934000C5EB010CDCF1000141EB0C011C4B984713
:10935000042D0DD8124B30461A781A4BC5EB020E6D
:10936000DEF1000253F8251042EB0E02164B98472F
:1093700008360135F6B2EDB29DF81730AB42DDD8B4
:10938000002009E013701046104B01219847104B44
:1093900001201870FF236B7007B0BDE8F08300BF99
:1093A000D5010020113D0008830300200948000872
:1093B000C3010108502C0020BF0101085DFA00081C
:1093C000453C0008A0000020B5370008C52C000867
:1093D0009E0000202DE9F04F7C4C89B094F8599004
:1093E0000746B9F1FF0F164640F0BE80084604F16B
:1093F0005802052104F15903754DA84794F85830D7
:1094000074490DF11F0238460093734D0523734FC5
:10941000A847B847DFF80C82DFF80CA2059098F84F
:109420003A50D0478346B84705990122491B002589
:109430000346009201955A46029503952846C9B203
:10944000DFF8E8B1D84798F83A30002B3BD0B8475E
:1094500098F83A3004900593D0478246B847059B68
:10946000049ADB43D2180AF1FF3A431E0121284631
:1094700000910195D1B202955FFA8AF20395DBB2B1
:10948000D847574D94F8583055F82300554B984716
:109490008246B847544B98F83A201B7898F83A100F
:1094A000CDF80090CB1A03EBD373C2EB630194F8B1
:1094B00058304118CDF8049055F823205046C9B2D1
:1094C0004B464A4DA847434B08251F7847E094F880
:1094D00058102846CA1B514241EB0201444B9847A1
:1094E000042F38D8394B284693F85820414B53F86D
:1094F0002710D31B5A4242EB03023F4B98477B1E77
:10950000032B28D8DFE803F0020B141D317894F800
:1095100058203A4B284653F82110012A16E071785A
:1095200094F85820364B284653F82110022A0DE0B3
:10953000B17894F85820334B284653F82110032A69
:1095400004E094F8582030492846042A14BF002229
:1095500001222E4B984708350137EDB2FFB29DF836
:109560001F30BB42B3D82CE0B9F1040F29D8DFE893
:1095700009F01A03081117001E4B254D5868FF23E8
:1095800004E01C4B234D98680132FF23A8470128B3
:1095900010D016E0174B0232D8681F4DFF23F5E7B5
:1095A00008461E4B98471E4B01201870FF2384F875
:1095B000593007E01A4B1870FF2384F859300138EE
:1095C00000E0002009B0BDE8F08F00BF4C01002092
:1095D000113D0008CB03002009480008C301010821
:1095E00038000020952D0008F000002015FF00082D
:1095F000453C000818000020B5370008B8000020DE
:109600003C010020F4000020F9290108F53700088A
:10961000DD900008DD910008D18F0008457F00082B
:109620009E000020502C0020BF0101085DFA0008B8
:109630002DE9FF41C1EB030E9DF828C01FFA8EFEF5
:109640000CFB0EFCDCB26FF063039CFBF3FCCEB2B0
:10965000E6446533C7B2D5B206EB0E0100937F3303
:1096600001930293039338462A462346C9B2DFF892
:109670002080C04700230093FF330193029303939C
:10968000384631462A462346C047BDE8FF8100BF21
:109690000DFC00082DE9F04F954B89B00E46984718
:1096A000944B044698470121A21F831FFF240320E7
:1096B0000091013902910391D2B20146DBB28E4D85
:1096C0000194A84705200094019401468B4A234643
:1096D0008B4DA847012E05D18A4B1A78022A08D84B
:1096E000013205E0022E04D1864B1A780AB1013A04
:1096F0001A70854A13789046CBB91A4602F59061E4
:1097000082480F3100EBC1010020C8804FF61000E5
:1097100088804FF4FE6008817D490020C8527D4951
:109720000132C8520233042AE8D1012354E0012B4C
:1097300055D1FF24784F7948B84723460D21774A01
:1097400000940194A8477648B84723461521744AE7
:1097500000940194A8477348B847009401942346A5
:109760001D21704AA847DFF8D4A1FF3CB946204626
:109770006D4B98470134E4B2042C2AF8020FF6D15D
:10978000604B634F1B78002237F9131001230093BD
:1097900005A81346654CA04705A8C847FF23252107
:1097A0000093019305AAA847032E40F09D806049CD
:1097B000002303F59062554C38880F3204EBC20247
:1097C0000133D0800022042B27F8022B21F8022F2E
:1097D000EFD198F80030013388F8003084E0022B94
:1097E00040F08280FF244C4F4C48B84723460D215F
:1097F0004A4A00940194A8474E48B8472346152189
:109800004C4A00940194A8474648B84723461D2176
:10981000444A00940194A8474748B84700940194EB
:1098200023462521444AA847394F3A4C4FF00009B6
:10983000BA46A34648463C4B984737F9023B09F1E4
:109840000109984234F9023BB8BF27F8020C5FFACD
:1098500089F99842C8BF24F8020CB9F1040FE9D184
:10986000284F00223B78A9F10309FF243AF913108D
:1098700005A81346DFF8B4A0CDF80090D0472D21FD
:109880000A2005AA234600940194A8473B780022A9
:109890003BF9131005A81346CDF80090D04764207B
:1098A0002D210094019405AA2346A847032E1BD11D
:1098B00022481F49002303F59062144C0F3204EB39
:1098C000C202D48830F8025F01332C1B9480D48804
:1098D00031F8025F042BC4EB05041481EBD1043B87
:1098E00088F80030012000E0002009B0BDE8F08FCA
:1098F000BF010108C30101080DFC0008F131010896
:1099000015FF0008CC03002097030020D00700209B
:10991000B0030020B8030020952D00089928010805
:10992000A0280108A7280108A9080108F5230008B4
:10993000B6030020AE280108B3280108AE030020BA
:109940002DE9F04F002389B081464FF00108904A7D
:10995000590151183831097A934619B908F10108AB
:109960005FFA88F80133402BF1D1B8F1010F00F014
:109970000981884B5C781D46FF2C40F0C9801A464F
:1099800041460133844E4846B0472B78834F0093BD
:109990008348434683490DF11F02834EB04797F831
:1099A0003A30002B34D0DFF84892C84797F83A3065
:1099B0007E4A0593824690470646C847059B721E1D
:1099C000DB439A440121431E0020D2B20091019052
:1099D0005FFA8AF102900390DBB2754EB047754B87
:1099E000754898470646C847744B97F83A201B7845
:1099F00097F83A100094CB1A03EBD373C2EB6301D0
:109A00004118019423463046C9B26B4A6C4CA047BA
:109A1000644B08261C7876E0297830460A1B5142B0
:109A200041EB0201674B9847444568D254B9594B02
:109A300030461A786449D2F1010238BF0022634BE4
:109A400098471EE00027B9467B010BEB0302383232
:109A5000127A92B9621E4A450BD14D4A3046D3184C
:109A60002A7803F12C01131B5A4242EB0302574B95
:109A7000984709F101095FFA89F90137402FE3D1CD
:109A80004CB92A783046D2F10102514938BF002240
:109A9000504B984733E04FF00009CA464FEA49134C
:109AA0005B4438331A7A2ABB611E51451ED1597A5C
:109AB00001290FD19F792B787FB2C4EB030C63315E
:109AC000DCF1000397FBF1F1304643EB0C03424F0E
:109AD000B8470BE02A789979C4EB020EDEF1000258
:109AE000304649B242EB0E023C4B98470AF1010A5C
:109AF0005FFA8AFA09F10109B9F1400FCED10836AF
:109B00000134F6B2E4B29DF81F30A34284D83BE0A2
:109B10002CB9334A01201070FF225A7035E000241E
:109B20002646204662010BEB02033833197AF1B95D
:109B30006F78013FB74218D1587A01280DD19A7930
:109B400012B964329A7100E09971600158443E3054
:109B50000121244B9847012007E00D4B22489A1819
:109B600049463E32FF23214FB8470136F6B2013451
:109B7000402CD7D1012807D1194B1870FF236B70E7
:109B8000013802E0404600E0002009B0BDE8F08F57
:109B9000D00700202C000020113D0008502C002090
:109BA000BA280108C303002009480008BF010108C2
:109BB0005DFA0008952D000887280108F0000020B4
:109BC00015FF0008453C000810260108B5370008BD
:109BD000F9290108F5370008D93800082D3A00089E
:109BE0009E000020C52C00082227010865440008BB
:109BF000C30101082DE9F047374C0025637886B092
:109C0000FF2B07468DF8175055D1084622460621EE
:109C1000631C324EB047324E237831460DF11702A5
:109C2000384600932F4F0623DFF8E480B847C0473B
:109C30002D4B824693F83A902C4B98470746C047E5
:109C4000C9EB0A090122034600920195029503958A
:109C500028465FFA89F1264D3A46A8473578082606
:109C600023E021783046C5EB010CDCF1000141EB2B
:109C70000C01204B9847052D13D8174B30461A7806
:109C80001D4BC5EB020EDEF1000253F8251042EB2E
:109C90000E021A4B98471A4B30465957FF22194B60
:109CA000984708360135F6B2EDB29DF81730AB4251
:109CB000D7D8002007E04BB1013B137010460121BB
:109CC000114B984702E006B0BDE8F0870F4B01202A
:109CD0001870FF236370F6E7C8000020113D0008EC
:109CE000A703002009480008502C0020BF010108EC
:109CF0005DFA0008453C000850000020B537000818
:109D0000B83901088D380008C52C00089E000020D5
:109D1000C30101082DE9F0475B4E86B074783546E3
:109D2000FF2C40F096803246731C4021574EB047BE
:109D30002B78574E00935748402357490DF117028F
:109D4000B047564E96F83A30002B33D0DFF890816A
:109D5000C047534B814696F83AA098470746C047FC
:109D60006FEA0A0A7A1E431E01210020D144D2B2B2
:109D7000009101905FFA89F102900390DBB2494FA4
:109D8000B847494B494898470746C047484B96F85B
:109D90003A201B7896F83A100094CB1A03EBD37351
:109DA000C2EB63014118019423463846C9B23F4AC9
:109DB000404CA047384B08261C7845E029783046AF
:109DC000C4EB010CDCF1000141EB0C013A4B98476C
:109DD0003F2CDFF8B48033D8384B394F84B998F82A
:109DE00000203046D2F1010238BF002235499847A1
:109DF0002A783046D2F10102334938BF00221EE0F2
:109E000098F80020DFF8D0906101C4EB020E4944BD
:109E10000C31DEF1000242EB0E0230469847631C23
:109E20005B014B449B7998F80020012BC4EB0203A3
:109E30000CBF264926495A42304642EB0302B84736
:109E400008360134F6B2E4B29DF81730A342B5D813
:109E500016E0204D24B90120FF232870737010E014
:109E600001341D486401001983790121C3F1010304
:109E700000F8063F194B984701232B70FE3373708F
:109E8000002006B0BDE8F08730000020113D00083A
:109E900009480008C9280108C9030020502C0020E7
:109EA000BF0101085DFA0008952D00088728010808
:109EB000F000002015FF0008453C0008B5370008F9
:109EC000F537000810260108F92901083C2B010884
:109ED000242601089E000020D0070020C52C000881
:109EE000C30101082DE9F047624E86B0747835460B
:109EF000FF2C40F09E803246731C40215E4EB047DE
:109F00002B785E4E00935E4840235E490DF11702A8
:109F1000B0475D4E96F83A30002B33D0DFF8AC8175
:109F2000C0475A4B814696F83AA098470746C04723
:109F30006FEA0A0A7A1E431E01210020D144D2B2E0
:109F4000009101905FFA89F102900390DBB2504FCB
:109F5000B847504B504898470746C0474F4B96F874
:109F60003A201B7896F83A100094CB1A03EBD3737F
:109F7000C2EB63014118019423463846C9B2464AF0
:109F8000474CA0473F4B08261C784DE029783046C7
:109F9000C4EB010CDCF1000141EB0C01414B984793
:109FA0003F2CDFF8D0803BD83F4B404F84B998F826
:109FB00000203046D2F1010238BF00223C499847C8
:109FC0002A783046D2F101023A4938BF002226E011
:109FD000621E4FF0180A0AFB02FADFF8E89098F8C0
:109FE000002009EB0A01C4EB020E01F502610C31FD
:109FF000DEF1000242EB0E023046D144984709F5EB
:10A00000026318339B7998F80020012BC4EB0203FC
:10A010000CBF294929495A42304642EB0302B8474E
:10A0200008360134F6B2E4B29DF81730A342ADD839
:10A030001CE0234D24B90120FF232870737016E023
:10A040001823013C5C431F480121031993F83E2863
:10A050000019C2F1010200F5026083F83E281E30AB
:10A06000194B984701232B70FE337370002006B004
:10A07000BDE8F08714000020113D000809480008E1
:10A08000D8280108AB030020502C0020BF01010894
:10A090005DFA0008952D000887280108F0000020CF
:10A0A00015FF0008453C0008B5370008F5370008E3
:10A0B00010260108F92901083C2B01082426010873
:10A0C0009E000020D0070020C52C0008C301010815
:10A0D0002DE9F04F754C87B0667B8046FF2E154604
:10A0E00040F0B180084604F10C02072104F10D0391
:10A0F0006F4FB847237B4046DFF81C8200936D49C1
:10A1000007230DF117026C4FB84798F83A30002B2F
:10A1100038D0DFF80892C847684B824698F83AB0C2
:10A1200098470746C8476FEA0B0BDA447A1E431E6E
:10A1300001210020D2B2009101905FFA8AF10290D1
:10A140000390DBB25E4FB847237B5E4F57F8230086
:10A150005D4B98478246C8475C4B98F83A201B787D
:10A1600098F83A100096CB1A03EBD373C2EB630155
:10A17000237B4118019657F8232050463346C9B235
:10A18000534EB0474B4B08261F7857E0217B304693
:10A19000C7EB010CDCF1000141EB0C014D4B984782
:10A1A000062FDFF8088145D898F80C204A4BC7EBFA
:10A1B000020EDEF1000253F8271042EB0E02304689
:10A1C000464B98474FB998F864203D21D2F10102DF
:10A1D000304638BF0022424B2BE0BB1E042B04D874
:10A1E000DFE803F00D13191F2800227B3046A2F18F
:10A1F00001035A4242EB030229463A4B19E0227B03
:10A200003046B5F91010022A0FE0227B3046B5F92E
:10A210001210032A09E0227B3046B5F91410042AF3
:10A2200003E0227BA97D3046052A2F4B14BF002274
:10A230000122984708360137F6B2FFB29DF8173071
:10A24000BB42A3D82EE0062E2CD8DFE806F0040A85
:10A250000E1114191E00254B01201870FF23637383
:10A2600021E02348FF23234D13E02348103204E06C
:10A270002248123201E022481432FF23214D08E027
:10A2800021481632FF23214D03E02148214D183289
:10A29000FF23A847012805D1144B1870FF236373CF
:10A2A000013800E0002007B0BDE8F08F4C0100202D
:10A2B000113D00088803002009480008BF0101087B
:10A2C0005DFA000874250108952D0008F0000020B3
:10A2D00015FF0008453C000854390108B53700084F
:10A2E0008D380008F53700085D3800089E00002012
:10A2F0007F3401086D330008222701080328010874
:10A30000E22B0108ED320008162B01080D2E000883
:10A31000B32A0108D9420008502C0020C3010108CB
:10A320002DE9FF479246394A0746D37B1446FF2B57
:10A3300052D108460E32212104F10F03344DA847B3
:10A34000344EA37B3146009305460DF10F0238468B
:10A350002123314FB8473678082738E0A17B3846AB
:10A36000C6EB010CDCF1000141EB0C012B4BDFF8DB
:10A370009C8098474EB998F80E103846D1F10101EB
:10A3800038BF0021264B98471DE0202E1BD8731E96
:10A390004FF01C0909FB03A998F80E203846C6EBBC
:10A3A000020EDEF1000242EB0E0249461D4B9847B9
:10A3B00098F80E203846931B5A4242EB0302B9F933
:10A3C0001010194B984708370136FFB2F6B29DF8C6
:10A3D0000F30B342C2D80EE02BB9144B01201870D5
:10A3E000FF23D3730EE0013B1C2202FB03A2104D9E
:10A3F000DBB2A8470546012D03D10C4B1D70FF238E
:10A40000E373002004B0BDE8F08700BF4C010020DA
:10A41000113D0008D303002009480008453C00080E
:10A42000D53C0008B53700085D3800089E000020C4
:10A43000D1A000082DE9F04F824C87B0667E80469F
:10A44000FF2E154640F0C880084604F11802072187
:10A4500004F119037C4FB847237E4046DFF864823D
:10A4600000937A4907230DF11702794FB84798F8FE
:10A470003A30002B38D0DFF85092C847754B8246EF
:10A4800098F83AB098470746C8476FEA0B0BDA448A
:10A490007A1E431E01210020D2B2009101905FFA82
:10A4A0008AF102900390DBB26B4FB847237E6B4F6B
:10A4B00057F823006A4B98478246C847694B98F87B
:10A4C0003A201B7898F83A100096CB1A03EBD37316
:10A4D000C2EB6301237E4118019657F823205046B2
:10A4E0003346C9B2604EB047584B08261F786EE01D
:10A4F000217E3046CA1B514241EB02015B4B98471B
:10A50000062FDFF840815ED898F81820584B304667
:10A5100053F82710D31B5A4242EB0302554B98477E
:10A520004FB998F864203D21D2F10102304638BF7E
:10A530000022514B46E0BB1E042B04D8DFE803F099
:10A54000081F28333900227E30462978012A1AE074
:10A5500095F801E0494BBEF13F0F03D9227E30460A
:10A56000474905E047494FEA4E1E227E3046714476
:10A57000A2F1020CDCF1000242EB0C0222E0227E8E
:10A58000A9783046032A14BF002201223E4B19E06D
:10A59000227E291DA2F1040EDEF10002304642EBBC
:10A5A0000E023A4B0EE0227E304605F10801052AE4
:10A5B00004E0227E304605F10C01062A344B14BF1C
:10A5C00000220122984708360137F6B2FFB29DF803
:10A5D0001730BB428CD830E0062E2ED8DFE806F0CC
:10A5E000040A0E13181D20002A4B01201870FF23A7
:10A5F000637623E02848FF23284D15E028480132E0
:10A60000FF23284D10E028480232FF23274D0BE09E
:10A6100027480432FF23274D06E02748083201E08F
:10A6200026480C32264DFF23A847012805D1194B97
:10A630001870FF236376013800E0002007B0BDE802
:10A64000F08F00BF4C010020113D0008980300204E
:10A6500009480008BF0101085DFA00081424010838
:10A66000952D0008F000002015FF0008453C00086B
:10A6700064240108B53700088D380008F537000854
:10A680003A270108FC0700205D380008513B00080C
:10A69000B53A00089E000020162B01080D2E000878
:10A6A000502A0108D56F00080129010899430008C4
:10A6B00011290108517500081A29010857260108B7
:10A6C0004D720008502C0020C30101082DE9F04F05
:10A6D00093465E4A9846D37E87B0FF2B04461646C3
:10A6E00040F08A8008461A32112106F11B03584DAA
:10A6F000A847584DB37E2946009381460DF11702B5
:10A7000020461123544CA0472C7808256FE0B17ED9
:10A7100028460B1B594241EB0301504B98474CB95B
:10A720004A4B2846997E4E4BD1F1010138BF00219A
:10A73000984758E0102C56D8631E4FF0140A0AFBB5
:10A7400003BA9AF80130434514D1464B9847464B1B
:10A750006FF003021B780021D21A8218EB1D0091C2
:10A76000FF3101910291039102202946D2B2DBB25E
:10A770003E4FB8479AF801703D4B3F2F15D9B27E36
:10A780002846C4EB020CDCF1000242EB0C02394912
:10A790009847B27E2846C4EB020EDEF1000236492D
:10A7A00042EB0E02354B98471DE0B27E34497F01E3
:10A7B0007918171B7A4242EB070228469847294B23
:10A7C0009847294B6FF003021B78611ED21A82183A
:10A7D00008206B1C009003380190D2B2C8B2DBB2E3
:10A7E000FF21284FB84708350134EDB2E4B29DF897
:10A7F0001730A3428BD81CE02BB9234B01201870D3
:10A80000FF23D3761EE0B8F1FF0F08D01422013BDE
:10A8100002FB03B35A78FF2A08BF83F80180F37E56
:10A820001422013B204602FB03B2184CDBB2A047C6
:10A830008146B9F1010F04D1134B83F80090FF2337
:10A84000F376002007B0BDE8F08F00BF4C01002078
:10A85000113D00088603002009480008453C000817
:10A86000D53C0008BF010108340000205DFA000853
:10A87000B53700083A2701081D290108F5370008F7
:10A88000FC070020A95A00089E00002035A40008FB
:10A890002DE9F04F784C87B0667F8046FF2E154635
:10A8A00040F0BD80084604F11C02052104F11D039F
:10A8B000724FB847237F4046DFF8308200937049DB
:10A8C00005230DF117026F4FB84798F83A30002B67
:10A8D00038D0DFF81C92C8476B4B824698F83AB0E4
:10A8E00098470746C8476FEA0B0BDA447A1E431EA7
:10A8F00001210020D2B2009101905FFA8AF102900A
:10A900000390DBB2614FB847237F614F57F82300B4
:10A91000604B98478246C8475F4B98F83A201B78AF
:10A9200098F83A100096CB1A03EBD373C2EB63018D
:10A93000237F4118019657F8232050463346C9B269
:10A94000564EB0474E4B08271E7863E0217F3846AD
:10A950008B1B594241EB0301514B9847042EDFF802
:10A96000188153D898F81C204E4BC6EB020CDCF132
:10A97000000253F8261042EB0C0238464A4B984727
:10A980004EB998F864203D21D2F10102384638BF13
:10A990000022464B39E0032E98F81C2021D0042ECB
:10A9A00029D0022E14D095F800E0414BBEF13F0FA4
:10A9B00002D938463F4904E03F494FEA4E1E384627
:10A9C0007144A2F1010EDEF1000242EB0E021CE026
:10A9D000A2F102035A4242EB030238466978374B30
:10A9E00013E0A2F1030C291DDCF10002384642EB12
:10A9F0000C02334B09E0A2F1040EDEF10002314BF0
:10AA0000384605F1080142EB0E0298470837013637
:10AA1000FFB2F6B29DF81730B34297D827E0042E64
:10AA200025D8DFE806F003090D121700264B012098
:10AA30001870FF2363771BE02448FF23244D0DE0AB
:10AA400024480132FF23244D08E024480432FF2328
:10AA5000234D03E02348244D0832FF23A847012853
:10AA600005D1194B1870FF236377013800E00020EF
:10AA700007B0BDE8F08F00BF4C010020113D000879
:10AA8000AD03002009480008BF0101085DFA000875
:10AA900050240108952D0008F000002015FF000843
:10AAA000453C0008E4250108B53700088D3800084A
:10AAB000F53700083A270108FC0700205D38000838
:10AAC000513B0008B53A00089E000020502A0108BA
:10AAD000D56F0008162B01080D2E0008112901085A
:10AAE00051750008242901084D720008502C0020DF
:10AAF000C30101082DE9F04F90465E4A9B46D37F83
:10AB000087B0FF2B0446164640F08A8008461E3266
:10AB1000112106F11F03584DA847584DB37F294610
:10AB2000009381460DF1170220461123544CA04793
:10AB30002C7808256FE0B17F28460B1B594241EB6A
:10AB40000301504B98474CB94A4B2846997F4E4BCE
:10AB5000D1F1010138BF0021984758E0102C56D898
:10AB6000631E4FF00C0A0AFB03FA18F80A305B4523
:10AB700014D1464B9847464B6FF003021B780021D7
:10AB8000D21A8218EB1D0091FF31019102910391BD
:10AB900002202946D2B2DBB23E4FB84718F80A70FD
:10ABA0003D4B3F2F15D9B27F2846C4EB020CDCF198
:10ABB000000242EB0C0239499847B27F2846C4EBA9
:10ABC000020EDEF10002364942EB0E02354B984789
:10ABD0001DE0B27F34497F017918171B7A4242EB9E
:10ABE000070228469847294B9847294B6FF00302E4
:10ABF0001B78611ED21A821808206B1C0090033843
:10AC00000190D2B2C8B2DBB2FF21284FB847083555
:10AC10000134EDB2E4B29DF81730A3428BD81CE0AA
:10AC20002BB9234B01201870FF23D3771EE0BBF113
:10AC3000FF0F08D00C22013B534318F80320FF2AD2
:10AC400008BF08F803B0F37F0C22013B204602FB4B
:10AC50000382184CDBB2A0478146B9F1010F04D141
:10AC6000134B83F80090FF23F377002007B0BDE873
:10AC7000F08F00BF4C010020113D00088D03002023
:10AC800009480008453C0008D53C0008BF01010800
:10AC9000340000205DFA0008B53700083A270108A3
:10ACA0002D290108F5370008FC0700206D59000820
:10ACB0009E00002091A800082DE9F04F734C87B04A
:10ACC00094F821608046FF2E154640F0B680084675
:10ACD00004F12002042104F121036D4FB84794F8D8
:10ACE00020304046DFF80C8200936A4904230DF1BE
:10ACF0001702694FB84798F83A30002B3AD0DFF87E
:10AD0000F891C847654B824698F83AB0984707468D
:10AD1000C8476FEA0B0BDA447A1E431E012100205C
:10AD2000D2B2009101905FFA8AF102900390DBB2F7
:10AD30005B4FB84794F820305A4F57F823005A4BCE
:10AD400098478246C847594B98F83A201B7898F89C
:10AD50003A100096CB1A03EBD373C2EB630194F85D
:10AD600020304118019657F8232050463346C9B287
:10AD70004F4EB047474B08271E7859E094F82010F3
:10AD800038468B1B594241EB03014A4B9847032E2F
:10AD9000DFF8F88048D898F82020474BC6EB020C23
:10ADA000DCF1000253F8261042EB0C023846434B0C
:10ADB00098474EB998F864203D21D2F101023846F7
:10ADC00038BF00223E4B2EE0022E98F8202016D0ED
:10ADD000032E1ED095F800E03A4BBEF13F0F02D98A
:10ADE0003846394904E039494FEA4E1E3846714425
:10ADF000A2F1010EDEF1000242EB0E0213E0A2F11D
:10AE0000020C291DDCF10002384642EB0C02304BEB
:10AE100009E0A2F1030EDEF100022E4B384605F1E7
:10AE2000080142EB0E02984708370136FFB2F6B22E
:10AE30009DF81730B342A1D823E0032E21D8DFE8D4
:10AE400006F002090D12244B01201870FF2384F82C
:10AE5000213017E02148FF23214D08E0214804322A
:10AE6000FF23214D03E02148214D0832FF23A8474D
:10AE7000012806D1184B1870FF2384F821300138BF
:10AE800000E0002007B0BDE8F08F00BF4C010020BB
:10AE9000113D0008C003002009480008BF01010857
:10AEA0005DFA0008F0240108952D0008F00000204C
:10AEB00015FF0008453C00089C380108B53700081C
:10AEC0008D380008F53700083A270108FC070020F4
:10AED000513B0008B53A00089E000020502A0108A6
:10AEE000D56F0008112901085175000832290108A1
:10AEF0004D720008502C0020C30101082DE9F04FCD
:10AF00009046634A9B4692F8233087B0FF2B044655
:10AF1000164640F0908008462232112106F12303A4
:10AF20005C4DA8475C4D96F8223029460093814637
:10AF30000DF1170220461123584CA0472C78082504
:10AF400074E096F8221028460B1B594241EB03018E
:10AF5000534B984754B94E4B284693F82210514B07
:10AF6000D1F1010138BF002198475BE0102C59D87E
:10AF7000631E4FF00C0A0AFB03FA18F80A305B450F
:10AF800014D1494B9847494B6FF003021B780021BD
:10AF9000D21A8218EB1D0091FF31019102910391A9
:10AFA00002202946D2B2DBB2414FB84718F80A70E6
:10AFB000404B3F2F17D996F822202846C4EB020CAD
:10AFC000DCF1000242EB0C023B49984796F8222044
:10AFD0002846C4EB020EDEF10002384942EB0E02B5
:10AFE000374B98471EE096F8222036497F017918A2
:10AFF000171B7A4242EB0702284698472A4B98478C
:10B000002A4B6FF003021B78611ED21A82180820A7
:10B010006B1C009003380190D2B2C8B2DBB2FF21A2
:10B02000294FB84708350134EDB2E4B29DF8173026
:10B03000A34286D81EE033B9244B01201870FF23A9
:10B0400082F8233020E0BBF1FF0F08D00C22013B37
:10B05000534318F80320FF2A08BF08F803B096F8F6
:10B0600023300C22013B204602FB0382184CDBB24A
:10B07000A0478146B9F1010F05D1144B83F8009028
:10B08000FF2386F82330002007B0BDE8F08F00BF13
:10B090004C010020113D0008A003002009480008D1
:10B0A000453C0008D53C0008BF01010834000020E1
:10B0B0005DFA0008B53700083A2701083829010869
:10B0C000F5370008FC070020155800089E000020F6
:10B0D000B9AC00082DE9F04F9A4C87B094F8256080
:10B0E0008046FF2E154640F05B81084604F124029D
:10B0F0000D2104F12503944FB84794F824304046BD
:10B10000DFF89482009391490D230DF11702904FBF
:10B11000B84798F83A30002B3AD0DFF88092C84709
:10B120008C4B824698F83AB098470746C8476FEA72
:10B130000B0BDA447A1E431E01210020D2B200918B
:10B1400001905FFA8AF102900390DBB2824FB84718
:10B1500094F82430814F57F82300814B984782465A
:10B16000C847804B98F83A201B7898F83A10009618
:10B17000CB1A03EBD373C2EB630194F8243041186C
:10B18000019657F8232050463346C9B2764EB04751
:10B190006E4B08261F78CFE094F824103046CA1B67
:10B1A000514241EB0201714B98470C2FDFF894811B
:10B1B00000F2BE8098F824206D4B304653F82710DB
:10B1C000D31B5A4242EB03026A4B98474FB998F897
:10B1D00064203D21D2F10102304638BF0022664B87
:10B1E000A5E0BB1E0A2B07D8DFE803F01A2633467A
:10B1F0004D60677A8197A20095F800E05F4BBEF141
:10B200003F0F04D994F8242030465D4906E05D499B
:10B210004FEA4E1E94F8242030467144012A78E00B
:10B2200094F82420291DA2F1020CDCF10002304622
:10B2300042EB0C02544B7AE094F824203046A2F101
:10B24000030EDEF1000205F1080142EB0E024F4B46
:10B250006DE02A7B494B3F2A04D994F824203046DC
:10B26000474907E04A49182000FB021194F82420BE
:10B2700030460431042A4CE094F82420304695F9F5
:10B280000D10052A4FE0AA7B3C4B3F2A04D994F8C5
:10B29000242030463A4907E03D49182000FB0211BE
:10B2A00094F8242030460431062A32E094F8242011
:10B2B000304695F90F10072A35E02A7C2F4B3F2A9C
:10B2C00004D994F8242030462D4907E0304918204D
:10B2D00000FB021194F8242030460431082A18E0BB
:10B2E00094F82420304695F91110092A1BE0AA7C15
:10B2F000224B3F2A04D994F824203046204907E005
:10B300002349182000FB021194F824203046043110
:10B310000A2A14BF0022012209E094F8242095F99A
:10B32000131030460B2A1B4B14BF002201229847F2
:10B3300008360137F6B2FFB29DF81730BB423FF630
:10B340002BAF75E04C010020113D00089D0300204B
:10B3500009480008BF0101085DFA0008203901080A
:10B36000952D0008F000002015FF0008453C00085E
:10B3700088230108B53700088D380008F537000824
:10B380003A270108FC070020513B0008B53A0008A5
:10B39000F80F00205D380008502C0020C301010880
:10B3A0000C2E45D8DFE806F0070E10151A1D2023D5
:10B3B00026292C313600204B01201870FF2384F8F9
:10B3C000253036E01D481DE01D480432FF231D4D89
:10B3D00024E01D480832FF231C4D1FE01C480C329E
:10B3E00010E01C480D3212E01B480E320AE01B48E8
:10B3F0000F320CE01A48103204E01A48113206E00D
:10B4000019481232FF23194D08E019481332FF235F
:10B41000184D03E01848194D1432FF23A84701289E
:10B4200006D1054B1870FF2384F82530013800E061
:10B43000002007B0BDE8F08F9E00002041290108E0
:10B4400011290108517500084C2901084D720008A6
:10B450005429010861290108702901087D29010882
:10B460008C29010899290108A82901089943000895
:10B47000B529010865440008C4290108BD6B00080E
:10B480002DE9F04F9046644A994692F8273089B0EA
:10B49000FF2B0746164640F093800846263241218E
:10B4A00006F127035D4CA0475D4D96F826300490C9
:10B4B000009329465B4C38460DF11F024123A047FB
:10B4C0002C78082577E096F826102846C4EB010C66
:10B4D000DCF1000141EB0C01534B4F4F98474CB945
:10B4E00097F826102846D1F1010138BF00214F4BB3
:10B4F00098475CE0402C5AD8631E34225A4318F80F
:10B5000002100592FF2997F82620494B02D12846C0
:10B5100048490DE0FE2902D12846474908E03F2965
:10B5200004D84F0145492846791801E04449284686
:10B53000C4EB020EDEF1000242EB0E02DFF814A1B2
:10B540009847D047DFF810B16FF001019BF8002059
:10B55000631E891A41180520009096F826006A1C7F
:10B56000071B784240EB07000190C9B2D8B2D2B2B3
:10B570000823344FB847B9F1FF0F18D0059A18F8CF
:10B5800002304B4513D1D0479BF800306FF00102D9
:10B59000D21A00218218EB1D0091FF310191029116
:10B5A000039102202946D2B2DBB2274FB8470835B3
:10B5B0000134EDB2E4B29DF81F30A34283D81EE0FF
:10B5C00033B9224B01201870FF2382F8273020E086
:10B5D000B9F1FF0F08D03422013B534318F8032080
:10B5E000FF2A08BF08F8039096F827303422013B61
:10B5F00002FB03823846DBB2154CA0470490049B43
:10B60000012B05D1114B049A1A70FF2386F82730BD
:10B61000002009B0BDE8F08F4C010020113D00086A
:10B620009A03002009480008453C0008D53C000862
:10B63000B5370008FD2601080C270108FC0700208B
:10B640003A270108D95000085DFA00089E00002042
:10B65000D5B00008BF010108340000202DE9F04FEB
:10B66000924C89B0667C8046FF2E1546994640F084
:10B670004F81084604F110020E2104F111038C4F92
:10B68000B847237C4046DFF88082009389490E2327
:10B690000DF11F02884FB84798F83A30002B39D087
:10B6A000DFF868A2D04798F83A30844A0593834679
:10B6B00090470746D047059B7A1EDB439B440121F8
:10B6C000431E0020D2B2009101905FFA8BF10290EC
:10B6D0000390DBB27A4FB847237C7A4F57F82300A8
:10B6E000794B98478346D047784B98F83A201B7897
:10B6F00098F83A100096CB1A03EBD373C2EB6301B0
:10B70000237C4118019657F8232058463346C9B286
:10B710006F4EB047674B4FF009081E78BDE0217CA3
:10B7200038468A1B514241EB02016A4B98470D2E65
:10B73000DFF878A100F2AB809AF81020664B38460B
:10B7400053F82610931B5A4242EB0302634B98476F
:10B750004EB99AF864203D21D2F10102384638BF33
:10B7600000225F4B9847554B98475E4B6FF00302A2
:10B770001B78D21A8218731ED2B20C2B00F287806B
:10B78000DFE803F007121D2930373D44505B646D3C
:10B790007600227C3846A2F1010CDCF10002294639
:10B7A00042EB0C02504B08E0227C95F9121038460F
:10B7B000022A4E4B14BF00220122984767E0227CE8
:10B7C0003846A2F1030EDEF1000295F9131042EBA8
:10B7D0000E02434BF1E7237C0222384695F9141000
:10B7E000042B19E0237C0322384695F91510052B0C
:10B7F00012E0227C384695F91610062AD9E7237CF8
:10B800000122384695F91A10072B05E0237C95F99B
:10B810001B1005223846082B14BF00230123344F88
:10B82000B84734E0227C3846A2F109077A4205F194
:10B830001C0142EB07022F4BBFE708230093033B99
:10B840000193FF20494643462B4F1FE008230093F6
:10B85000033B0193FF2049464346284F16E0082347
:10B860000093033B0193FF2049464346244F0DE0DC
:10B8700005230093237C234FA3F10D014B4243EB9F
:10B88000010301931146484642460823B847013652
:10B8900008F10808F6B25FFA88F89DF81F3008F141
:10B8A000FF37B342FFB23FF63AAF84E04C010020CD
:10B8B000113D00089F03002009480008BF0101084E
:10B8C0005DFA0008E8380108952D0008F000002016
:10B8D00015FF0008453C000850230108B537000853
:10B8E0008D38000834000020F53700085D38000866
:10B8F000D9380008B53A0008155800086D590008F5
:10B90000A95A0008F14F0008502C0020C30101087B
:10B910000D2E50D8DFE806F0070D1114191C212652
:10B92000292E33383D42264B01201870FF236374C3
:10B9300042E02448FF23244D34E0244812320EE034
:10B9400023481332FF23234D2CE0234814320EE00A
:10B9500022481532FF23224D24E022481632FF23CD
:10B96000214D1FE021481A3201E021481B32FF23FC
:10B97000204D17E020481C32FF23204D12E02048C4
:10B98000204A4B46204D0DE02048214A4B46214D90
:10B9900008E02148214A4B46214D03E02148224A34
:10B9A000224D4B46A847012805D1054B1870FF23AF
:10B9B0006374013800E0002009B0BDE8F08F00BFDB
:10B9C0009E0000207F3401086D3300082227010803
:10B9D000AB2F0108B53E0008012A0108162B01080B
:10B9E000F59B00080C2A0108654400083C2B01085F
:10B9F000142A01080D2E0008202A01084D720008A3
:10BA0000A1260108841A0020FDAE00089C2601082A
:10BA1000C4190020F5AA0008AA260108441B00202A
:10BA2000CDA60008F7260108841C002081B4000878
:10BA30002DE9F04F8DB009927B4A0546D37C9346A1
:10BA4000FF2B40F0D6800846123241210BF1130340
:10BA5000764CA0479BF81230754C0790009328460F
:10BA600021460DF12F024123724DA8474FF00808DF
:10BA70002478B8E09BF812104046C4EB010EDEF1CA
:10BA8000000141EB0E016C4B98474CB9664A4046A9
:10BA9000917C6A4BD1F1010138BF002198479CE0AD
:10BAA000402C00F29A80099A04F1FF394FEA4913B9
:10BAB000D31808935C4B08999A7C4046151B6A4240
:10BAC00042EB05025E4B98475E4A90475E4A052767
:10BAD0001378554A00976FF0030AC3EB0A0A937C68
:10BAE0008244181B434208F1010643EB00035FFA4E
:10BAF00089F9F6B25FFA8AFA514601933246082371
:10BB0000524D4846A847C0EB0A0A5FFA8AFC4FF03C
:10BB1000080A6246FF20494633464D4DCDF818C00D
:10BB2000CDF800A00197A847DDF818C04946C0EB42
:10BB30000C0C5FFA8CFC6246FF203346454DCDF875
:10BB400018C0CDF800A00197A847DDF818C04946F5
:10BB5000C0EB0C0C5FFA8CFC6246FF2033463E4D76
:10BB6000CDF818C0CDF800A00197A8472E4A00973D
:10BB7000937CDDF818C0191B4B42C0EB0C0C43EB57
:10BB800001035FFA8CFC614632460193334D534604
:10BB9000CDF818C04846A847DDF818C0294BC0EBBF
:10BBA0000C0C5FFA8CF59847274B1A786FF003035B
:10BBB0009B1A1B189D4210D1089A083D92F9123029
:10BBC000EDB26421009301950296CDF80CA0049784
:10BBD00023480A460023234DA84708F108080134EA
:10BBE0005FFA88F8E4B29DF82F30A3423FF642AFE7
:10BBF0000EE02BB91C4B01201870FF23D37410E00A
:10BC0000099C013B5A01A218DBB2184CA0470790CF
:10BC1000079A012A04D1144B1A70FF238BF81330B2
:10BC200000200DB0BDE8F08F4C010020113D000850
:10BC3000CA03002009480008453C0008D53C00081C
:10BC4000B5370008BF01010834000020F14F00089B
:10BC5000155800086D590008A95A0008755E0008BB
:10BC6000272A0108755400089E0000205DB60008D0
:10BC70002DE9F04F774C87B094F829608046FF2E6D
:10BC8000154640F0BB80084604F12802052104F166
:10BC90002903714FB84794F828304046DFF82082D6
:10BCA00000936E4905230DF117026D4FB84798F8C0
:10BCB0003A30002B3AD0DFF80C92C847694B8246E5
:10BCC00098F83AB098470746C8476FEA0B0BDA4432
:10BCD0007A1E431E01210020D2B2009101905FFA2A
:10BCE0008AF102900390DBB25F4FB84794F8283096
:10BCF0005E4F57F823005E4B98478246C8475D4B1E
:10BD000098F83A201B7898F83A100096CB1A03EB73
:10BD1000D373C2EB630194F828304118019657F8A9
:10BD2000232050463346C9B2534EB0474B4B0827E9
:10BD30001E785EE094F8281038468B1B594241EB80
:10BD400003014E4B9847042EDFF808814DD898F830
:10BD500028204B4BC6EB020CDCF1000253F82610F6
:10BD600042EB0C023846474B98474EB998F864208E
:10BD70003D21D2F10102384638BF0022424B33E068
:10BD8000032E98F8282022D0042E25D0022E14D07D
:10BD900028783E4B3F2802D938463D4906E03D49C8
:10BDA0004FF0180E0EFB001138460431A2F1010EBF
:10BDB000DEF1000242EB0E0216E0A2F1020C291D98
:10BDC000DCF10002384642EB0C02334B0CE0384603
:10BDD00005F10801032A03E0384605F10C01042AA5
:10BDE0002E4B14BF00220122984708370136FFB2BC
:10BDF000F6B29DF81730B3429CD827E0042E25D820
:10BE0000DFE806F0030A0E131600254B0120187018
:10BE1000FF2384F829301AE02248FF23224D0BE04B
:10BE200022480432FF23224D06E02248083201E076
:10BE300021480C32214DFF23A847012806D1184B79
:10BE40001870FF2384F82930013800E0002007B083
:10BE5000BDE8F08F4C010020113D00089103002047
:10BE600009480008BF0101085DFA0008E839010827
:10BE7000952D0008F000002015FF0008453C000843
:10BE8000D0250108B53700088D380008F5370008BF
:10BE90003A270108F80F0020513B0008B53A000886
:10BEA0009E000020502A010849710008112901084C
:10BEB000517500081A290108572601084D7200081B
:10BEC000502C0020C30101082DE9F04F9046624A32
:10BED0009B4692F82B3087B0FF2B0446164640F065
:10BEE000918008462A32112106F12B035B4DA847A9
:10BEF0005B4D96F82A302946009381460DF11702D2
:10BF000020461123574CA0472C78082575E096F859
:10BF10002A1028460B1B594241EB0301524B98470C
:10BF200054B94D4B284693F82A10504BD1F10101DA
:10BF300038BF002198475CE0102C5AD804F1FF3A32
:10BF40004FEA0A1A18F80A305B4514D1484B984753
:10BF5000484B6FF003021B780021D21A8218EB1DA8
:10BF60000091FF3101910291039102202946D2B242
:10BF7000DBB2414FB84718F80A20404B3F2A17D987
:10BF800096F82A202846C4EB020CDCF1000242EBB2
:10BF90000C023B49984796F82A202846C4EB020E2B
:10BFA000DEF10002374942EB0E02374B984720E0A2
:10BFB0003649182000FB021196F82A200431171B7D
:10BFC0007A4242EB070228469847294B9847294B6B
:10BFD0006FF003021B78611ED21A821808206B1CB6
:10BFE000009003380190D2B2C8B2DBB2FF21284FD3
:10BFF000B84708350134EDB2E4B29DF81730A342DA
:10C0000085D81CE033B9234B01201870FF2382F838
:10C010002B301EE0BBF1FF0F07D0013B1B0118F8CE
:10C020000320FF2A08BF08F803B096F82B302046FB
:10C03000013B08EB0312184CDBB2A0478146B9F173
:10C04000010F05D1134B83F80090FF2386F82B30A6
:10C05000002007B0BDE8F08F4C010020113D000822
:10C06000AA03002009480008453C0008D53C000808
:10C07000BF010108340000205DFA0008B537000850
:10C080003A2701082D2A0108F5370008F80F00208B
:10C09000055C00089E00002071BC00082DE9F04FEF
:10C0A000764C87B094F82D608046FF2E154640F000
:10C0B000B980084604F12C02052104F12D03704FCC
:10C0C000B84794F82C304046DFF81C8200936D4945
:10C0D00005230DF117026C4FB84798F83A30002B42
:10C0E0003AD0DFF80892C847684B824698F83AB0D1
:10C0F00098470746C8476FEA0B0BDA447A1E431E7F
:10C1000001210020D2B2009101905FFA8AF10290E1
:10C110000390DBB25E4FB84794F82C305D4F57F870
:10C1200023005D4B98478246C8475C4B98F83A20FD
:10C130001B7898F83A100096CB1A03EBD373C2EB36
:10C14000630194F82C304118019657F8232050468B
:10C150003346C9B2524EB0474A4B08271E785CE0BE
:10C1600094F82C1038468A1B514241EB02014D4B8A
:10C170009847042EDFF804814BD898F82C204A4BBE
:10C18000384653F82610931B5A4242EB0302474BA2
:10C1900098474EB998F864203D21D2F10102384603
:10C1A00038BF0022424B33E0032E98F82C2022D0D7
:10C1B000042E25D0022E14D028783E4B3F2802D9D9
:10C1C00038463D4906E03D494FF0180E0EFB001180
:10C1D00038460431A2F1010CDCF1000242EB0C0202
:10C1E00016E0A2F1020E291DDEF10002384642EBF4
:10C1F0000E02334B0CE0384605F10801032A03E038
:10C20000384605F10C01042A2E4B14BF00220122EE
:10C21000984708370136FFB2F6B29DF81730B3429F
:10C220009ED827E0042E25D8DFE806F0030A0E1377
:10C230001600254B01201870FF2384F82D301AE0DA
:10C240002248FF23224D0BE022480432FF23224DD7
:10C2500006E02248083201E021480C32214DFF233C
:10C26000A847012806D1184B1870FF2384F82D30F9
:10C27000013800E0002007B0BDE8F08F4C0100203D
:10C28000113D00088503002009480008BF0101088E
:10C290005DFA000870390108952D0008F0000020B3
:10C2A00015FF0008453C0008B8220108B537000812
:10C2B0008D380008F53700083A270108F80F0020EC
:10C2C000513B0008B53A00089E000020502A0108A2
:10C2D0004971000811290108517500081A2901083F
:10C2E000572601084D720008502C0020C301010898
:10C2F0002DE9F04F9046624A9B4692F82F3087B066
:10C30000FF2B0446164640F0918008462E3211213C
:10C3100006F12F035B4DA8475B4D96F82E3029465A
:10C32000009381460DF1170220461123574CA04778
:10C330002C78082575E096F82E1028460B1B5942DC
:10C3400041EB0301524B984754B94D4B284693F8A3
:10C350002E10504BD1F1010138BF002198475CE00D
:10C36000102C5AD804F1FF3A4FEA0A1A18F80A308A
:10C370005B4514D1484B9847484B6FF003021B783C
:10C380000021D21A8218EB1D0091FF310191029118
:10C39000039102202946D2B2DBB2414FB84718F8C8
:10C3A0000A20404B3F2A17D996F82E202846C4EB86
:10C3B000020CDCF1000242EB0C023B49984796F874
:10C3C0002E202846C4EB020EDEF10002374942EB74
:10C3D0000E02374B984720E03649182000FB021127
:10C3E00096F82E200431171B7A4242EB07022846AA
:10C3F0009847294B9847294B6FF003021B78611E21
:10C40000D21A821808206B1C009003380190D2B217
:10C41000C8B2DBB2FF21284FB84708350134EDB26E
:10C42000E4B29DF81730A34285D81CE033B9234B02
:10C4300001201870FF2382F82F301EE0BBF1FF0FA0
:10C4400007D0013B1B0118F80320FF2A08BF08F89A
:10C4500003B096F82F302046013B08EB0312184C2E
:10C46000DBB2A0478146B9F1010F05D1134B83F828
:10C470000090FF2386F82F30002007B0BDE8F08F32
:10C480004C010020113D0008CE030020094800089F
:10C49000453C0008D53C0008BF01010834000020DD
:10C4A0005DFA0008B53700083A270108312A01086B
:10C4B000F5370008F80F00203D5D00089E000020C1
:10C4C0009DC000082DE9F04F964C89B094F831607A
:10C4D0008046FF2E15469A4640F0EB80084604F150
:10C4E0003002082104F131038F4FB84794F83030FF
:10C4F0004046DFF8C48200938C4908230DF11F02E7
:10C500008B4FB84798F83A30002B3BD0DFF8AC920D
:10C51000C84798F83A30874A0593834690470746BC
:10C52000C847059B7A1EDB439B440121431E002024
:10C53000D2B2009101905FFA8BF102900390DBB2CE
:10C540007D4FB84794F830307C4F57F823007C4B30
:10C5500098478346C8477B4B98F83A201B7898F851
:10C560003A100096CB1A03EBD373C2EB630194F835
:10C5700030304118019657F8232058463346C9B247
:10C58000714EB047694B4FF009081E7888E094F867
:10C59000301038468A1B514241EB02016B4B9847E1
:10C5A000072EDFF8809175D899F83020684B38460F
:10C5B00053F82610931B5A4242EB0302654B9847EF
:10C5C0004EB999F864203D21D2F10102384638BFB6
:10C5D0000022614B9847574B9847604B6FF003021E
:10C5E0001B78D21A8218731ED2B2062B52D8DFE8FB
:10C5F00003F004101E26333F480094F830203846DC
:10C60000A2F1010CDCF10002294642EB0C02544B72
:10C610000BE094F83020B5F91010A2F1020EDEF113
:10C620000002504B384642EB0E02984732E094F835
:10C6300030300122384695F91210032B06E094F8A9
:10C64000303095F9131005223846042B14BF00230F
:10C650000123454FB8471DE094F830203846A2F139
:10C6600005077A4205F1140142EB07023F4BDCE774
:10C6700008230093033B0193FF20514643463C4F60
:10C6800007E0082300933B4F033B0193FF205146F3
:10C690004346B847013608F10808F6B25FFA88F851
:10C6A0009DF81F3008F1FF37B342FFB23FF66FAF7E
:10C6B00086E0072E00F28480DFE806F0040B0F14FA
:10C6C000171C21262C4B01201870FF2384F83130D1
:10C6D00077E02A48FF232A4D1AE02A481032FF2328
:10C6E000294D15E02948123201E029481332FF2371
:10C6F000284D0DE028481432FF23284D08E0284833
:10C70000284A5346284D03E02848294A294D5346D4
:10C71000A847012854D1184B1870FF2384F83130F2
:10C7200001384EE04C010020113D00088B03002031
:10C7300009480008BF0101085DFA000894240108B7
:10C74000952D0008F000002015FF0008453C00086A
:10C7500030240108B53700088D3800083400002067
:10C76000F53700085D380008D9380008B53A0008E8
:10C77000055C00083D5D00089E0000207F34010834
:10C780006D33000822270108ED3200083C2B010818
:10C79000142A01080D2E0008202A01084D720008F5
:10C7A000B126010884290020C9BE0008B526010869
:10C7B000842A0020F1C20008502C0020C301010887
:10C7C000002009B0BDE8F08F2DE9F04F8FB00B923B
:10C7D0006C4A054692F833301646FF2B40F0B58080
:10C7E00008463232412106F13303674CA04796F8E0
:10C7F0003230664C0990009328462146644D0DF175
:10C8000037024123A8472478082598E096F832108B
:10C810002846C4EB010CDCF1000141EB0C015D4B3F
:10C82000DFF860B198474CB99BF832102846D1F137
:10C83000010138BF0021584B98477CE0402C7AD842
:10C840000B9A671E182303FB07239BF83220194617
:10C85000C4EB020EDEF1000242EB0E020A93284600
:10C860004E4B98474E4B98474E4B05F101081A78AE
:10C870006FF003039B1AC3185FFA87FCDBB25FFA01
:10C8800088F84FF008094FF0050A61461A460893E8
:10C89000FF204346444FCDF81CC0CDF80090CDF8A2
:10C8A00004A0B847089ADDF81CC0101AC0B208905E
:10C8B0006146FF20089A43463C4FCDF80090CDF8E2
:10C8C00004A0B847089BDDF81CC0181A9BF832304A
:10C8D000C0B2191B4B4243EB010308900193604621
:10C8E000089942464B46324FCDF800A0B847089A07
:10C8F0002B4B101AC7B298472A4B1A786FF00303D4
:10C900009B1A1B189F4216D10A9B083FB3F91020AF
:10C91000142392FBF3F35BB2FFB2642100930197FF
:10C92000CDF80880CDF80C90CDF810A021480A462B
:10C930000023214FB84708350134EDB2E4B29DF829
:10C940003730A3423FF662AF10E033B91B4B0120F2
:10C950001870FF2382F8333011E00B9C013B182242
:10C9600002FB0342DBB2164CA0470990099A012A48
:10C9700004D1124B1A70FF2386F8333000200FB019
:10C98000BDE8F08F4C010020113D00088F0300200E
:10C9900009480008453C0008D53C0008B5370008A8
:10C9A000BF01010834000020055C00083D5D00085F
:10C9B0009D500008392A0108755400089E00002087
:10C9C000C5C400082DE9F04F694C87B094F8396070
:10C9D0008046FF2E154640F0A080084604F138023C
:10C9E000052104F13903634FB84794F838304046C5
:10C9F000DFF8D4810093604905230DF117025F4FE2
:10CA0000B84798F83A30002B3AD0DFF8C091C847C1
:10CA10005B4B824698F83AB098470746C8476FEA9A
:10CA20000B0BDA447A1E431E01210020D2B2009182
:10CA300001905FFA8AF102900390DBB2514FB84740
:10CA400094F83830504F57F82300504B984782469F
:10CA5000C8474F4B98F83A201B7898F83A10009640
:10CA6000CB1A03EBD373C2EB630194F8383041184F
:10CA7000019657F8232050463346C9B2454EB04779
:10CA80003D4B08271E7843E094F8381038468A1B3F
:10CA9000514241EB0201404B9847042EDFF8D08011
:10CAA00032D898F838203D4B384653F82610931B5F
:10CAB0005A4242EB03023A4B98474EB998F8642029
:10CAC0003D21D2F10102384638BF0022354B1AE031
:10CAD000032E98F83820344B0BD0042E0DD0022EA4
:10CAE00003D038462978012A0AE038466978022AB4
:10CAF00006E03846A978032A02E0E9783846042A95
:10CB000014BF00220122984708370136FFB2F6B25F
:10CB10009DF81730B342B7D825E0042E23D8DFE8BC
:10CB200006F0030A0C0F1400204B01201870FF239D
:10CB300084F8393018E01E4809E01E48013206E04A
:10CB40001D480232FF231D4D03E01D4803321D4DD9
:10CB5000FF23A847012806D1144B1870FF2384F83F
:10CB60003930013800E0002007B0BDE8F08F00BF89
:10CB70004C010020113D0008D103002009480008A5
:10CB8000BF0101085DFA000888380108952D0008EA
:10CB9000F000002015FF0008453C000800250108B2
:10CBA000B53700088D3800085D3800089E00002069
:10CBB000402A01084C2A0108162B01080D2E0008F6
:10CBC000582A010899430008502C0020C30101088D
:10CBD0002DE9FF41384E074696F83B303446FF2B8F
:10CBE0004FD106F13A0206F13B030846334D0321CB
:10CBF000A847334E94F83A303146009305460DF17C
:10CC00000F02384603232F4FB8473678082733E002
:10CC100094F83A1038468B1B594241EB03012A4BDA
:10CC2000DFF8948098474EB998F83A103846D1F119
:10CC3000010138BF0021254B984719E0022E17D873
:10CC400098F83A203846C6EB020CDCF1000242EBC1
:10CC50000C021F491F4B984798F83A20711EC6EBEB
:10CC6000020EDEF10002384642EB0E021A4B9847E4
:10CC700008370136FFB2F6B29DF80F30B342C7D87D
:10CC80000FE033B9154B01201870FF2386F83B30B5
:10CC90000FE0013B242505FB0322114DDBB2A84721
:10CCA0000546012D04D10D4B1D70FF2384F83B3048
:10CCB000002004B0BDE8F0814C010020113D0008C7
:10CCC000D203002009480008453C0008D53C000874
:10CCD000982B0108B53700085D3800089E00002039
:10CCE000C5C900082DE9F04F944C87B094F8356021
:10CCF0008046FF2E154640F0E280084604F13402DB
:10CD00000A2104F135038E4FB84794F83430404679
:10CD1000DFF8AC8200938B490A230DF117028A4F8A
:10CD2000B84798F83A30002B3AD0DFF89892C847C5
:10CD3000864B824698F83AB098470746C8476FEA4C
:10CD40000B0BDA447A1E431E01210020D2B200915F
:10CD500001905FFA8AF102900390DBB27C4FB847F2
:10CD600094F834307B4F57F823007B4B984782462A
:10CD7000C8477A4B98F83A201B7898F83A100096F2
:10CD8000CB1A03EBD373C2EB630194F83430411830
:10CD9000019657F8232050463346C9B2704EB0472B
:10CDA000684B082693F8008083E094F834103046EE
:10CDB000C8EB0103594241EB03016A4B9847B8F1B4
:10CDC000090F5E4F6FD897F83420674BC8EB020C01
:10CDD000DCF1000253F8281042EB0C023046634BA2
:10CDE0009847B8F1000F09D197F864203D21D2F19E
:10CDF0000102304638BF00225D4B53E0A8F1020328
:10CE0000072B05D8DFE803F00A121A272D33394320
:10CE100094F8342030462978012A33E094F83430ED
:10CE20000422304695F90110022B0EE094F83430BC
:10CE30000022304695F90210032B06E094F83430B6
:10CE400095F9031000223046042B14BF0023012360
:10CE5000484FB84727E094F834203046A988052A7F
:10CE600010E094F834203046E988062A0AE094F865
:10CE7000342030462989072A04E094F8342069894F
:10CE80003046082A14BF002201223B4B0AE094F8E6
:10CE900034203A49A2F1090EDEF10002384B304647
:10CEA00042EB0E029847083608F10108F6B25FFA25
:10CEB00088F89DF8173043453FF677AF84E0092E98
:10CEC00000F28280DFE806F0050C1114171C1F2207
:10CED000262C2C4B01201870FF2384F8353074E089
:10CEE0002A462948FF23294D1DE029486A1C04E0F1
:10CEF0002848AA1C01E02848EA1CFF23274D12E01D
:10CF000027482A1D09E02748AA1D06E0264805F102
:10CF1000080202E0254805F10A02FF23244D02E041
:10CF20002448254A254DA84701284DD1154B187096
:10CF3000FF2384F83530013847E000BF4C01002062
:10CF4000113D0008A503002009480008BF010108A1
:10CF50005DFA0008CC220108952D0008F0000020A1
:10CF600015FF0008453C0008C8240108B537000833
:10CF70008D380008D93800085D380008F929010803
:10CF8000F53700089E000020582A01089943000840
:10CF9000612A0108682A01086E2A01080D2E00087E
:10CFA000792A0108742A01084E2601087F2A0108FF
:10CFB00089320008852A0108DC2B0020D1CB00082B
:10CFC000502C0020C3010108002007B0BDE8F08FFD
:10CFD0002DE9FF41384E074696F837303446FF2B8F
:10CFE0004FD106F1360206F137030846334D0321CF
:10CFF000A847334E94F836303146009305460DF17C
:10D000000F02384603232F4FB8473678082733E0FE
:10D0100094F8361038468B1B594241EB03012A4BDA
:10D02000DFF8948098474EB998F836103846D1F119
:10D03000010138BF0021254B984719E0022E17D86F
:10D0400098F836203846C6EB020CDCF1000242EBC1
:10D050000C021F491F4B984798F83620711EC6EBEB
:10D06000020EDEF10002384642EB0E021A4B9847E0
:10D0700008370136FFB2F6B29DF80F30B342C7D879
:10D080000FE033B9154B01201870FF2386F83730B5
:10D090000FE0013B2C2505FB0322114DDBB2A84715
:10D0A0000546012D04D10D4B1D70FF2384F8373048
:10D0B000002004B0BDE8F0814C010020113D0008C3
:10D0C0009B03002009480008453C0008D53C0008A7
:10D0D0008E2A0108B53700085D3800089E00002040
:10D0E000E5CC00082DE9F04F914D87B095F84160EF
:10D0F0008046FF2E144640F0EA80084605F14002C3
:10D100000D2105F141038B4FB84795F8403040465B
:10D11000DFF88C82009388490D230DF11702874FA9
:10D12000B84798F83A30002B3AD0DFF87892C847E1
:10D13000834B824698F83AB098470746C8476FEA4B
:10D140000B0BDA447A1E431E01210020D2B200915B
:10D1500001905FFA8AF102900390DBB2794FB847F1
:10D1600095F84030784F57F82300784B984782461F
:10D17000C847774B98F83A201B7898F83A100096F1
:10D18000CB1A03EBD373C2EB630195F8403041181F
:10D19000019657F8232050463346C9B26D4EB0472A
:10D1A000654B08261F788CE095F840103046C7EB99
:10D1B000010CDCF1000141EB0C01674B98470C2F8F
:10D1C000DFF86C8179D898F84020644BC7EB020EE9
:10D1D000DEF1000253F8271042EB0E023046604B9E
:10D1E00098474FB998F864203D21D2F101023046AA
:10D1F00038BF00225B4B5FE0BB1E0A2B07D8DFE87D
:10D2000003F00C1319252B31373D434A510095F893
:10D2100040203046217D012A4AE095F840203046E2
:10D2200094F91510022A43E095F840203046A17D7C
:10D23000032A3DE095F840203046A2F104035A420B
:10D2400042EB030204F11801474B35E095F840200A
:10D250003046217F052A2BE095F840203046617F3B
:10D26000062A25E095F840203046A17F072A1FE0D6
:10D2700095F840203046218C082A19E095F8402086
:10D280003046618C092A13E095F84020304694F826
:10D2900025100A2A0CE095F84020304694F8261014
:10D2A0000B2A05E095F8402094F8271030460C2A08
:10D2B0002E4B14BF00220122984708360137F6B2E0
:10D2C000FFB29DF81730BB423FF66EAF79E00C2EEF
:10D2D00077D8DFE806F0070E1116191E21247070AA
:10D2E000272A6900224B01201870FF2385F841305E
:10D2F00068E02048143259E01F481532FF231F4CC4
:10D3000056E01F48163251E01E481832FF231E4CCB
:10D310004EE01E481C3249E01D481D3246E01D48C3
:10D320001E3243E01C48253240E01C4826323DE0D6
:10D330004C010020113D0008C103002009480008ED
:10D34000BF0101085DFA0008FC390108952D0008AD
:10D35000F000002015FF0008453C0008E02301080C
:10D36000B53700088D380008B53A00085D38000868
:10D370009E000020AE2A0108B92A01086544000871
:10D38000C52A0108D22A01084D720008DC2A0108CA
:10D39000E92A0108F52A0108012B01080E2B0108D2
:10D3A000502C0020C301010808482732084CFF23F5
:10D3B000A047012805D1074B01221A70FF2385F8E9
:10D3C0004130002007B0BDE8F08F00BF1B2B0108E3
:10D3D000994300089E0000202DE9F04F734B87B061
:10D3E00093F845608046FF2E15461C4640F0C780E6
:10D3F00003F144020846453308216D4FB84794F8BD
:10D4000044304046DFF8E88100936A4908230DF173
:10D410001702694FB84798F83A30002B3AD0DFF836
:10D42000D491C847654B824698F83AB0984707466A
:10D43000C8476FEA0B0BDA447A1E431E0121002015
:10D44000D2B2009101905FFA8AF102900390DBB2B0
:10D450005B4FB84794F844305A4F57F823005A4B63
:10D4600098478246C847594B98F83A201B7898F855
:10D470003A10CB1A03EBD373C2EB630194F8443038
:10D4800041180096019657F8232050463346C9B2FA
:10D490004F4EB047474B08261F786BE094F8441076
:10D4A0003046C7EB010CDCF1000141EB0C01494BAC
:10D4B0009847072FDFF8F48058D898F84420464B57
:10D4C000C7EB020EDEF1000253F8271042EB0E020A
:10D4D0003046424B98474FB998F864203D21D2F12D
:10D4E0000102304638BF00223D4B3EE0BB1E052BFB
:10D4F00004D8DFE803F00E141B22293094F84420EE
:10D500003046A2F101035A4242EB03022968354B2F
:10D510002BE094F84420291D3046022A21E094F89B
:10D520004420304605F11401032A1AE094F84420FF
:10D53000304605F12401042A13E094F844203046D3
:10D5400005F13401052A0CE094F84420304605F139
:10D550004401062A05E094F84420304605F5A271FE
:10D56000072A214B14BF00220122984708360137B1
:10D57000F6B2FFB29DF81730BB428FD80AE016B161
:10D58000072E07D80AE0194A01201070FF2283F8FD
:10D59000452000E0002007B0BDE8F08F134A0121CC
:10D5A0001170FF2283F84520F4E700BF4C010020F2
:10D5B000113D00089903002009480008BF01010837
:10D5C0005DFA000890250108952D0008F000002064
:10D5D00015FF0008453C0008B0250108B5370008D4
:10D5E0008D3800085D380008F53700089E000020DF
:10D5F000502C0020C30101082DE9F0475A4F064680
:10D6000097F84D4086B0FF2C08463D4640F08F808D
:10D6100007F14C0207F14D030221544FB84795F82A
:10D620004C3030460093524E022352490DF11702FE
:10D63000B047514E96F83A30002B3AD0DFF87C8153
:10D64000C0474E4B814696F83AA098470746C047D8
:10D650006FEA0A0AD1447A1E431E01210020D2B289
:10D66000009101905FFA89F102900390DBB2444F80
:10D67000B84795F84C30434F57F82300424B984732
:10D680008146C047414B96F83A201B7896F83A10ED
:10D69000CB1A03EBD373C2EB630195F84C304118FE
:10D6A0000094019457F8232048462346C9B2384CC9
:10D6B000A047304B08261C7834E095F84C103046D3
:10D6C0000B1B594241EB0301324B9847012C264F6B
:10D6D00024D897F84C20304BC4EB020CDCF100024C
:10D6E00053F8241042EB0C0230462C4B98474CB9AF
:10D6F00097F864203D21D2F10102304638BF002264
:10D70000274B0AE097F84C202649A2F1010EDEF1E2
:10D710000002254B304642EB0E0298470836013492
:10D72000F6B2E4B29DF81730A342C6D817E014B1A0
:10D73000012C14D106E01D4B01201870FF2387F83F
:10D740004D300DE01A481B4A1B4B9847012806D163
:10D75000164B1870FF2387F84D30013800E0002089
:10D7600006B0BDE8F08700BF4C010020113D000865
:10D7700009480008D7030020502C0020BF010108F1
:10D780005DFA000814250108952D0008F00000201E
:10D7900015FF0008453C00084C250108B537000876
:10D7A0008D380008F9290108F53700089E0000208F
:10D7B0002A2B01084C2C002095960008C301010873
:10D7C0002DE9F04F9A4C87B094F851608046FF2EB7
:10D7D000154640F00681084604F15002092104F183
:10D7E0005103944FB84794F850304046DFF8AC826C
:10D7F0000093914909230DF11702904FB84798F80B
:10D800003A30002B3AD0DFF89892C8478C4B8246CA
:10D8100098F83AB098470746C8476FEA0B0BDA44C6
:10D820007A1E431E01210020D2B2009101905FFABE
:10D830008AF102900390DBB2824FB84794F85030DF
:10D84000814F57F82300814B98478246C847804B49
:10D8500098F83A201B7898F83A100096CB1A03EB08
:10D86000D373C2EB630194F850304118019657F816
:10D87000232050463346C9B2764EB0476E4B082639
:10D880001F78A8E094F850103046C7EB010CDCF18B
:10D89000000141EB0C01704B9847082FDFF8908195
:10D8A00000F2958098F850206C4BC7EB020EDEF129
:10D8B000000253F8271042EB0E023046684B98479F
:10D8C0004FB998F864203D21D2F10102304638BFAB
:10D8D0000022644B7AE0BB1E062B05D8DFE803F07C
:10D8E000181F333A4E556C0095F800E05E4BBEF1C0
:10D8F0003F0F04D994F8502030465C4906E05C495B
:10D900004FEA4E1E94F8502030467144012A4FE0F1
:10D9100094F85020304695F90110022A52E095F80B
:10D9200002E0514BBEF13F0F04D994F8502030462D
:10D930004E4906E04E494FEA4E1E94F850203046BC
:10D940007144032A34E094F85020304695F90310CE
:10D95000042A37E095F804E0434BBEF13F0F04D9A9
:10D9600094F850203046414906E041494FEA4E1EA6
:10D9700094F8502030467144052A19E094F850205C
:10D98000304695F90510062A1CE095F806E0364B5E
:10D99000BEF13F0F04D994F850203046334906E0D9
:10D9A00033494FEA4E1E94F8502030467144072AFE
:10D9B00014BF0022012209E094F8502095F90710C5
:10D9C0003046082A2B4B14BF002201229847083604
:10D9D0000137F6B2FFB29DF81730BB423FF652AFA7
:10D9E0006EE0082E6CD8DFE806F0050C0E11141757
:10D9F0001A1D5D00204B01201870FF2384F8513060
:10DA00005FE01E4810E01E4801324DE01D48023222
:10DA10000AE01D48033247E01C48043204E01C4879
:10DA2000053241E01B480632FF231B4D3EE000BF9C
:10DA30004C010020113D0008D003002009480008D7
:10DA4000BF0101085DFA0008BC230108952D0008FC
:10DA5000F000002015FF0008453C0008643801086C
:10DA6000B53700088D380008F53700083A27010857
:10DA7000FC0700205D3800089E0000202E2B0108C6
:10DA8000352B0108442B01084B2B01085A2B0108A8
:10DA9000612B0108702B010899430008502C0020CD
:10DAA000C301010808480732084DFF23A847012891
:10DAB00006D1074B1870FF2384F85130013800E07D
:10DAC000002007B0BDE8F08F772B010865440008FF
:10DAD0009E0000202DE9F04F804D87B095F85560ED
:10DAE0008046FF2E144640F09980084605F1540206
:10DAF0000C2105F155037A4FB84795F8543040464C
:10DB0000DFF87082009377490C230DF11702764FEE
:10DB1000B84798F83A30002B3AD0DFF85C92C84703
:10DB2000724B824698F83AB098470746C8476FEA62
:10DB30000B0BDA447A1E431E01210020D2B2009161
:10DB400001905FFA8AF102900390DBB2684FB84708
:10DB500095F85430674F57F82300674B9847824633
:10DB6000C847664B98F83A201B7898F83A10009608
:10DB7000CB1A03EBD373C2EB630195F85430411811
:10DB8000019657F8232050463346C9B25C4EB04741
:10DB9000544B08271E783CE095F8541038468A1BF1
:10DBA000514241EB0201574B98470B2EDFF82C8175
:10DBB0002BD898F85420544B384653F82610931B12
:10DBC0005A4242EB0302514B98474EB998F86420F1
:10DBD0003D21D2F10102384638BF00224C4B13E000
:10DBE000022E08D001D30B2E0FD995F854203846B9
:10DBF0002168012A04E098F8542021793846022A45
:10DC0000444B14BF00220122984708370136FFB267
:10DC1000F6B29DF81730B342BED85BE00B2E59D850
:10DC2000DFE806F0060D11161B21272D343B424874
:10DC3000394B01201870FF2385F855304BE03748E9
:10DC4000FF23374C3CE037480432FF23364C37E0A3
:10DC500036484832FF23364C32E0364802F58472AB
:10DC6000FF23354C2CE0354802F5E472FF23344C99
:10DC700026E0344802F54272FF23334C20E002F5DF
:10DC8000805232480832FF23314C19E002F58852A5
:10DC900030480832FF23304C12E002F590522F48F2
:10DCA0000832FF232E4C0BE02E4802F59352FF233F
:10DCB0002D4C05E002F594522C482D4C2832FF23C0
:10DCC000A047012806D1144B1870FF2385F8553062
:10DCD000013800E0002007B0BDE8F08F4C010020C3
:10DCE000113D0008C703002009480008BF010108D2
:10DCF0005DFA00081C250108952D0008F0000020A1
:10DD000015FF0008453C000820230108B53700082E
:10DD10008D3800085D3800089E000020862B010821
:10DD2000213200088C2B0108994300089C26010829
:10DD3000F5AA0008A1260108FDAE0008AA260108E0
:10DD4000CDA60008F726010881B40008B126010815
:10DD5000C9BE0008B5260108F1C20008962B0108CB
:10DD6000D1CF0008852A0108D1CB0008A12B0108DA
:10DD7000C1D70008502C0020C30101082DE9F04F45
:10DD80006D4C87B094F861608046FF2E154640F0D8
:10DD9000A980084604F16002052104F16103674F80
:10DDA000B84794F860304046DFF8E8810093644952
:10DDB00005230DF11702634FB84798F83A30002B4E
:10DDC0003AD0DFF8D491C8475F4B824698F83AB012
:10DDD00098470746C8476FEA0B0BDA447A1E431E82
:10DDE00001210020D2B2009101905FFA8AF10290E5
:10DDF0000390DBB2554FB84794F86030544F57F852
:10DE00002300544B98478246C847534B98F83A2012
:10DE10001B7898F83A100096CB1A03EBD373C2EB39
:10DE2000630194F860304118019657F8232050465A
:10DE30003346C9B2494EB047414B08271E784CE0E3
:10DE400094F860103846C6EB010CDCF1000141EBA0
:10DE50000C01434B9847042EDFF8DC8039D898F842
:10DE60006020404BC6EB020EDEF1000253F8261094
:10DE700042EB0E0238463C4B98474EB998F8642066
:10DE80003D21D2F10102384638BF0022374B1FE056
:10DE9000032E98F860200BD0042E11D0022E03D050
:10DEA00038462968012A06E0291D3846022A0BE077
:10DEB000A9683846032A14BF002201222C4B07E030
:10DEC000384605F10C01042A2A4B14BF0022012216
:10DED000984708370136FFB2F6B29DF81730B342C3
:10DEE000AED825E0042E23D8DFE806F0030A0C0F95
:10DEF0001400214B01201870FF2384F8613018E0D2
:10DF00001E4804E01E48043206E01E480832FF2383
:10DF10001D4D03E01D480C321D4DFF23A84701286D
:10DF200006D1154B1870FF2384F86130013800E0EA
:10DF3000002007B0BDE8F08F4C010020113D000823
:10DF4000C503002009480008BF0101085DFA000868
:10DF5000A4390108952D0008F000002015FF0008E5
:10DF6000453C0008C0390108B53700088D38000865
:10DF70005D380008513B00089E000020E62B010898
:10DF8000ED2B0108F92B010821320008002C0108B3
:10DF900051750008502C0020C30101082DE9F04FF5
:10DFA000794C87B094F865608046FF2E154640F0A6
:10DFB000A380084604F16402082104F16503734F4D
:10DFC000B84794F864304046DFF8348200937049D3
:10DFD00008230DF117026F4FB84798F83A30002B1D
:10DFE0003AD0DFF82092C8476B4B824698F83AB097
:10DFF00098470746C8476FEA0B0BDA447A1E431E60
:10E0000001210020D2B2009101905FFA8AF10290C2
:10E010000390DBB2614FB84794F86430604F57F813
:10E020002300604B98478246C8475F4B98F83A20D8
:10E030001B7898F83A100096CB1A03EBD373C2EB17
:10E04000630194F864304118019657F82320504634
:10E050003346C9B2554EB0474D4B08271E7846E0AF
:10E0600094F8641038468B1B594241EB0301504B26
:10E070009847072EDFF8108135D898F864204D4B6B
:10E08000C6EB020CDCF1000253F8261042EB0C0246
:10E090003846494B984746B998F864203D21D2F15B
:10E0A0000102384638BF00221BE0022E0FD001D3F8
:10E0B000072E18D994F864203846A2F1010EDEF13B
:10E0C000000205F1180142EB0E023C4B0AE098F801
:10E0D000642095F92810A2F102035A42384642EB17
:10E0E0000302374B984708370136FFB2F6B29DF866
:10E0F0001730B342B4D842E0072E40D8DFE806F02C
:10E10000040B10151A21282F2E4B01201870FF2305
:10E1100084F8653034E02C481832FF232B4D24E07E
:10E120002B482832FF232B4D1FE02B482C32FF2396
:10E130002A4D1AE002F5026229480C32FF23294DCC
:10E1400013E002F5626228480C32FF23274D0CE0F1
:10E1500002F58C5226482C32FF23264D05E002F5AD
:10E1600010522548254D5C32FF23A847012806D1CF
:10E17000144B1870FF2384F86530013800E000204C
:10E1800007B0BDE8F08F00BF4C010020113D000832
:10E19000AE03002009480008BF0101085DFA00082D
:10E1A00054250108952D0008F000002015FF0008F7
:10E1B000453C000884390108B5370008F5370008E8
:10E1C0008D3800089E0000207F3401086D33000860
:10E1D000AB2F0108B53E0008272A010831BA000814
:10E1E000392A0108C9C700085B30010821A30008CB
:10E1F0000C2C0108D5DA00087A3101087DDD000811
:10E20000502C0020C30101082DE9F0475C4B86B07B
:10E2100093F869400646FF2C1D4640F09B8003F1B1
:10E220006802084669330421564FB84795F86830AC
:10E2300030460093544E042354490DF11702B04761
:10E24000534E96F83A30002B3AD0DFF87C81C04725
:10E25000504B814696F83AA098470746C0476FEA68
:10E260000A0AD1447A1E431E01210020D2B2009135
:10E2700001905FFA89F102900390DBB2464FB847F4
:10E2800095F86830454F57F82300454B984781462D
:10E29000C047444B96F83A201B7896F83A10CB1AB0
:10E2A00003EBD373C2EB630195F868304118009417
:10E2B000019457F8232048462346C9B23A4CA04758
:10E2C000324B08261C7840E095F868103046C4EBC5
:10E2D000010CDCF1000141EB0C01344B9847032C9D
:10E2E000274F2ED897F86820314BC4EB020EDEF191
:10E2F000000253F8241042EB0E0230462D4B984793
:10E300004CB997F864203D21D2F10102304638BF64
:10E310000022294B14E0022C97F86820274B05D0E7
:10E32000032C07D030462649012A06E0304624490E
:10E33000022A02E022493046032A14BF00220122A9
:10E34000984708360134F6B2E4B29DF81730A3427C
:10E35000BAD80AE014B1032C07D80AE0194A012000
:10E360001070FF2283F8692000E0002006B0BDE8AD
:10E37000F087144A01211170FF2283F86920F4E725
:10E380004C010020113D0008094800089C030020B2
:10E39000502C0020BF0101085DFA0008F825010893
:10E3A000952D0008F000002015FF0008453C0008EE
:10E3B000AC380108B53700088D380008F53700087B
:10E3C000F92901089E000020C30101082DE9F0474A
:10E3D0007E4C86B094F86D500646FF2D40F0BA8012
:10E3E000084604F16C020B2104F16D03784FB84725
:10E3F00094F86C3030460093764E0B2376490DF13D
:10E400001702B047754E96F83A30002B3AD0DFF835
:10E410003082C047724B814696F83AA0984707462B
:10E42000C0476FEA0A0AD1447A1E431E0121002028
:10E43000D2B2009101905FFA89F102900390DBB2B1
:10E44000684FB84794F86C30674F57F82300674B14
:10E4500098478146C047664B96F83A201B7896F855
:10E460003A100095CB1A03EBD373C2EB630194F817
:10E470006C304118019557F8232048462B46C9B205
:10E480005C4DA847544B08251E785EE094F86C104C
:10E4900028468A1B514241EB0201574B98470A2EEE
:10E4A0004A4F4ED897F86C20544B284653F8261004
:10E4B000931B5A4242EB0302514B98474EB997F8CF
:10E4C00064203D21D2F10102284638BF00224D4B85
:10E4D00036E0B31E082B06D8DFE803F00B11171D3A
:10E4E00033333323290094F86C2028464649012A07
:10E4F00022E094F86C2028464349022A1CE094F854
:10E500006C2028464049032A16E094F86C202846DF
:10E510003D49042A10E094F86C2028463A49052A1F
:10E520000AE094F86C2028463749092A04E094F858
:10E530006C20354928460A2A344B14BF0022012298
:10E54000984708350136EDB2F6B29DF81730B34260
:10E550009CD836E00A2D34D8DFE805F0060D1013FC
:10E5600016191D21262D2D00294B01201870FF237F
:10E5700084F86D3026E00846264B0AE00846264B14
:10E5800007E00846254B04E00846254B01E0254BF3
:10E59000084698470DE02448FF23244D08E024480E
:10E5A0002032FF23234D03E02348244D4832FF232C
:10E5B000A847012805D1164B01221A70FF2384F8C1
:10E5C0006D30002006B0BDE8F08700BF4C01002090
:10E5D000113D000809480008A3030020502C00202A
:10E5E000BF0101085DFA0008BC380108952D00083C
:10E5F000F000002015FF0008453C0008F422010847
:10E60000B53700088D380008F9290108F5370008EA
:10E610009E00002085780008D57B000841990008FD
:10E62000159D0008E59E0008F1310108F9D50008A4
:10E63000132C0108E5D000081B2C0108D9D30008D1
:10E64000C30101082DE9F047604C86B094F8715081
:10E650000646FF2D40F08680084604F17002052131
:10E6600004F171035A4FB84794F870303046009364
:10E67000584E052358490DF11702B047574E96F8EA
:10E680003A30002B3AD0DFF8A481C047544B814682
:10E6900096F83AA098470746C0476FEA0A0AD1445D
:10E6A0007A1E431E01210020D2B2009101905FFA30
:10E6B00089F102900390DBB24A4FB84794F870306A
:10E6C000494F57F82300494B98478146C047484B6C
:10E6D00096F83A201B7896F83A100095CB1A03EB7F
:10E6E000D373C2EB630194F870304118019557F869
:10E6F000232048462B46C9B23E4DA847364B082634
:10E700001D782AE094F870103046C5EB010CDCF15E
:10E71000000141EB0C01384B9847042D2B4F18D8C2
:10E7200097F87020354BC5EB020EDEF1000253F86E
:10E73000251042EB0E023046314B98474DB997F801
:10E7400064203D21D2F10102304638BF00222D4B1A
:10E75000984708360135F6B2EDB29DF81730AB4256
:10E76000D0D82FE0042D2DD8DFE805F0030A0E15D0
:10E770001C00254B01201870FF2384F8713022E023
:10E780002248FF23224D13E002F51052214878322F
:10E79000FF23214D0CE002F5105220487832FF2370
:10E7A0001F4D05E002F510521E481F4D7C32FF231D
:10E7B000A847012806D1144B1870FF2384F8713044
:10E7C000013800E0002006B0BDE8F0874C010020D1
:10E7D000113D00080948000895030020502C002036
:10E7E000BF0101085DFA0008D4390108952D000821
:10E7F000F000002015FF0008453C0008B424010883
:10E80000B53700088D3800089E000020E82D01086B
:10E810009DDF0008232C010809E200082E2C0108C6
:10E82000D5930008352C0108CDE30008C301010889
:10E830002DE9F04FA64C93B025780146FF2D40F00E
:10E840008487A44E23460F213246A34CA047377835
:10E85000A24B012FA24CA34EDFF8C49240F0C0831C
:10E86000A1489847A0478046B0474FF0000ADFF81C
:10E87000B4B208F1FF32431E009750460821D2B2CD
:10E88000DBB2CDF804A0CDF808A0CDF80CA0C847A5
:10E89000BBF838103B465246DFF88C82009709B22D
:10E8A0000DA8C047DFF884C290490DA8E047904901
:10E8B0000DA88847BBF854100BF1400C0DAACDF8F9
:10E8C00010C03B4609B2009710185246C047894F06
:10E8D0000DA8B847DFF858822B460A210DAA0095EB
:10E8E0000195C047A04740085FFA80F9B0478046CD
:10E8F000B047083800EBD070A8F10808401008EBCA
:10E90000D8780C384FEA680880B208F108085FFA36
:10E9100080FE5FFA88F80790009501952B46CDF8A8
:10E9200020E0484641467246734DA8475046734B17
:10E930009847FF250AF10F0A0346009001950295BA
:10E94000039548464146089A6D4F1FFA8AFAB84720
:10E95000BAF5B47FEAD1DDF820C04FF0000BACF17E
:10E96000050248464146674FD2B25B46CDF800B03B
:10E97000CDF804B0B847DDF820E0DFF8B8A1AEF17B
:10E98000040C5FFA8CFC484641466246CDF828C02C
:10E990005B46CDF800B0CDF804B0B8470AF5865113
:10E9A000088F0B8F584F0993089B00B29A1E5FFA8D
:10E9B00082FCCDF810C0B847544A55499047554F8E
:10E9C0005549B847DDF824E0034605930FFA8EF069
:10E9D0004D4988474D4A4E4990474F49B847DDF861
:10E9E00010C0414662460090DFF814C148460195C8
:10E9F00002950395059BE0470AF58851888A8B8A22
:10EA000000B21A460692404B9847DFF800C14049D1
:10EA1000E0474149B8474FF07E51404B9847069A2E
:10EA20000346059310B238498847384A3849904719
:10EA30003949B8474FF07E51B8474146009001959B
:10EA40004846029503950A9A059B2D4FB847DDF875
:10EA500020C04846ACF10707FFB241463A46DFF80E
:10EA6000A4C05B46CDF800B0CDF804B0E0474846FE
:10EA700041463A462B46009501951F4FB847DDF8B1
:10EA80001CE0BAF8381F4FEA5E0CBAF8383F5FFA5C
:10EA90008CFCCCEB0900079ACDF820C009B2DDF858
:10EAA0001CC01BB2A1F50071A3F50073514303FB19
:10EAB0000CF30327BEFBF7FE5FFA8EF791FBF5F12F
:10EAC00093FBF5F3C7EB09024144434434E000BF34
:10EAD0004C0000208A030020113D0008A13E0008E0
:10EAE000BF010108C30101085B3001083C2C01088B
:10EAF0009D120008C12D0008A90001084D0C000856
:10EB0000BD01010891FF0008550C0008650E0008C2
:10EB100000002041ED0A00080000B442E90A0008A4
:10EB20005DFA000890180020F523000899110008EC
:10EB3000CDFE0008D0070020009501950295C0B2D7
:10EB4000C9B2D2B2DBB2DFF8B4C2E047BAF8383F9C
:10EB5000BAF8382F19B2079BA1F500715943DDF8B7
:10EB60001CC013B2A3F5007303FB0CF3DDF820E027
:10EB700091FBF5F193FBF5F30EEB0900414407EB34
:10EB8000090E43445FFA8EF2009501950295C0B2DA
:10EB9000C9B2DBB2DFF864C2E047BAF8382FDDF85B
:10EBA0001CE00FFA82FCACF5007C0CFB0EFCBAF802
:10EBB0001C3F9CFBF5FCBAF81C0F053FC4445FFAF0
:10EBC0008CFC1BB2FFB2CDF810C0089709907E49AB
:10EBD000A3F5007088477D4A90477D4F00224FF093
:10EBE0007E53B84774A3D3E90023B847794B9847BD
:10EBF000DDF824E00A900FFA8EF07349A0F500705A
:10EC00008847724A904700224FF07E53B8476AA364
:10EC1000D3E90023B8476F4B9847DDF810C0009048
:10EC200061464846DFF8B0C1019502950395089A00
:10EC30000A9BE047BAF8382FDDF81CE012B2A2F5C3
:10EC4000007202FB0EF2BAF81C0F92FBF5F2BAF852
:10EC50001C3F4244D2B200B2099307925A49A0F530
:10EC600000708847594A904700224FF07E53B847BA
:10EC700051A3D3E90023B84751A3D3E90023DFF818
:10EC80008081C047534B9847DDF824E084460FFA53
:10EC90008EF0CDF810C04C49A0F5007088474B4A63
:10ECA000904700224FF07E53B84743A3D3E9002397
:10ECB000B84743A3D3E90023C047464B9847DDF844
:10ECC00010C0009063464846019502950395079948
:10ECD000089A414DA847B047BAF8007F0C3880B277
:10ECE000BFB207905546DFF814913C4B97B90DA879
:10ECF0003B4998473B4B3A4619880A2389B2B1FBF6
:10ED0000F3F1093B00930DF1370009B20133364F9F
:10ED1000B84714E035490DA89847B5F8001F4FF4DF
:10ED20007A7309B2890291FBF3F1012300930DF18B
:10ED3000370009B25A46DB18DFF8AC80C047DFF86D
:10ED4000C4C02B490DA8E0472A490DA888470746AB
:10ED5000B047FF23A0F10801274E384600930193E6
:10ED6000C9B20DAAB047079F00264FEA5708A8F17D
:10ED700002080A271AE07301EB1893F83E2039467F
:10ED800052B2002AB8BF0F321211FF230A32009389
:10ED9000019302930A203B46D2B201360237C8479C
:10EDA000402EFFB202D10A27002650E04645E2DBA2
:10EDB000F9E700BFAFF3008000000000008046408C
:10EDC0000000000000806640550C0008D5030008D4
:10EDD0007D040008410A0008BD010108E111000896
:10EDE0003E2C010850040020F5230008422C0108A5
:10EDF00020320108C12D0008CDFE000861FD000889
:10EE00001901000899110008A0478246A04718235D
:10EE100003FB065303F5026318339B88AAF10A0A21
:10EE20001BB2002BB8BFFF331B120A3BC2185FFA9C
:10EE30008AFAFF2300930193029339463B465046DA
:10EE4000D2B201360237C847402EFFB201D0464544
:10EE5000DADBB5F8742EDDF81C800326B8FBF6F675
:10EE6000642112B2B31D4A4348BF1F32DFF8BC828F
:10EE7000521119274FF0320AD2B2DFF8B492089338
:10EE80000092CDF804A00297CDF80C8014200A213E
:10EE90003A461BB2C84706F10A030993F31C5B000C
:10EEA0000A93B5F8583E4FF0640B1BB20BFB03F30B
:10EEB000FF22DDF824C0DDF828E093FBF2F3DBB29B
:10EEC0000FFA8CF10093CDF804A00FFA8EF302979D
:10EED000CDF80C8014203A46C8470536B5F8902E78
:10EEE0000798760031B20B9612B25E46831D5643E8
:10EEF000B34648BF06F11F0B4FEA6B1B5FFA8BF25C
:10EF000000926FF0180201929218079302921BB2BE
:10EF10004B32CDF80C801420C847A04747468046A6
:10EF2000A047B5F8AC6EA0F1140236B26420464397
:10EF300048BF1F36A8F119017611DDF82080F6B21E
:10EF40000FFA88F300964FF01908322609B212B270
:10EF500001960846CDF808800A210397C847A047C4
:10EF60008246A047B5F8E41EAAF1190309B24FF092
:10EF7000640A0AFB01F1A0F11402FF20DDF824C0AD
:10EF8000DDF828E091FBF0F1C9B212B200910196D0
:10EF90000FFA8CF118B2CDF808800FFA8EF30397B0
:10EFA000C847A0470646A047B5F8C84E0B9A24B2FA
:10EFB00011B2A0F114025046193E444348BF1F3419
:10EFC000079D64116FF0180036B2E4B2019000188A
:10EFD000029012B22BB2009403973046C847BDE3AB
:10EFE00048489847A0470746B0474FF000087A1EA8
:10EFF000431E4FF0010A08214046D2B2DBB2CDF8E1
:10F000000480CDF80880CDF80C80CDF800A0C8476A
:10F01000A047DFF820918008143899F828300C2197
:10F020000222CDF80480384FCDF800A0C0B2B84716
:10F03000A047364F834609F11800B8474FEA9B0BAB
:10F04000ABF1050BABEB50001E2109F118022B466A
:10F05000DFF8CCC000950195C0B2E0472C492D4B9C
:10F060000DA89847DFF8D0C00A23BCF8001042462C
:10F0700089B2B1FBF3F1CDF810C0083B09B2CDF86D
:10F0800000A00EA8DFF8B480C0472349234A0DA88A
:10F090009047B047A0F112012B4600950195022040
:10F0A000C9B20DAA1E4DA8471E4BBB461B7809F5D9
:10F0B0001257022BDDF810C055D1BCF8002041F2E8
:10F0C000180392B29A423BD97A6C4FF47A73B2FB2E
:10F0D000F3F103FB1123B3F5FA7F44D9B047B0F144
:10F0E0000C0148BFA0F1090189100931FF23490033
:10F0F00000930193042001F0FE010B4ADFF8208009
:10F10000C04730E0462C0108E5FA00089DFE0008E3
:10F110004F2C0108E1110008203201089911000864
:10F12000CDFE0008EE010020542C010877470108AD
:10F1300031960008D007002050040020F523000875
:10F14000B047B0F10C0148BFA0F1090189100931A5
:10F15000FF23490000930193042001F0FE016D4A52
:10F16000DFF8C8C1E0476C4D4FF47A78E96D4FF095
:10F170000109B1FBF8F10422002309B2DFF8B0C1A4
:10F18000CDF800900DA8E047A04782460DA8D847CB
:10F19000AAF1020AFF23C0EB0A00DFF890C10B219D
:10F1A000009301930DAAC0B2E0476B6E0422B3FB3B
:10F1B000F8F80FFA88F10023CDF80090DFF870819D
:10F1C0000DA8C047A04781460DA8D8478046B04744
:10F1D0000346B3F10C0148BFA3F10901A9F10209EB
:10F1E0008910FF25C8EB09080B312B46DFF83CC11D
:10F1F0005FFA88F000950195C9B20DAAE047796CD5
:10F200004EF660234FF0010AB1FBF3F10222002316
:10F2100009B2DFF81C81CDF800A00DA8C047DFF8C7
:10F2200004C13E490DA8E0473D490DA888477A6CC6
:10F230004FF47A78B2FBF8F23C23B2FBF3F103FB14
:10F2400011210DAADFF8E8C03C3B101809B20222D8
:10F25000CDF800A0E0473149324A0DA89047304B25
:10F260000DA898477B6C0A21B3FBF8F208FB123813
:10F270000DAFB8FBF1F10222002309B23818DFF814
:10F28000B080CDF800A0C047A04780460DA8D84761
:10F290000746B047A8F10208C7EB0807A0F1120122
:10F2A0002B460DAAC9B2DFF884C000950195F8B2CB
:10F2B000E047A04720FA0AF8B047DFF86C905FFA01
:10F2C00088F809F5105393F854200F38A8F10E0868
:10F2D0003F2A1FFA88F885B200F2B68093F85420CE
:10F2E000023252014A449279524523D193F8542074
:10F2F0005201914499F83E1093F8552049B20FFA03
:10F3000088F303EBD37B4B4352B293FBF2F3C3EB93
:10F310006B0B24E0592C0108D02B00200E2601088D
:10F320009D12000899110008D0070020CDFE0008AA
:10F33000F523000893F854205201914499F83EB007
:10F3400093F855204FFA8BFB0FFA88F30BFB03FB66
:10F3500052B29BFBF2FB03EBD3730BEB630B0FFA85
:10F3600088F30FFA8BFB9B45D4BF2BEAEB7BC3469C
:10F37000A0475FFA88FCCDF810C06FF0030ACCEB11
:10F380000A0A0746B0470690A0478146B04706994B
:10F390005FFA8AFA5744A9F10402031F4FF0FF09EC
:10F3A00000200A39C9B2D2B2DBB20090CDF8049085
:10F3B000F8B2CDF808907A4FCDF80C90B847A04736
:10F3C0000590B0470690A0470746B047059B0699B1
:10F3D00053445FFA8BFBBA440BEB030E0B39D34457
:10F3E000C31E5FFA8BF2C9B2DBB25FFA8EF0CDF8C2
:10F3F0000090CDF80490CDF808906A4FB847A04728
:10F400000FFA88FADDF810C00AEBDA7A0590CCEB37
:10F410006A0AB0470690A0478346B047AAF1040A9B
:10F42000059B06995FFA8AFA03EB0A020839831FE3
:10F43000DA44802001900290CDF80090D0B2C9B299
:10F440005FFA8AF2DBB2B847574A02F5105393F8D5
:10F4500056103F2900F2818093F85610023149017D
:10F4600051188979012912D193F85610490152187F
:10F4700092F83E1093F8572049B22BB203EBD37A9F
:10F480004B4352B293FBF2F3C3EB6A0A13E093F8D7
:10F4900056104901521892F83EA093F857204FFA9F
:10F4A0008AFA2BB20AFB03FA52B29AFBF2FA03EB86
:10F4B000D3730AEB630A0FFA8AFA2BB29A45DABFC2
:10F4C0002AEAEA7A1FFA8AFAAA46A0470746A0471C
:10F4D0007F0842084FF0FF0902370021083205F18A
:10F4E0000B03D2B2DBB2F8B200912D4F0B31CDF845
:10F4F0000490CDF80890CDF80C90B847A047074687
:10F50000A0470AF10B0A42087F085FFA8AF1013727
:10F5100009320B46D2B2F8B2CDF80090CDF8049083
:10F52000CDF808901F4FB847A0478246A0472BB29E
:10F5300003EBD373591042080B314FEA5A0A802368
:10F54000C9B20AF1040A063201930293CDF8009081
:10F550005FFA8AF0D2B20B46B847134A02F510534D
:10F5600093F858103F2900F2878093F85810023121
:10F57000490151188979012918D193F85810490186
:10F58000521892F83E1093F8592049B22BB203EB6F
:10F59000D37A4B4352B293FBF2F3C3EB6A0A19E0FE
:10F5A0000DFC000861FD0008D007002093F85810FA
:10F5B0004901521892F83EA093F859204FFA8AFA5E
:10F5C0002BB20AFB03FA52B29AFBF2FA03EBD373A3
:10F5D0000AEB630A0FFA8AFA2BB29A45D6BF2AEAD7
:10F5E000EA7AAA461FFA8AFAA0470746A0477F0888
:10F5F00042084FF0FF09093F05F10B030021033AD0
:10F60000D2B2DBB2F8B20091564F0B31CDF8049074
:10F61000CDF80890CDF80C90B847A0470746A04712
:10F620000AF10B0A42087F085FFA8AF10A3F023AA0
:10F630000B46D2B2F8B2CDF80090CDF80490CDF8D8
:10F640000890494FB847A0478246A0472DB205EB26
:10F65000D575691042080B314FEA5A0A8023C9B2A6
:10F66000AAF1070A053A01930293CDF800905FFAD8
:10F670008AF0D2B20B46B8473C4A02F5105393F8D1
:10F680005A103F295DD893F85A10364D023149017E
:10F690005118897993F85A104901521892F83E701E
:10F6A00093F85B207FB20FFA88F35F4352B297FB67
:10F6B000F2F703EBD37307EB63073FB20FFA88F35C
:10F6C0009F42D6BF27EAE7774746BFB2B047044616
:10F6D000B047A4F10A0108F10302FF24031F002030
:10F6E000C9B2D2B2DBB20090019403300294039409
:10F6F000A847B0470546B0470337FFB2A5F10B0155
:10F70000C31E3A46C9B2DBB2384600940194029453
:10F71000154DA847B0478146B0470FFA88F808EB67
:10F72000D8784FEA680703378022FFB2831FA9F118
:10F7300008010192029200943846C9B23A46DBB2FF
:10F74000A8470B480023037008E000230948074A34
:10F75000094DA847012801D1FF232370002013B0D1
:10F76000BDE8F08F0DFC000861FD0008D007002007
:10F770008A030020622C010845E60008AFF30080F0
:10F780005F2810B532D8192930D8CB08602404FB83
:10F790000300683C04FB0311022AC9B20AD0032A01
:10F7A00011D0012A22D112FA01F1114B1A5C42EA5E
:10F7B000010106E0012212FA01F10D4B1A5C22EA66
:10F7C0000101195410BD0A4B1A5C52FA01F414F0ED
:10F7D000010F4FF0010405D014FA01F122EA0102F1
:10F7E0001A5410BD14FA01F10A431A5410BD00BF97
:10F7F000F80400202DE9F04F572885B0824600918B
:10F80000934603939DF838503EDC13019B1A002465
:10F8100001930646A14621E0224B019A9B181B5DED
:10F820003B4113F0010F07D030464146039A1E4B6F
:10F830009847DDF8089005E025B1304641462A4654
:10F84000194B9847013708F10108082F5FFA88F82B
:10F85000E2D1013401360F2CF6B205D0E3B20293A7
:10F86000DDF800800027D7E785B10024009A0AF16F
:10F870000F00A1180134C0B2C9B22A460A4BE4B243
:10F880009847082CF2D101E04FF00009BBF1560F68
:10F8900086BF09F101095FFA89F00F2005B0BDE8C4
:10F8A000F08F00BFE23F010881F700082DE9F04F1B
:10F8B00085B0009040480191039301783F4B1F2A87
:10F8C0005C5C9DF838A0C4F10804E4B2029483465D
:10F8D00004D97E2A34BF15467E2500E02025384B0A
:10F8E0005A5C009952185F2A54DC203DEDB24FF06B
:10F8F00000090E464C46A8462BE03149CA5C314906
:10F9000051F82330029902FB0832125D7B1852FA3B
:10F9100003F313F0010F06D030462946039A2A4B11
:10F920009847A14607E0BAF1000F04D030462946B7
:10F930005246254B984701370135FFB2EDB29BF88F
:10F9400000301E49CA5CBA42D7D801340136E4B24D
:10F95000F6B29BF800301A4AD35CA34202D9019D4B
:10F960000027ECE74546BAF1000F15D000260AE063
:10F97000009B019AE018B118C0B2C9B25246124BAE
:10F9800098470136F6B29BF800300C49CB5CB34285
:10F99000EED801E04FF00009103DEDB2092D04D87A
:10F9A0009BF80030064AD05C03E009F101095FFAD8
:10F9B00089F005B0BDE8F08FE8010020153C010892
:10F9C000DF3F0108DC01002081F700082DE9F0414C
:10F9D0001E4B1A781E4B9E5CA0F13003DBB2C6F1C1
:10F9E0000807092BFFB21B4B02D8985CBDE8F081D9
:10F9F0001F2803D95E2828BF5E2000E020209D5CE0
:10FA00002038C4B200206C43034617E0DFF848C03A
:10FA10005CF822C01CF8048001EB070C48FA0CFCCF
:10FA20000CF0010CBCF1000F18BF184601315FFA51
:10FA300081FCB445EAD30133DBB20134AB4201D0DF
:10FA40000021F4E70130C0B2BDE8F081E8010020F8
:10FA5000153C0108DF3F0108DC0100202DE9F047DB
:10FA600098469DF924609DF82030002EACBF0226F8
:10FA70000126012B82460C4615460CD00F461AE093
:10FA8000384621463246164B98470137FFB2AF42FF
:10FA9000F6D90134E4B244451FD85746F7E7394652
:10FAA00050463246DFF83890C84739462846324635
:10FAB000C8470137FFB24745F1D90CE0504621460F
:10FAC0003246074FB847504641463246B8470AF1DA
:10FAD000010A5FFA8AFAAA45F0D9BDE8F08700BFAB
:10FAE00081F700082DE9F04F8DB088469DF85C1035
:10FAF000572814460793089176DC079A1B0100F1FA
:10FB0000FF3A9B1AA24400250A935FFA8AFA8346B9
:10FB100006950B9039E03B4B0A995B189A5D42FAC7
:10FB200009F212F0010210D0059A5846D3190122A9
:10FB30000092FE32019202920392DBB239465246A3
:10FB4000314CA047099B06930EE0089961B10599D5
:10FB50000192CB1901210091029203925846394635
:10FB60005246DBB2284CA04709F101097F19B9F1CF
:10FB7000080FFFB2CFD12C46751CA344A2440F2D11
:10FB80005FFA8BFB5FFA8AFA0AD0631EEAB2DBB235
:10FB90002E460992059347464FF000092546BAE7DD
:10FBA000089BDDF82CC00BB305FB04C50599EEB22C
:10FBB0008F19FFB2059A09F1FF3902EB0803012200
:10FBC0000092013A019202920392414630463A462F
:10FBD000DBB20D4DA0445FFA89F9A8475FFA88F8B7
:10FBE000B9F1000FE6D101E00023069307995629E9
:10FBF00003D9069A501CC0B200E00F200DB0BDE83A
:10FC0000F08F00BFE23F01085DFA00082DE9F74FD1
:10FC10001F469DF934609DF83030002EACBF02269F
:10FC20000126012B04460D46924656D101F1010BE7
:10FC30005FFA8BFBD94611E004F1010806E040466B
:10FC400049463246454B984708F101085FFA88F863
:10FC5000C245F4DC09F101095FFA89F94F45EBDC93
:10FC600005F1020909E0494620463246C0474946A7
:10FC700050463246C04709F101095FFA89F97B1EF7
:10FC80004B45DFF8D880EEDC04F1020909E0484674
:10FC900029463246C047484639463246C04709F1F0
:10FCA00001095FFA89F90AF1FF334B45EFDC0134B2
:10FCB000E4B22046594632460193C047019B013FBA
:10FCC000DDB2FFB2284639463246C04720463946A3
:10FCD0003246C047284659463CE001F1020909E096
:10FCE000494620463246C047494650463246C047FC
:10FCF00009F101095FFA89F97B1E4B45DFF85C8049
:10FD0000EEDC04F1020909E0484629463246C047C4
:10FD1000484639463246C04709F101095FFA89F978
:10FD20000AF1FF3BCB45EFDC01340135E4B2EDB223
:10FD3000013F2046294632465FFA8BFBFFB2C0479F
:10FD4000584639463246C047204639463246C047B3
:10FD5000584629463246C047BDE8FE8F81F7000865
:10FD60002DE9F04F87B005939DF940300546049288
:10FD7000121A0598002BACBF0223012392B2039301
:10FD8000431A9BB297B250000C46590017F4004F2B
:10FD90009EB280B289B204D180B201904FF00108C6
:10FDA00006E04042574280B2BFB201904FF6FF7862
:10FDB00016F4004F04D189B202914FF0010B06E016
:10FDC00049425E4289B2B6B202914FF6FF7B2846A5
:10FDD0002146039ADFF89C90C8470FB9002E46D001
:10FDE00032B23BB29A42AA46A14620DC1FFA88F8FA
:10FDF0004544ADB20024029A2E46A418A3B29CB288
:10FE000021B23AB2914205DD0199D9445C1A1FFA38
:10FE100089F9A4B2E8B25FFA89F1039A154B9847C1
:10FE2000049836B245448642ADB2E4D11FE01FFAD1
:10FE30008BFB5C44A4B20025019932B26D18ABB2C1
:10FE40009DB229B29142274605DD029AC2449D1A0D
:10FE50001FFA8AFAADB25FFA8AF0E1B2039A054B53
:10FE6000984705983FB25C448742A4B2E4D107B0FA
:10FE7000BDE8F08F81F7000838B50546002404E09E
:10FE8000054B984701302418E4B215F8010B0028FF
:10FE9000F6D1204638BD00BFCDF90008F8B5094BB2
:10FEA00000241F7805461C701E4604E0064B984748
:10FEB00001302418E4B215F8010B0028F6D1377090
:10FEC0002046F8BDE8010020CDF900082DE9F743F0
:10FED0000E4B0E46002193F800800446197015461B
:10FEE000994609E000230093204631460333084F2A
:10FEF000B84701302418E4B215F8012B002AF1D1DB
:10FF000089F800802046BDE8FE8300BFE80100209C
:10FF1000ADF800080B4BF7B50E46012104461970E9
:10FF2000154609E000230093204631460333064F6F
:10FF3000B84701302418E4B215F8012B002AF1D19A
:10FF40002046FEBDE8010020ADF800082DE9F04391
:10FF500087B0884699469DF838609DF83C5001234B
:10FF600011B200220446009302A81346064FB84778
:10FF7000009601952046414602AA4B46034CA047F5
:10FF800007B0BDE8F08300BFF523000815FF0008A7
:10FF90002DE9F04F8DB09B469DF85830C2F1010617
:10FFA00009939DF85C304FF0010C002481468A468D
:10FFB0000A931546B6B20894E0465F46C4EB0903BF
:10FFC0005FFA85FBDBB20B93099A0A9B0BEB0A01E4
:10FFD00004EB090C5FFA8CFCC9B26046CDF814C082
:10FFE000019202930B9A0B46DFF8B8C00097E047E6
:10FFF000099A0A9BCBEB0A01C9B2019202930598B8
:020000040801F1
:100000000B460B9ADFF89CC00097E047099A0A9BC1
:10001000CBEB090CC4EB0A01CB445FFA8CFCC9B2F0
:100020005FFA8BFB6046CDF82CC0019202935A46D2
:100030000B46DFF870C00097E047099A0A9B04EB73
:100040000A01C9B20192029300970B985A460B46D7
:10005000DFF850C0E04716F4004F06D0089A033688
:1000600006EB4206B6B243460BE0DDF820C02BB2E9
:10007000C3EB0C03053606EB4306013DB6B243461F
:10008000ADB2089A1BB2013208922AB2013C08F1C3
:1000900001089342E4B21FFA88F88FDD0DB0BDE885
:1000A000F08F00BF61FD00082DE9F04F5BB289B011
:1000B000C2F10108002602900391002BACBF02247C
:1000C000012417461FFA88F84FF0010AB346029937
:1000D0005FFA87F98B1B0399DBB2069309EB0103E7
:1000E000DBB2354D1946069822460093A84702997F
:1000F00009EB0102D2B20492039A0498C6EB020CF7
:100100005FFA8CFC61462246CDF804C0A8470299EC
:10011000009B7218D2B21046194607922246A84791
:10012000029ADDF804C0C9EB0203DBB2614618464F
:1001300022460593A847039904987318DBB2194621
:1001400022460093A847039A0698C9EB02095FFA72
:1001500089F949462246A847079849462246A847B2
:10016000009B059819462246A84718F4004F07D06F
:1001700008F1030808EB4B081FFA88F853460BE018
:100180003BB2C3EB0B0308F1050808EB4308013F42
:100190001FFA88F85346BFB21BB23AB2013E0AF1C9
:1001A000010A93420BF1010BF6B21FFA8AFA8EDDB7
:1001B00009B0BDE8F08F00BF81F7000870476020EC
:1001C00070471A207047000008B500214FF49C7258
:1001D000014B0248984708BDE5100008F8040020CC
:1001E00008B50248024B984708BD00BFF80400203C
:1001F0007502010808B5024B9847002008BD00BFF2
:10020000B9020108704770472DE9F8434FF4806147
:10021000154E81461548B04709254FF48074B04605
:1002200012484FF48071C04714EA090F104F04D0F0
:100230000E484FF40071B84704E00C484FF40071C9
:10024000094B984709484FF48071B8476408013D4D
:10025000074EE5D105484FF40071B04703484FF40D
:100260008061B047BDE8F883A31901080018014078
:100270009F1901082DE9F041064640240D4D20202C
:10028000A8478320A8472046A847B046602798F88B
:100290005F00013F00F58070BFB2A84708F1FF384A
:1002A000002FF4D10134A4B26036442CE6D1BDE86D
:1002B000F08100BF0902010837B510238DF807301F
:1002C0000D3B02AC8DF806304FF4807324F8043DEA
:1002D000174D21461748A8474FF40073214615488B
:1002E000ADF80430A8474FF4806321461148ADF8BB
:1002F0000430A8474FF4006321460E48ADF804309F
:10030000A8474FF400610B480B4B984740F6B830B4
:100310000A4B984707484FF40061094B984700245F
:10032000084B185D084B01349847102CF8D13EBD9E
:10033000F518010800180140A31901084B05010830
:100340009F190108FB4401080902010810B52D4955
:100350002D4C2E48A0472E492E48A0472E4B98479B
:100360002E4B98474FF480302D4B98472D4B984794
:100370000128044628D110202B4B984702202B4BF4
:10038000984700202A4B984700202A4B98474FF463
:100390008060294B98474FF40040284B98474FF412
:1003A0004030274B4FF4801198472046254B984703
:1003B0003920254B98470028FAD00220234B984734
:1003C000234B98470828FBD101212248224B98470C
:1003D000012145F67D20214B984701200146204B05
:1003E000984700214FF000601E4B98474FF4407033
:1003F0001D4B98471D4B98471D4B98471D4B9847E1
:10040000002010BD9E220108E1110008A82C002048
:100410000B450108B82C00209D160108111A01088F
:10042000511A0108391C0108311E01081D1E01085E
:10043000D11A0108F91A0108E51A01080D1B010873
:10044000891A0108A11A0108111C0108AD1A010836
:10045000C11A010807403E00F91B0108E11B010811
:10046000C91B0108A921010835210108F506010869
:10047000F10801080505010808B5024B9847024B31
:10048000984708BDFD09010829070108034B4000F2
:1004900018800A234B43024A13807047DC03002074
:1004A000DA03002038B5002517E0114B1148402130
:1004B0009847238801E000BF013B9BB2002BFAD193
:1004C0000D4B0C4840219847238801E000BF013BB9
:1004D0009BB2002BFAD10135ADB2084B084C1A88FB
:1004E00092B29542E1D3002222801A8038BD00BF2B
:1004F0009F19010800100140A3190108DA03002028
:10050000DC03002007B510238DF807300D3B02A94E
:100510008DF80630402321F8043D0448044B9847E9
:1005200040F2E2400A21034B98470EBD0010014003
:10053000F51801088D0401084FF4FA53434301E014
:10054000013B00BF002BFBD1704701E0013800BF29
:100550000028FBD1704770477047000050FA01F146
:1005600050FA02F201F0010100290CBF0321002121
:1005700012F0010F08BF81F00101184110F0010FC6
:100580000FD00A4A13785B1A13F001000CD003F065
:100590000203013B002B117005DC0CBF0020012081
:1005A0007047022070470320704700BFDF03002020
:1005B000F8B5394C2388012B06D1384B4FF496609F
:1005C00014219847238800E00BB1013B2380344D70
:1005D00095F8423013B9043385F842304FF4006186
:1005E0003048314FB8474FF40051061E2D4818BF10
:1005F0000126B84710B146F00206F6B229484FF47A
:100600000051B84708B146F00406304600210122E7
:100610000223264EB04701280BD1254B95F84210F6
:100620001A7801321A7052B291424FF000022EDC59
:100630002BE003280DD11E4B95F842101A78C1F11A
:100640000101013A1A7052B28A424FF0000220DAD8
:100650001BE00228174B0BD193F9002012B94FF47D
:10066000C872228002221A70114B00201870F8BD47
:1006700093F90020022A0DD12088023A1A700C4BFF
:1006800000280CBF0420022022801A70F8BD1046FA
:10069000F8BD1046F8BD00BFE20300208D0401083C
:1006A000502C002000100140931901085D0501083D
:1006B000E0030020DE03002008B5094B984702281C
:1006C00008D0032808D0012808D004280CBF4420F3
:1006D000002008BD432008BD412008BD422008BDC0
:1006E000B1050108024B000183F82300704700BFE9
:1006F00000ED00E038B5094C4AF6C77363600F207F
:10070000074DA8470023A360073323606FF0040060
:10071000044B98470420A84738BD00BF10E000E014
:10072000E5060108BD2101087047000008B5014B2E
:10073000984708BDD10F01082DE9F043394EDFF885
:10074000388193B0002501350024EDB2022326F84C
:10075000024F354818F8011F2A46344FB847032D79
:10076000F1D12E46ADF844503148324D11A98DF8E3
:100770004740A847112311A9ADF844302E488DF801
:100780004740A8472D482E4B98472E4B2B480193A6
:100790002D4B01A9029330230493503306938033E9
:1007A00007934FF480630893202309930394274B06
:1007B00005940A940B94984720480121244B9847AC
:1007C00001254FF460230E9317480CA9214B0C947C
:1007D0008DF834508DF835500F948DF8406098475F
:1007E000114829461C4B98470F4829461B4B9847F0
:1007F00028461B4B98470C481A4B98470A481A4BF7
:1008000098470028FAD10848184B98470648184BD3
:1008100098470028FAD104480121164B984713B095
:10082000BDE8F083E203002000240140F51E01082A
:10083000000C0140F51801080010014008000240BA
:10084000C51C01084C240140E4030020C51D01081B
:10085000051E0108491E0108A91E0108951E010870
:10086000851F0108BD1E0108C71E0108CF1E010813
:10087000D91E0108E11E01081145010800231A468E
:10088000054901EB4001C95A0633602B0A44F7D1F0
:10089000120990B2704700BFE403002008B5014B75
:1008A000984708BD39070108022808B506D840B2A4
:1008B0000D4B9847A0F5FE600F3813E00F2810D9B4
:1008C000FF280ED0FE2809D03F280AD8074B400148
:1008D000C0188079142340B2584303E040F2FF70FF
:1008E00000E0002000B208BD7D08010808080020D3
:1008F00070B5802286B003251826394CADF8142037
:100900008DF816508DF8176005A93648A04740238A
:10091000ADF8143048238DF817308DF8165005A91E
:100920003048A0472022ADF814208DF816508DF8DD
:10093000176005A92B48A04710238DF816500135E4
:100940008DF81730ADF8145005A92648A0474FF48C
:10095000004629462348244DA847ADF8146005A950
:100960002248A04731462148A8474FF40053ADF82C
:10097000143005A91D48A0474FF48042ADF814205B
:1009800005A908261948A04705A9ADF8146015481F
:10099000A04700211648174CA0474FF4827200234D
:1009A000ADF802200222ADF80030ADF80430ADF809
:1009B000062001254FF40072ADF80E300723ADF884
:1009C00010306946ADF80850ADF80A20ADF80C605B
:1009D0000748094B984706482946A04706B070BD0E
:1009E000F5180108000801409F190108001801408E
:1009F00000300140A91C0108691C010808B5024823
:100A00000021024B984708BD00300140A91C010895
:100A100038B5044670B9084840F225512246074DC2
:100A2000A847054840F227712246A84702482146B8
:100A3000034B984738BD00BF003801406B180108D0
:100A40005118010870B5032386B08DF816300023C5
:100A50004824ADF80430ADF80630ADF80830ADF8F4
:100A60000C300C230646ADF80A308DF817401F4BAA
:100A70009847002E38D14FF48063ADF814308DF8CC
:100A800017401B481B4C05A9A0474FF40073ADF855
:100A9000143018238DF81730154805A9A04706A96A
:100AA0004FF4E13341F8183D13486946134B98471A
:100AB000012406A8252300F8083D8DF81140104BAD
:100AC0008DF812408DF8134098470E4D0A4840F2B9
:100AD00025512246A847084840F227713246A847C8
:100AE00005482146084B984706B070BD110A010819
:100AF00000080140F5180108003801409917010865
:100B0000492101086B1801085118010808B528B9D6
:100B1000034840F227710122024B984708BD00BFED
:100B2000003801406B180108024B002223F8102006
:100B3000704700BFA8070020F0B5002312E00B4C5F
:100B400011F8017B34F81050094EADB285EA070761
:100B500007F0FF0736F81760013386EA152524F8F9
:100B600010509BB29342EAD1F0BD00BFA80700200D
:100B7000204501082DE9F041184B044608460E4671
:100B800098474FF6FF73DFF86C8038F81470BFB2E7
:100B90001FB9022B05D8BDE8F081013BF3D1BDE8B8
:100BA000F08185B2B5F5967F15D26A1C2046314694
:100BB00092B20B4B98470B4B4FF4967000FB0430EE
:100BC0003146094B9847094B28F81450204623F822
:100BD0001470074B9847BDE8F08100BF9D120008D4
:100BE000390B01087A060020E11100087806002080
:100BF0000D0B0108A607002030B5012387B00022A5
:100C00000446009302A81346034DA847204602A9B4
:100C1000024B984707B030BDF5230008750B01085B
:100C200008B5034B33F81010024B09B2984708BDC2
:100C3000A8070020F90B010870B5184840F22551AB
:100C4000174CA047054628B1144840F22551154BD2
:100C5000984770BD114840F22771A047E8B1124C87
:100C60000E4840F227710F4B984723880F4A9BB2DA
:100C7000D15C0F4E0133238008480E4B98472288E1
:100C8000338892B29BB29A4207D1044840F227714E
:100C90002A46094B98473580258070BD00380140B1
:100CA000A9180108E9180108780600207A06002032
:100CB000A6070020A11801086B18010830B5012112
:100CC0008BB02648264B98474FF48073ADF82430FC
:100CD00018238DF82730153B09A98DF826302148B7
:100CE000214B98471D2301248DF820301B3B8DF8A4
:100CF00021308DF8223008A88DF823401B4B9847EF
:100D00004FF0FF330025ADF818301123ADF8143043
:100D100005A9ADF81A50ADF816501548154B98476F
:100D20003023ADF804304FF47A73ADF80A3001A9DE
:100D3000ADF80640ADF80C500D480F4B98472946CA
:100D40000B480E4B9847214609480D4B98470848D9
:100D5000082122460B4B98470BB030BD000C1A00FF
:100D6000A919010800100140F518010849210108DE
:100D700000040040A11F010849200108FD200108CE
:100D8000CD200108E72001087047000030B500239E
:100D900014E00D4D32F9020B05F50E543E34248853
:100DA000A4B26408444340F2FF7094FBF0F403F5EE
:100DB0008E501C3005EB400004810133D8B28842CC
:100DC00001D2102BE5D130BDD00700202DE9F8432A
:100DD0006E4808216E4B9847002800F0D580082106
:100DE0006A486C4B98476C4B684898476B4C6C4B07
:100DF00020804FF480716B48984722466A4B08B1B7
:100E0000002100E001216948197090F8351001298E
:100E100003D11978C1F1010119701978644D654B3E
:100E200079B9018F1288644C89B2218002EB81016B
:100E3000564889B298472B882288D3182B80BDE862
:100E4000F8835E4C90F834002778DFF878E1874229
:100E50000EF50E51264680F08A800EF51050447B28
:100E6000A742554C61D1DFF860C190F80F809CF823
:100E70000070474519D2B1F83C90B1F8388007F5B9
:100E8000905104310EEB410109891FFA89F909B229
:100E90000029B8BF03311FFA88F88910C8EB090E82
:100EA00001EB4101714421801FE090F80FE0BE4545
:100EB0001FDB807B50B9888FB1F838E0C98F1FFAEB
:100EC0008EFE89B2CEEB510109180DE0B1F83C80DD
:100ED000B1F838E0C88F1FFA88F81FFA8EFE80B28A
:100EE000CEEB0801A1EB5001218001378CF8007096
:100EF0002DE0807B40B9888F0F8FC98FBFB289B238
:100F0000C7EB510109180BE0B1F83CE00F8FC88F17
:100F10001FFA8EFEBFB280B2C7EB0E01A1EB5001EB
:100F2000218000218CF8001011E0B1F83C80B1F86C
:100F300038C007F58E511C310EEB410108891FFAAC
:100F400088F81FFA8CFCCCEB080109182180128864
:100F500021880E4802EB810189B298472B882288AC
:100F6000D3182B80337801333370BDE8F883498F71
:100F7000128889B202EB8101044889B298470023A4
:100F800023702B800E4B9847BDE8F8830004004087
:100F9000192101082F21010813210108460400200E
:100FA000931901080010014045040020502B002037
:100FB0004A0400200F2101084C04002048040020AE
:100FC00035100108D00700204404002070470000BD
:100FD00038B5114C114D636CA4F1200005336364E6
:100FE000A847012804D154F8243C053344F8243C94
:100FF0000B48A847012803D10A4B5A6E05325A669E
:10100000094B1B78012B05D1084C237813B9084BE9
:101010009847207038BD00BF502C0020C11E00082A
:10102000382C0020D02B0020560400204E04002035
:10103000B906010808B5024B9847024B984708BD0E
:10104000852400086D1F000870B5294886B0294B1B
:101050009847294B9847294B9847294B9847294B44
:101060000020294C984700202849A0470020284903
:10107000A04700221346012503A842F20871254E1D
:101080000095B047002003A9A04700202249A047AF
:10109000224B984700202249A047224B9847002026
:1010A0002149A047214B2248984700202149A047C9
:1010B000214B984700202149A04700202049A04704
:1010C000204B9847204B984700202049A047204BB1
:1010D000984720490020A04700201F4B98472846EA
:1010E0001E4B984700201E49A04706B070BD00BFA8
:1010F000D0070020811D0008412000084D03010891
:10110000A5040108450A0108750B010820470108DC
:1011100031470108F52300080A270108F5010108F5
:101120003C470108B1400008404701083D45000820
:101130004447010850470108E101010854470108EC
:101140005D4701089D08010857050108634701082C
:10115000070201086A470108BD0C0108890D010852
:1011600070470108F8B5104E104FB047104CB84703
:10117000104D1148A847A047104B9847B847104852
:10118000A847A0470F4D4FF47A70A847B047A04733
:101190000D4B98476420A8470C4B984700200C4BF8
:1011A00098470C4B9847F8BDC9010108B1400008A9
:1011B000E10101083D45000878470108C12C0008FD
:1011C000874701083905010805020108590501088A
:1011D000110A0108790401082DE9F041454B464CFC
:1011E00000250122257028461A704449444EB04714
:1011F000444B1D72803B93F84320012A03D12846BB
:101200004149B04768E093F84330022B64D1284647
:101210003E49B0475AE01A78002A39D01A781A782D
:10122000412A02D01A78482A02D14FF4487027E0A8
:101230001A78422A02D01A78502A02D14FF46170EB
:101240001EE01A78432A05D01A780A2A02D01A78A2
:101250000D2A02D14FF47A7012E01B78442B02D190
:1012600040F24C400CE02278234B712A32D01A789D
:10127000952A08D91A78C72A05D81B784FF4FA702E
:101280000A21234B9847234B0A20984700232370B9
:10129000214BDFF8B0809847C047204D204F297878
:1012A0002A78401A15F8023C0021C0B2B847C0475E
:1012B0000246002015F8023C01461A4DA8471A4B79
:1012C00098471A4BFF221A70194B984722780A4BFD
:1012D000712AA0D10023237016490020164DB04773
:1012E000164CA8471648A047A8471548A047BDE890
:1012F000F08100BF560400204E04002093470108EF
:10130000750B0108D02C00209A470108A547010859
:101310008D04010839050108B14000088B2C00201C
:10132000813D00084D410008E1010108E90100206C
:10133000A50401087047010885240008A5240008B9
:10134000FC070020BF0101082DE9F74F674B9847C4
:10135000674B984767496848684AFF23684E03709F
:101360000B701370FF3B3370664B01241C708B466F
:101370002DE11A78002A52D0634CB4F9002002B94A
:101380001A70327832785E4B412A02D01A78482A95
:1013900005D15E4B02221A704FF4487034E01A787F
:1013A000422A02D01A78502A05D1584B01221A70CD
:1013B0004FF4617028E01A78432A05D01A780A2A77
:1013C00002D01A780D2A05D1504B03221A704FF41F
:1013D0007A7019E01A78442A05D14C4B403A1A70B9
:1013E00040F24C4010E01A78712A00F0F5801B782A
:1013F000952B0CD93378C72B09D8414B4FF4FA7091
:101400001A78424B323A1A700A21414B9847414BA5
:101410000A209847002342F2107133702180022085
:101420003D4B98473D4BDFF8209119785A78484357
:101430000A2190FBF1F052B201FB0202A9F8002050
:10144000B9F800209B7892B2B2FBF1F29A4203D233
:101450004FF461702E4B9847314B1B785BB1274B93
:101460001A783F2A07D81A780A218BF800202D4ACB
:101470001170FF221A702C4FDFF8D0A0D047B84768
:101480002A4C2B4D21782278401A14F8023C002176
:10149000C0B2A847B8470246002014F8023C0146F3
:1014A000244CA047244CDFF86480237823B998F8B3
:1014B0000000224B98474CE0022B4FF0000547D02C
:1014C000032B45D0042B43D002AAFF2302F8015D71
:1014D0001B4898F800101B4FB847012839D19DF8D8
:1014E0000730042B34D1257076E000BF4910010885
:1014F000D9110108EC010020E9010020ED010020D4
:101500004E04002056040020EA010020530400206D
:101510008D040108390501087D080108802C002090
:10152000912C002054040020BF0101088B2C0020C6
:10153000813D00084D4100085204002031E80008B8
:10154000682A0108D592000850040020B140000824
:101550002570002388F80030224B1A7852B1013AE6
:101560009BF800001A70204B4201D31899791F4B49
:1015700049B298471E4C237853B11E4B1E48214652
:1015800098471E4B1A78013A1A701B7803B92370DA
:10159000B9F8002040F6736392B29A42184C10D802
:1015A0001848194B9847D0470521184B4FF49660BF
:1015B0009847A047164B1A8811B20A2901DD0A3A4A
:1015C0001A80144B9847144AFF231370A0473278AF
:1015D000124B712A7FF4CDAE114B98470020BDE825
:1015E000FE8F00BF5404002008080020B945000801
:1015F000AC07002055470008B247010855040020F9
:10160000A5040108BB470108A13E00088D0401089C
:10161000EA010020E1010108E90100204E04002058
:10162000651101080A4A0B4B9A4205D10A4B0AE0A0
:1016300052F8041B43F8041B08498B42F8D3F5E722
:10164000002243F8042B064A9342F9D3704700BFA7
:10165000D448010800000020FC020020FC02002009
:10166000D82E0020684620F007018D4601B50023E2
:1016700082B001E0019B01330193019A034B9A422E
:10168000F8D9034B9847034B9847FEE71FA1070083
:101690002516010849130108FEE700003A4B82B005
:1016A0001A6842F001021A605968384A01EA0202D7
:1016B0005A601A6822F0847222F480321A601A6822
:1016C00022F480221A605A6822F4FE025A604FF413
:1016D0001F029A600022019200921A6842F480323E
:1016E0001A60294B1B6803F400330093019B0133FC
:1016F0000193009B1BB9019BB3F5A06FF1D1224B65
:101700001B6813F4003318BF01230093009B012BC7
:1017100034D11F4B1A6842F010021A601A6822F086
:1017200003021A601A6842F002021A60164B5A68E5
:101730005A605A685A605A6842F480625A605A681D
:1017400022F47C125A605A6842F4E8125A601A680D
:1017500042F080721A600C4B1A6812F0007FFAD0C7
:101760005A6822F003025A605A6842F002025A6034
:10177000054B5B6803F00C03082BF9D1054B4FF0C8
:1017800000629A6002B07047001002400000FFF84B
:101790000020024000ED00E0038ACA8823F4405391
:1017A0001B041B0C134330B503820D468389098942
:1017B000AA8823F4B05341EA0202698923F00C039A
:1017C0000A431B041B0C92B242EA03038381838AFF
:1017D000AA8923F440731B041B0C87B013430446EF
:1017E0008382194B01A89847184BA2899C4212B2D8
:1017F0000CBF049B039B002A4FF019012A6802DAF0
:101800005943520001E0594392006423B1FBF2F1C5
:10181000B1FBF3F21201100903FB1011A08900B211
:10182000002806DAC9003231B1FBF3F303F00703F5
:1018300005E009013231B1FBF3F303F00F0343EA92
:101840000202228107B030BD211B0108003801408F
:1018500021B183899BB243F4005304E0838923F4CC
:1018600000531B041B0C83817047CBB210B55B097E
:10187000012401F01F0114FA01F1A34201D10C303F
:1018800004E0022B01D1103000E014301AB10368DB
:1018900043EA010102E0036823EA0101016010BD8F
:1018A000C905C90D8180704710B5CCB20122640909
:1018B00001F01F039A40012C01D1838903E0022C1F
:1018C0000CBF038A838A9BB202EA0303028892B2A6
:1018D00043B1090A012313FA01F111420CBF0020A0
:1018E000012010BD184610BD090A01238B40DB43BF
:1018F00003807047CB78F0B513F0100F03F00F02A0
:101900000E881CBF8B781A4316F0FF0F1DD0046899
:10191000002301279F4007EA0605BD4211D19F0021
:101920004FF00F0C0CFA07FC12FA07F724EA0C042C
:101930003C43CF78282F01D1456102E0482F08BFF2
:1019400005610133082BE4D104600E88FF2E1FD9F6
:101950004468002303F108050127AF4007EA0605A4
:10196000BD4211D19F004FF00F0C0CFA07FC12FA88
:1019700007F724EA0C043C43CF78282F01D14561B6
:1019800002E0482F08BF05610133082BE2D1446013
:10199000F0BD836819420CBF00200120704701612F
:1019A00070474161704700000028184B30B500F4C3
:1019B0004014B4BFDB695B68B4F5401F82B207D145
:1019C000124C23F07063656825F07065656011E066
:1019D00010F4801F06D000F47024240C032515FA9F
:1019E00004F403E0440D240112FA04F423EA04038E
:1019F00043F0706319B1410D09018A401343034A52
:101A00000028B4BFD361536030BD00BF0000014067
:101A10000D4B1A6842F001021A6059680B4A01EA3C
:101A200002025A601A6822F0847222F480321A602C
:101A30001A6822F480221A605A6822F4FE025A6060
:101A40004FF41F029A607047001002400000FFF838
:101A50000C4BB0F5803F1A6822F480321A601A6885
:101A600022F480221A6003D0B0F5802F09D104E05F
:101A70001A6842F480321A6070471A6842F4A02251
:101A80001A60704700100240044B5A6822F47C121E
:101A900040EA02020A435A60704700BF0010024049
:101AA000014B1860704700BF60004242034B5A6808
:101AB00022F0030240EA02025A607047001002401E
:101AC000024B586800F00C00704700BF0010024045
:101AD000034B5A6822F0F00240EA02025A60704753
:101AE00000100240034B5A6822F4E06240EA02020E
:101AF0005A60704700100240034B5A6822F460524B
:101B000042EAC0025A60704700100240034B5A6814
:101B100022F4404240EA02025A607047001002403C
:101B2000224B10B55A6802F00C02042A03D0082A8E
:101B300004D01F4B00E01F4B036012E05A68596845
:101B400002F47012920C023211F4803F01D11A4B50
:101B500005E05B6813F4003F14BF184B154B5A4364
:101B60000260124B16495A68046802F0F00212092A
:101B70008A5C34FA02F242605C6804F4E064240A8D
:101B80000C5D32FA04F484605C6804F46054E40A86
:101B9000095DCA40C2605B680A4903F440439B0B7D
:101BA000CB5CB2FBF3F2026110BD00BF001002403B
:101BB00000127A0040787D0100093D0020BCBE0083
:101BC000F3010020EF010020044B11B15A691043CA
:101BD00002E05A6922EA0000586170470010024092
:101BE000044B11B19A69104302E09A6922EA00009D
:101BF0009861704700100240044B11B1DA6910433C
